:10000000F6C5000025C6000023C6000021C600007A
:100010001FC600001DC600001BC6000019C6000058
:1000200017C6000015C6000013C6000011C6000068
:100030000FC600000C948E4F0BC6000009C60000CE
:1000400007C600000C94687003C6000001C60000DB
:10005000FFC50000FDC50000FBC500000C94EA4B85
:10006000F7C500000C94A96E0C94806EF1C50000D9
:10007000EFC50000EDC50000EBC50000E9C50000BC
:100080000C943A70E5C50000E3C50000E1C500002E
:100090000C94566E0C942D6EDBC500000C943A50F7
:1000A000D7C50000D5C500000C940C70D1C5000068
:1000B000CFC50000CDC50000CBC500000C94DE6F9D
:1000C000C7C50000C5C50000C3C500000C94036E81
:1000D0000C94DA6DBDC500000C94B06D0C94876D66
:1000E000B7C50000267E297E187E1C7E227E607E9B
:1000F0002D7E317E377E3B7E3F7E457E497E4D7E26
:10010000607E537E577E5B7E4E414E494E49545928
:10011000494E46CDCCCC3D0AD7233C17B7D13877D2
:10012000CC2B329595E6241FB14F0A0000204100E8
:1001300000C84200401C4620BCBE4CCA1B0E5AAE32
:10014000C59D7400407A10F35A00A0724E18090041
:1001500010A5D4E80000E87648170000E40B54022C
:100160000000CA9A3B000000E1F505000080969867
:1001700000000040420F000000A0860100000010B7
:100180002700000000E803000000006400000000F9
:10019000000A00000000000100000000002C76D8DA
:1001A00088DC674F0823DFC1DFAE59E1B1B796E5C0
:1001B000E3E453C63AE651997696E8E6C28426EB24
:1001C000898C9B62ED407C6FFCEFBC9C9F40F2BA37
:1001D000A56FA5F490055A2AF75C936B6CF9676DCF
:1001E000C11BFCE0E40D47FEF520E6B500D0ED9024
:1001F0002E0300943577050080841E080000204EF1
:100200000A000000C80C333333330F986E12831189
:1002100041EF8D2114893BE65516CFFEE6DB18D160
:10022000844B381BF77C1D901DA4BBE42420328432
:10023000725E228100C9F124ECA1E53D2746696E7A
:1002400064696E672057694669204950004E4554DD
:100250003D426C7565746F6F7468204C45004E4567
:10026000543D426C7565746F6F7468004E45543D23
:100270005769466900696E70757420445354636110
:100280006C6962726174653A005344206F70656EE8
:10029000206661696C004E6577206461746120633B
:1002A0006F6C6C656374696F6E20737461727465D2
:1002B000640043757272656E742073657474696E40
:1002C00067733A0053797374656D20726573657452
:1002D000206174200023445320546865726D6F6D53
:1002E000657465722063616C696272617465642013
:1002F000666F72202300496E76616C696420616EBE
:10030000676C6520666F72200020737465707320BF
:1003100070657220616E676C653D00207374657056
:10032000732070657220616E676C653D002020202F
:10033000202020202020202020202020200057695D
:1003400046692049503A004C6F67676572204E61DC
:100350006D653A20005265626F6F74696E672E2E6C
:100360002E0074696D6520696E74657276616C3DEE
:100370000053797374656D2072657374617274656E
:100380006421002053797374656D20726573746104
:1003900072746564210023436F6D6D616E6440006B
:1003A00054657374204C616D70732F46616E7300D9
:1003B0004448435020537563636573730044484356
:1003C00050204641494C454400776562736572761A
:1003D0006572202E2E2E006572726F72206F70650E
:1003E0006E696E672066696C653A20004C616D70BD
:1003F000204F74686572002354696D6520202020A9
:1004000020204461746520202020205365636F6E96
:10041000647320506F6C61726F6964205461626C08
:10042000652054286F43292048282529202000646E
:100430006F6E652100696E69742E20646F6E652E83
:1004400000534420696E69742E206661696C65648E
:100450002100696E69742E206661696C65642100F3
:1004600057656C636F6D6520746F20456455484B0C
:1004700000496E697469616C697A696E67205344DA
:1004800020636172642E2E2E0075706C6F61642083
:10049000627920465450206661696C65642100755C
:1004A000706C6F616420627920465450204F4B215C
:1004B00000485454502F312E3020343030204261C7
:1004C0006420526571756573740D0A5365727665A3
:1004D000723A205765626475696E6F2F312E370D41
:1004E0000A436F6E74656E742D547970653A20748A
:1004F0006578742F68746D6C0D0A0D0A3C68313E86
:1005000045504943204641494C3C2F68313E004804
:100510005454502F312E3020323030204F4B0D0AA2
:100520005365727665723A205765626475696E6FBD
:100530002F312E370D0A4163636573732D436F6E40
:1005400074726F6C2D416C6C6F772D4F7269676997
:100550006E3A202A0D0A436F6E74656E742D5479BD
:1005600070653A2000417070656E64206D6561733E
:100570002E200053696E676C65206D6561732E20B7
:100580000053617665206D65617375726520746FC7
:100590003A00436F6E6E656374696F6E3A20636CE8
:1005A0006F73650D0A436F6E74656E742D547970A8
:1005B000653A206170706C69636174696F6E2F7841
:1005C0002D7777772D666F726D2D75726C656E6302
:1005D0006F64656400506F7374206661696C656454
:1005E0000055706C6F6164204661696C65643A20E7
:1005F000003C703E4C616D7020616E64204F7468E9
:10060000657220537461747573EFBC9A3C2F703E11
:10061000003C68313E43616E6E6F742067657420E4
:1006200073656E736F722072656164696E677321A2
:100630003C2F68313E003C21646F63747970652003
:1006400068746D6C3E3C68746D6C3E3C68656164BA
:100650003E3C6D65746120636861727365743D2210
:100660007574662D38223E3C7469746C653E4F6E1D
:100670006C696E65206578706572696D656E742051
:100680006F6E20706F6C6172697A6174696F6E2031
:100690006F66206C696768743C2F7469746C653E82
:1006A0003C2F686561643E3C626F64793E3C683112
:1006B0003E4F6E6C696E65206578706572696D6518
:1006C0006E74206F6E20706F6C6172697A617469EC
:1006D0006F6E206F66206C696768743C2F68313ECE
:1006E000002346616E7320737769746368656420C4
:1006F0006F6E20666F7220002348656174657220FA
:100700007377697463686564206F6E20666F72200A
:10071000000000010001001010020001000100B003
:10072000000000160000002800000010000000205B
:1007300000000001000100000000000000000000B7
:1007400000000000000000000000000000000000A9
:10075000000000FF000000FFFF0000FFFF0000FF9F
:10076000FF0000CFBF0000C7BF0000C3BF0000C133
:10077000BF0000C0BF000000000000C0BF0000C1FB
:10078000BF0000C3BF0000C7BF0000CFBF0000FF15
:10079000FF0000FFFF00000000000000000000005C
:1007A0000000000000000000000000000000000049
:1007B0000000000000000000000000000000000039
:1007C0000000000000000000000000000000000029
:1007D00000000000000000557365722D6167656EB2
:1007E000743A202A0D0A446973616C6C6F773A2061
:1007F0002F0D0A004E6574776F726B206D61696E04
:100800007461696E65642061742000005EBCE26101
:100810003FDD83C29C7E20A3FD1F41009D23BE4679
:10082000DB65F88C11AF32CA57E9747C3C3E5E2B15
:100830003D3F2F5B5D3B2C2A225C000000220025FF
:100840000028002B002E00310034000201000005BA
:100850000108010B0100002100240027002A002DBF
:10086000003000330001010000040107010A01010A
:1008700002102020080810204010204080020102B1
:100880000108040201010204081020408080402079
:1008900010080402018004020180402010080402B4
:1008A0000108040201010204081020408001020432
:1008B00008102040800505050507050808080802FE
:1008C0000202020A0A0808040404040101010101E9
:1008D0000101010303030303030303040707070CD8
:1008E0000C0C0C0C0C0C0C0202020206060606068E
:1008F0000606060B0B0B0B0B0B0B0B495020616410
:1009000064726573733A20003C68343E436F7079BB
:100910007269676874284329323031382D32303299
:100920003020456455484B204861732043656E7400
:1009300072652E3C2F68343E3C2F626F64793E3CDA
:100940002F68746D6C3E0020202020202020202065
:1009500020202020202020002020202020202020B7
:1009600020202020202020200020202020202020A7
:100970002020202020202020200020202020202097
:100980002020202020202020202000496E76616C2D
:10099000696420534D2073746570732070657220F4
:1009A000616E676C653D00534D20737465707320F4
:1009B00070657220616E676C653D00000020002349
:1009C00000260029002C002F003200000100000347
:1009D000010601090100000A0B02090C0D0E0807AF
:1009E00003040100000000000000000000000000FF
:1009F00000000000000000000000000000000000F7
:100A000000121110000000000000000000000000B3
:100A10000000000000000000000000234E6F207363
:100A2000656E736F7220666F722074656D7020261C
:100A30002068756D696469747921004E6F20536573
:100A40006E736F72210020666F722074656D702066
:100A5000262068756D696469747921002353656E79
:100A6000736F72204572726F72200053656E736FE0
:100A700072204572726F7221002357726F6E672069
:100A800073656E736F7220666F722074656D70206F
:100A9000262068756D6964697479210057726F6EDC
:100AA000672053656E736F7221004320483D0054E8
:100AB0003D00202020202020202020202020202039
:100AC0002020002020202020202020202020202046
:100AD0002020002020202020202020202020202036
:100AE000202000506172616D6574657273207265BB
:100AF00073657420646F6E6521007365737573652B
:100B0000722F736D6C69676874706F2F73312F006B
:100B100043757272656E7420534D206973202300F3
:100B2000534D3A5461626C65207374657073207024
:100B3000657220616E676C653D00534D3A506F6C75
:100B400061726F69642073746570732070657220C0
:100B5000616E676C653D00234448543D00236E651B
:100B6000743D424C4500236E65743D5769466900EB
:100B7000236E65743D42540023667470207573655E
:100B8000726E616D653A00236674702073657276CB
:100B900065722049503A002352656C617920646582
:100BA00076696365733A002352656C6179207374CA
:100BB00061747573206C6162656C733A2000235216
:100BC000656C6179207374617465733A00235265B2
:100BD0006C61792070696E733A00234E6F2E206F1E
:100BE000662072656C6179733D0053A51DAA1124BE
:100BF0001FBECFEFD1E2DEBFCDBF00E00CBF1AE0D9
:100C0000A0E0B2E0E2EAF2E701E00BBF02C0079029
:100C10000D92A43DB107D9F729E1A4EDBAE001C0D6
:100C20001D92A130B207E1F715E0C6EFD5E000E074
:100C300006C021970109802FFE010E94B5B3C53F70
:100C4000D10780E00807A9F70E949A910C9440B957
:100C5000D7C92F923F924F925F926F927F928F925D
:100C60009F92AF92BF92CF92DF92EF92FF920F933B
:100C70001F93CF93DF93CDB7DEB7C055D1090FB621
:100C8000F894DEBF0FBECDBF69E076E1CE018F5B89
:100C90009F4F0E94306C23960EAD1FAD2397011518
:100CA000110569F0D8018C91882349F0082E000CB9
:100CB000990B0E94DDB5F80181938F01F3CF6DE6AA
:100CC00074E0CE0101960E94386CBE016F5F7F4FC9
:100CD000CE018F5B9F4F0E94633E182FCE0101967D
:100CE0000E94A86B112309F4C4C045E050E069E0FC
:100CF00076E1CE0101960E948C36BE016F5F7F4F78
:100D00008BEE95E10E94C56ACE0101960E94A86B08
:100D10008BEE95E10E94FE6960E08BEE95E10E940A
:100D20009E6A4091EF155091F0156CE677E18BEEDD
:100D300095E10E942D3E69E874E0CE0101960E9483
:100D4000386CBE016F5F7F4F8BEE95E10E94633E72
:100D5000182FCE0101960E94A86B112319F063E7AA
:100D600074E002C068E774E0CE0101960E94386C1E
:100D70006BEE75E1CE0101960E94286BBC0186E600
:100D800098E10E94936BCE0101960E94A86B86E6C3
:100D900098E10E94FE6940916A1850916B18415089
:100DA000510966E678E1CE0101960E948C36BE01BB
:100DB0006F5F7F4F88E498E10E94C56ACE0101967B
:100DC0000E94A86B88E498E10E94344C0E94FBB01A
:100DD0009B01AC010E9492B3882309F4A6C06091E4
:100DE0006A1870916B186250710986E698E10E944A
:100DF0005E6A682FCE0101960E94086CBE016F5F8B
:100E00007F4F88E498E10E94C56ACE0101960E9456
:100E1000A86B69E874E0CE0101960E94386CBE01AF
:100E20006F5F7F4F88E498E10E94633E182FCE01E8
:100E300001960E94A86B112309F477C060916A188B
:100E400070916B186350710986E698E10E945E6AA2
:100E5000682FCE0101960E94086CBE016F5F7F4F24
:100E600088E498E10E94C56ACE0101960E94A86BB1
:100E70005CC06BE874E0CE0101960E94386CBE0144
:100E80006F5F7F4FCE018F5B9F4F0E94633E182F95
:100E9000CE0101960E94A86B112309F458C045E0C9
:100EA00050E069E076E1CE0101960E948C36BE01E9
:100EB0006F5F7F4F8BEE95E10E94C56ACE01019670
:100EC0000E94A86B8BEE95E10E94FE6960E08BEEBC
:100ED00095E10E949E6A4091EF155091F01564E4EF
:100EE00077E18BEE95E10E942D3E64E477E1CE013F
:100EF0004C960E94386C61E974E0CE0101960E9424
:100F0000386CBE01645E7F4FCE0101960E94286B53
:100F1000BC0180E698E10E94936BCE0101960E948D
:100F2000A86BCE014C960E94A86B84EF91E0909341
:100F3000AC028093AB0264E177E10E94479064E6E3
:100F400070E080E090E00E9441820C94622967E9A1
:100F500074E0CE0101960E94386CBE016F5F7F4F36
:100F6000CE018F5B9F4F0E94633E182FCE010196EA
:100F70000E94A86B1123E1F043E050E069E076E1C4
:100F8000CE0101960E948C36BE016F5F7F4F8BEEC3
:100F900095E10E94C56ACE0101960E94A86B6BEE96
:100FA00075E1CE0101960E94306CCE010196BBCF57
:100FB0006BE974E0CE0101960E94386CBE016F5F50
:100FC0007F4FCE018F5B9F4F0E94633E182FCE0153
:100FD00001960E94A86B112301F144E050E069E002
:100FE00076E1CE0101960E948C36BE016F5F7F4F85
:100FF0008BEE95E10E94C56ACE0101960E94A86B16
:101000008BEE95E10E94344C7093D3176093D21706
:10101000709388026093870288CF60EA74E0CE0103
:1010200001960E94386CBE016F5F7F4FCE018F5BCF
:101030009F4F0E94633E182FCE0101960E94A86B1D
:101040001123E1F045E050E069E076E1CE01019640
:101050000E948C36BE016F5F7F4F8BEE95E10E9440
:10106000C56ACE0101960E94A86B8BEE95E10E94A5
:10107000344C70932F1860932E1831C066EA74E0D8
:10108000CE0101960E94386CBE016F5F7F4FCE018A
:101090008F5B9F4F0E94633E182FCE0101960E94E6
:1010A000A86B112309F44AC044E050E069E076E1FE
:1010B000CE0101960E948C36BE016F5F7F4F8BEE92
:1010C00095E10E94C56ACE0101960E94A86B8BEE45
:1010D00095E10E94344C709331186093301884EF7E
:1010E00091E09093AC028093AB0264E177E10E94BF
:1010F000479064E670E080E090E00E94418266EDF7
:1011000076E0CE0101960E94386C69E076E1CE016E
:1011100001960E94286BBC01CE014C960E94306C57
:10112000CE014C960E94DA83CE014C960E94A86BA9
:10113000CE0101960E94A86B0C9462296BEA74E0C0
:10114000CE0101960E94386CBE016F5F7F4FCE01C9
:101150008F5B9F4F0E94633E182FCE0101960E9425
:10116000A86B1123A1F044E050E069E076E1CE01E4
:1011700001960E948C36BE016F5F7F4F8BEE95E12A
:101180000E94C56ACE0101960E94A86BB2CF60EBA7
:1011900074E0CE0101960E94386CBE016F5F7F4FF4
:1011A000CE018F5B9F4F0E94633E182FCE010196A8
:1011B0000E94A86B111115C068EB74E0CE01019676
:1011C0000E94386CBE016F5F7F4FCE018F5B9F4FD7
:1011D0000E94633E182FCE0101960E94A86B112336
:1011E000A1F047E050E069E076E1CE0101960E946F
:1011F0008C36BE016F5F7F4F8BEE95E10E94C56A12
:10120000CE0101960E94A86B9ACE60EC74E0CE01EC
:1012100001960E94386CBE016F5F7F4FCE018F5BDD
:101220009F4F0E94633E182FCE0101960E94A86B2B
:10123000112321F081E00E943F3581CE6AEC74E0F9
:10124000CE0101960E94386CBE016F5F7F4FCE01C8
:101250008F5B9F4F0E94633E182FCE0101960E9424
:10126000A86B112319F00E945D7769CE61ED74E0DF
:10127000CE0101960E94386CBE016F5F7F4FCE0198
:101280008F5B9F4F0E94633E182FCE0101960E94F4
:10129000A86B112309F451C04AE050E069E076E1FF
:1012A000CE0101960E948C36BE016F5F7F4F8BEEA0
:1012B00095E10E94C56ACE0101960E94A86B8BEE53
:1012C00095E10E94344C0E94FE4D0E94254E609391
:1012D000A90C7093AA0C8093AB0C9093AC0C0E9459
:1012E000254E6093AD0C7093AE0C8093AF0C909331
:1012F000B00CCE014C960E944A376CED74E0CE01E2
:1013000001960E94386CBE01645E7F4FCE0101964B
:101310000E94286BBC01CE018A960E94306CCE01DF
:101320008A960E94DA83CE018A960E94A86BCE012B
:1013300001960E94A86B0C94BE116AE476E0CE017F
:1013400001960E94386CBE016F5F7F4FCE018F5BAC
:101350009F4F0E94633E182FCE0101960E94A86BFA
:10136000112309F467C045E050E069E076E1CE0161
:1013700001960E948C36BE016F5F7F4F8BEE95E128
:101380000E94C56ACE0101960E94A86B0E94254E5C
:101390006093A90C7093AA0C8093AB0C9093AC0C47
:1013A0008BEE95E10E94344C6093990270939A02FF
:1013B00080939B0290939C0260931418709315186D
:1013C00080931618909317182091131820933E0BB2
:1013D000672B682B692B11F410923E0B84EF91E080
:1013E0009093AC028093AB0264E177E10E94479056
:1013F00064E670E080E090E00E94418262E673E083
:10140000CE0101960E94286CCE0101960E943B7C81
:10141000CE0101960E94A86B4091990250919A02C8
:1014200060919B0270919C02CE0101960E947D7C8E
:101430000C94C7266DEE74E0CE0101960E94386CC4
:10144000BE016F5F7F4FCE018F5B9F4F0E94633E57
:10145000182FCE0101960E94A86B1123D9F14AE002
:1014600050E069E076E1CE0101960E948C36BE0123
:101470006F5F7F4F8BEE95E10E94C56ACE010196AA
:101480000E94A86B8BEE95E10E94344C613071058F
:101490008105910519F481E0809313188BEE95E195
:1014A0000E94344C672B682B692B11F4109213188F
:1014B0008091131880933E0B882309F410CE0E946C
:1014C000254E6093A90C7093AA0C8093AB0C90935B
:1014D000AC0C05CE68EF74E0CE0101960E94386C2A
:1014E000BE016F5F7F4FCE018F5B9F4F0E94633EB7
:1014F000182FCE0101960E94A86B112359F148E0E4
:1015000050E069E076E1CE0101960E948C36BE0182
:101510006F5F7F4F8BEE95E10E94C56ACE01019609
:101520000E94A86B8BEE95E10E94344C61307105EE
:101530008105910519F481E08093B10C8BEE95E162
:101540000E94344C672B682B692B09F0D8CD109280
:10155000B10CD5CD61E075E0CE0101960E94386CEA
:10156000BE016F5F7F4FCE018F5B9F4F0E94633E36
:10157000182FCE0101960E94A86B112339F145E086
:1015800050E069E076E1CE0101960E948C36BE0102
:101590006F5F7F4F8BEE95E10E94C56ACE01019689
:1015A0000E94A86B8BEE95E10E94344C613071056E
:1015B00029F481E08093D20B0C946229672B11F0FF
:1015C0000C9462291092D20B0C94622967E075E0AA
:1015D000CE0101960E94386CBE016F5F7F4FCE0135
:1015E0008F5B9F4F0E94633E182FCE0101960E9491
:1015F000A86B112309F476C066E070E089E096E1FB
:101600000E945E6A682FCE0101960E94086CBE019E
:101610006F5F7F4F8BEE95E10E94C56ACE01019608
:101620000E94A86B8BEE95E10E94FE6960E08BEE54
:1016300095E10E949E6A8BEE95E10E94344C6B010D
:101640007C01CB011816190614F00C946229209124
:101650008502309186022617370714F40C9462290C
:1016600048E050E069E076E1CE0101960E948C36B8
:10167000BE016F5F7F4F8BEE95E10E94C56ACE0180
:1016800001960E94A86B8BEE95E10E94FE69809105
:10169000EF159091F0150997A8F028E030E040E0B0
:1016A00050E06BEE75E1CE0101960E944C6CBE01DC
:1016B0006F5F7F4F8BEE95E10E94C56ACE01019668
:1016C0000E94A86BC60163E0880F991F6A95E1F735
:1016D000BC01685D784E48E050E08BEE95E10E94D9
:1016E0002D3E23CC6EE075E0CE0101960E94386C51
:1016F000BE016F5F7F4FCE018F5B9F4F0E94633EA5
:10170000182FCE0101960E94A86B112309F4DFC1A6
:101710006AE175E0CE014C960E94386C65E175E097
:10172000CE0101960E94386CAE01445E5F4FBE014F
:101730006F5F7F4FCE018F5B9F4F0E9404A3CE014E
:1017400001960E94A86BCE014C960E94A86B6AE19C
:1017500075E0CE014C960E94386C67E175E0CE01D1
:1017600001960E94386CAE01445E5F4FBE016F5F10
:101770007F4FCE018F5B9F4F0E9404A3CE01019645
:101780000E94A86BCE014C960E94A86B6AE175E09E
:10179000CE014C960E94386C69E175E0CE0101964D
:1017A0000E94386CAE01445E5F4FBE016F5F7F4F99
:1017B000CE018F5B9F4F0E9404A3CE0101960E9431
:1017C000A86BCE014C960E94A86B6DE175E0CE012E
:1017D0004C960E94386C6CE175E0CE0101960E9437
:1017E000386CAE01445E5F4FBE016F5F7F4FCE012C
:1017F0008F5B9F4F0E9404A3CE0101960E94A86BAD
:10180000CE014C960E94A86B6DE175E0CE014C961E
:101810000E94386C69E878E0CE0101960E94386C2D
:10182000AE01445E5F4FBE016F5F7F4FCE018F5BA5
:101830009F4F0E9404A3CE0101960E94A86BCE0187
:101840004C960E94A86BCE018F5B9F4F0E94FE6951
:101850000E94254E60939E0C70939F0C8093A00C69
:101860009093A10C36E0E32EF12C44E6442E512C4B
:10187000612C712C88248394912C5701F3E0AF0ED6
:10188000B11C27968EAD9FAD27970197A816B90674
:1018900010F00C946229B701CE018F5B9F4F0E941C
:1018A0005E6A682FCE014C960E94086C670122E0A8
:1018B000C20ED11C3FEFE31AF30A9601A701BE0145
:1018C0006F5B7F4FCE0101960E944C6CCE0101965A
:1018D0000E94344C8B01CE0101960E94A86B01300E
:1018E000110521F400912E1810912F1803301105C5
:1018F00021F400913018109131186AE175E0CE01A1
:1019000001960E94386CA601BE016F5F7F4FCE0129
:101910008F5B9F4F0E94189A6C01CE0101960E9426
:10192000A86B62ED7AE0CE0101960E94386C1C141F
:101930001D04E4F49601A501BE016F5B7F4FCE014B
:101940008A960E944C6CBE01665D7F4FCE01019667
:101950000E94C56ACE018A960E94A86B10161106D5
:10196000E4F076014FEFE41AF40AA8C0A501BE0125
:101970006F5B7F4FCE018A960E948C36BE01665DFA
:101980007F4FCE0101960E94C56ACE018A960E94C1
:10199000A86B101611060CF091C0809185029091F1
:1019A0008602801791070CF485C060E070E0CE01DC
:1019B0004C960E945E6A8235F9F4CE0101960E942F
:1019C000344C672B682B692B39F4F801EE0FFF1F9D
:1019D000E158FD4F11821082CE0101960E94344CD5
:1019E000613071058105910509F064C0F801EE0FC1
:1019F000FF1FE158FD4F1FC08634A1F5CE010196AF
:101A00000E94344C672B682B692B39F4F801EE0FD8
:101A1000FF1FED5EFD4F11821082CE0101960E94E4
:101A2000344C613071058105910539F4F801EE0FF0
:101A3000FF1FED5EFD4F91828082000F111F000F8E
:101A4000111FF801E357FD4F80819181A281B3817D
:101A5000181619061A061B0624F14082518262826A
:101A600073821FC0843461F4CE0101960E94344C0D
:101A7000000F111F000F111FF801EF5FFD4F0DC088
:101A80008435C1F4CE0101960E94344C000F111F21
:101A9000000F111FF801E357FD4F608371838283AC
:101AA00093830E94254EF801E75EFD4F60837183AA
:101AB000828393831C141D040CF453CFCE01019632
:101AC0000E94A86BCE014C960E94A86BD6CE6FE107
:101AD00075E0CE0101960E94386CBE016F5F7F4FAA
:101AE000CE018F5B9F4F0E94633E182FCE0101965F
:101AF0000E94A86B112309F41EC144E050E069E084
:101B000076E1CE0101960E948C36BE016F5F7F4F59
:101B10008BEE95E10E94C56ACE0101960E94A86BEA
:101B20008BEE95E10E94FE6960E08BEE95E10E94EC
:101B30009E6A4091EF155091F01562EC7BE08BEEC0
:101B400095E10E942D3E6CE477E0CE01CB960E9499
:101B5000386C6BEE75E1CE01C3960E94306C8FA994
:101B600098AD892B09F492C062ED7AE0CE018A9695
:101B70000E94386C21968EAD9FAD2197DE01A95B46
:101B8000BF4F5D01892B39F4CE01C3960E94344CBE
:101B9000F501608375C040E050E0BE01655C7F4F99
:101BA000CE01C3960E94189A7C01892B11F4EFA8EC
:101BB000F8AC8E01045E1F4F62ED7AE0C8010E940E
:101BC000386C4501C12CD12C702E612E84010A196C
:101BD0001B091E141F0484F59701A601BE016D5C4C
:101BE0007F4FCE0101960E944C6CBE016F5F7F4F0C
:101BF000872D962D0E94C56ACE0101960E94A86B82
:101C0000872D962D0E94344CD4016D934D016701B0
:101C1000BFEFCB1ADB0AA601BE01655C7F4FCE0188
:101C2000C3960E94189A7C018FA998ADC816D90650
:101C300068F2E12CF12CCACF8FA998ADC816D9064D
:101C4000D8F4A601BE016D5C7F4FCE0101960E94C3
:101C50008C36BE016F5F7F4FCE014C960E94C56AE5
:101C6000CE0101960E94A86BCE014C960E94344C86
:101C7000F501E00FF11F6083CE014C960E94A86B26
:101C8000CE018A960E94A86B11E001C010E0CE013F
:101C9000C3960E94A86BCE01CB960E94A86B11231D
:101CA00011F40C9462298E01095B1F4F70E4E72E3A
:101CB00077E1F72E6801E4E0CE0ED11CD8018D91BA
:101CC0008D01F70181937F011D8E1C8E1F8E1E8E4C
:101CD00019A218A24AE0BE016F5F7F4F90E00E94F8
:101CE00010ADBE016F5F7F4FCE014C960E947E6BA0
:101CF000CE014C960E94DA83CE014C960E94A86BCE
:101D00000C151D05D9F684EF91E09093AC028093F9
:101D1000AB0264E177E10E94479064E670E080E006
:101D200090E00E94418264E275E0CE0101960E943B
:101D3000386C0C94C7266FE275E0CE0101960E94C4
:101D4000386CBE016F5F7F4FCE018F5B9F4F0E944B
:101D5000633E182FCE0101960E94A86B1123A9F0B3
:101D600065E573E0CE0101960E94286C64E670E0A0
:101D7000CE0101960E940D7CCE0101960E94A86BB7
:101D8000E0E0F0E019950C94622966E375E0CE017D
:101D90004C960E94386CBE01645E7F4F89E096E1EC
:101DA0000E94633E811116C06EE375E0CE0101967C
:101DB0000E94386CBE016F5F7F4F89E096E10E9400
:101DC000633E11E0811101C010E0CE0101960E9436
:101DD000A86B01C011E0CE014C960E94A86B1123A4
:101DE000B1F066E475E0CE0101960E94386C6EE4B5
:101DF00078E1CE0101960E94286BBC0181EF95E14C
:101E00000E94936BCE0101960E94A86B38C060E5DA
:101E100075E0CE014C960E94386CBE01645E7F4F27
:101E200089E096E10E94633E811116C067E575E086
:101E3000CE0101960E94386CBE016F5F7F4F89E032
:101E400096E10E94633E11E0811101C010E0CE01D5
:101E500001960E94A86B01C011E0CE014C960E9431
:101E6000A86B1123B1F067E473E081EF95E10E9464
:101E7000396B64E578E181EF95E10E94BF6A66ED18
:101E800076E0CE0101960E94386C61EF75E10C940A
:101E9000851C6EE575E0CE0101960E94386CBE018E
:101EA0006F5F7F4FCE018F5B9F4F0E94633E182F65
:101EB000CE0101960E94A86B112321F00E940676A4
:101EC0000C94602967E675E0CE014C960E94386C50
:101ED000BE01645E7F4F89E096E10E94633E8111FE
:101EE00016C06CE675E0CE0101960E94386CBE010A
:101EF0006F5F7F4F89E096E10E94633E11E08111A0
:101F000001C010E0CE0101960E94A86B01C011E053
:101F1000CE014C960E94A86B112309F443C06DE1D9
:101F200075E0CE0101960E94386C40910D165091DB
:101F30000E168D819E81481B590BBE016F5F7F4F2E
:101F400089E096E10E94CA99AC014F5F5F4F69E05A
:101F500076E1CE014C960E948C36BE01645E7F4FC6
:101F60008BEE95E10E94C56ACE014C960E94A86B4B
:101F7000CE0101960E94A86B8BEE95E10E94344C35
:101F80006115710521F481E08093AA0207C06130D8
:101F9000710511F00C9460291092AA020E9495A478
:101FA0000C94602961E775E0CE0101960E94386CBF
:101FB000BE016F5F7F4FCE018F5B9F4F0E94633EDC
:101FC000182FCE0101960E94A86B112309F43BC182
:101FD00043E050E069E076E1CE0101960E948C3644
:101FE000BE016F5F7F4F8BEE95E10E94C56ACE0107
:101FF00001960E94A86B6BEE75E1CE0101960E94DE
:10200000306CCE0101960E94C38DCE0101960E94D4
:10201000A86B84EF91E09093AC028093AB026BEEDF
:1020200075E1CE0101960E94306C60E0CE01019610
:102030000E94553EBC018AE598E10E94936BCE0157
:1020400001960E94A86B6BEE75E1CE0101960E948D
:10205000306C60E0CE0101960E94553EBC0184E5E3
:1020600098E10E94936BCE0101960E94A86B40916B
:102070005E1850915F1864ED77E18AE598E10E945F
:102080002D3E40915818509159186FED77E184E535
:1020900098E10E942D3E64E177E18091AB0290913E
:1020A000AC020E94479065E775E0CE0101960E9460
:1020B000386C6BEE75E1CE0101960E94286BBC0175
:1020C000CE018A960E94306CCE0101960E94A86BC8
:1020D0008091D0179091D117892B39F4BE01665D9C
:1020E0007F4F82EE91E10E94366D68EB7BE080E0ED
:1020F00090E00E9441828091D0179091D117029771
:1021000009F087C06BEE75E1CE01C3960E94306C7A
:102110006DE775E0CE0101960E94386CCE01019604
:102120000E94FCA3CE0101960E94A86B64EF71E0AF
:1021300080E090E00E94418260E875E0CE01019667
:102140000E94386CCE0101960E94FCA3CE0101963C
:102150000E94A86B6CED75E080E090E00E944182E7
:1021600069E875E0CE0101960E94386CCE010196B7
:102170000E94FCA3CE0101960E94A86B64EF71E05F
:1021800080E090E00E94418267E975E0CE0101960F
:102190000E94386CCE0101960E94FCA3CE010196EC
:1021A0000E94A86B64EF71E080E090E00E944182A1
:1021B00065E775E0CE0101960E94386CBE016D5C4A
:1021C0007F4FCE0101960E94286BBC01CE014C9638
:1021D0000E94306CCE0101960E94A86BCE014C96F5
:1021E0000E94FE69BE01645E7F4FCE0101960E948F
:1021F000306CCE0101960E94FCA3CE0101960E9494
:10220000A86BCE014C960E94A86BCE01C3960E948B
:10221000A86B68EB7BE080E090E00E94418264ED77
:1022200077E1CE0101960E94386CCE0101960E94A2
:10223000C38DCE0101960E94A86B10920002CE01C0
:102240008A960C94B12865EA75E0CE0101960E9449
:10225000386CBE016F5F7F4FCE018F5B9F4F0E9436
:10226000633E182FCE0101960E94A86B112309F43A
:1022700089C044E050E069E076E1CE0101960E9419
:102280008C36BE016F5F7F4F8BEE95E10E94C56A71
:10229000CE0101960E94A86B6AEA75E0CE01019614
:1022A0000E94386C6BEE75E1CE0101960E94286B9E
:1022B000BC01CE014C960E94306CCE0101960E946A
:1022C000A86B8091D0179091D117892B39F4BE015A
:1022D000645E7F4F82EE91E10E94366D68E873E1A3
:1022E00080E090E00E9441828091D0179091D117B8
:1022F000029709F041C061EB75E0CE0101960E94A2
:10230000386C8091EF159091F015892B39F46AEBB8
:1023100075E0CE0101960E947E6B15C0BE016F5F15
:102320007F4FCE018A960E94306CCE018A960E9421
:10233000FCA3CE018A960E94A86B60E777E180E05B
:1023400090E00E944182BE01645E7F4FCE018A967A
:102350000E94306CCE018A960E94FCA3CE018A9620
:102360000E94A86B68E873E180E090E00E944182DF
:10237000CE0101960E94A86B10920002CE014C96ED
:102380000C94B12863EC75E0CE0101960E94386C84
:10239000BE016F5F7F4FCE018F5B9F4F0E94633EF8
:1023A000182FCE0101960E94A86B112309F45CC07E
:1023B00069E076E18BEE95E10E94936B81E080937A
:1023C000000269E076E1CE0101960E94306CCE01F8
:1023D00001960E94C38DCE0101960E94A86B809148
:1023E000D0179091D117029709F16BEE75E182EE4B
:1023F00091E10E94366D68EB7BE080E090E00E9406
:102400004182CE0101960E94C2A4BE016F5F7F4F40
:1024100089E096E10E94C56ACE0101960E94A86BF0
:1024200060ED77E080E090E00E9441828091D017DB
:102430009091D117029771F46BEE75E1CE01019680
:102440000E94306CCE0101960E94FCA3CE01019641
:102450000E94A86B80910D1690910E16892B11F495
:102460000C9460290C947D1C67EC75E0CE010196FC
:102470000E94386CBE016F5F7F4FCE018F5B9F4F14
:102480000E94633E182FCE0101960E94A86B112373
:1024900009F47FC18091D0179091D117019711F065
:1024A0000C9460296DEC75E0CE01C3960E94386CE7
:1024B000BE016D5C7F4F82EE91E10E94366D6CE251
:1024C00071E080E090E00E944182CE018A960E94F5
:1024D000C2A464E670E080E090E00E944182E12CBA
:1024E000F12C55E0C52ED12C6AE0A62EB12C68ED5A
:1024F00075E0CE0101960E94386C40E050E0BE01CC
:102500006F5F7F4FCE018A960E94189A8C01CE0190
:1025100001960E94A86BA8014F5F5F4FBE01665DE8
:102520007F4FCE0101960E948C36BE016F5F7F4FB8
:10253000CE01C3960E94C56ACE0101960E94A86B87
:102540008FA998AD892B71F060E070E0CE01C39641
:102550000E945E6A082E000C990BC0970A9710F42F
:102560000C94762910E06DE372E0CE0101960E9492
:10257000286C64E170E0CE0101960E94359ACE018C
:1025800001960E94A86BFFEFEF1AFF0A62E370E06A
:1025900080E090E00E944182C701B6010E94A2B390
:1025A000019771F5CE0101960E9425848D819E814F
:1025B000892B59F0BE016F5F7F4F89E096E10E9441
:1025C000936B0E94290611E017C024E1E216F10482
:1025D0009CF0C701B5010E94A2B3892B69F4BE012A
:1025E0006D5C7F4F82EE91E10E94366D68EC70E089
:1025F00080E090E00E944182CE0101960E94A86B8B
:10260000CE0101960E94C2A4BE016F5F7F4FCE0132
:102610008A960E94C56ACE0101960E94A86B62E369
:1026200070E080E090E00E94418234E6E316F1041D
:1026300019F0112309F45BCF8091FA188823F1F087
:1026400066ED76E0CE014C960E94386CBE016D5C62
:102650007F4FCE014C960E94286BBC01CE010196A3
:102660000E94306CCE0101960E94DA83CE01019661
:102670000E94A86BCE014C960E94A86B8FA998ADC2
:10268000892B61F060E070E0CE01C3960E945E6A23
:10269000082E000C990BC0970A9738F06AED75E088
:1026A000CE0101960E94386C1BC06AE377E0CE0130
:1026B00001960E94386CBE016F5F7F4FCE01C396BA
:1026C0000E94633E182FCE0101960E94A86B111143
:1026D000E5CFBE016D5C7F4FCE0101960E94206C5C
:1026E000CE018A960E94A86BCE01C3960E94A86B69
:1026F0008D819E81009711F40C945C29E981FA8107
:102700002081222311F40C945C29079710F40C9477
:102710005C296EE373E0CE014C960E94286C68EC55
:1027200070E0CE014C960E94359ACE014C960E94E4
:10273000A86BBE016F5F7F4FCE014C960E94306C3C
:1027400060ED77E0CE014C960E940D7CCE014C9658
:102750000E94A86B66EE75E0CE014C960E94386C24
:1027600069E076E1CE014C960E94286BBC01CE0157
:102770008A960E94306CCE018A960E94DA83CE013E
:102780008A960E94A86BCE014C960E94A86B0C946E
:102790005C2964EF75E0CE0101960E94386CBE01A1
:1027A0006F5F7F4FCE018F5B9F4F0E94633E182F5C
:1027B000CE0101960E94A86B112309F4E9C025E01F
:1027C00030E044E050E069E076E1CE0101960E94FD
:1027D0004C6CBE016F5F7F4F8BEE95E10E94C56A26
:1027E000CE0101960E94A86B69E076E1CE010196C8
:1027F0000E94306CCE0101960E94C38DCE010196DD
:102800000E94A86B8BEE95E10E94344C61307105FB
:10281000D1F57093D1176093D0176CE672E0CE01BA
:1028200001960E94286CCE0101960E94C38DCE01B4
:1028300001960E94A86B69EF75E0CE014C960E944C
:10284000386C64E578E1CE014C960E94286BBC019F
:10285000CE0101960E94306C48EC50E06FEF7FEFA4
:10286000CE0101960E946C85CE0101960E94A86B54
:10287000CE014C960E94A86B0E94D6A840E052EC74
:1028800061E070E056C061157105A9F41092D1178E
:102890001092D0176EE572E0CE0101960E94286C6E
:1028A000CE0101960E94C38DCE0101960E94A86BB5
:1028B0006FEF75E019C06230710511F00C9460295A
:1028C0007093D1176093D0176DE472E0CE0101963A
:1028D0000E94286CCE0101960E94C38DCE01019604
:1028E0000E94A86B63E076E0CE014C960E94386CA3
:1028F00064E578E1CE014C960E94286BBC01CE01C4
:1029000001960E94306C48EC50E06FEF7FEFCE01F3
:1029100001960E946C85CE0101960E94A86BCE01A3
:102920004C960E94A86B0E94D6A840E855E260E051
:1029300070E082EE91E10E94287984EF91E090931B
:10294000AC028093AB0264E177E10E94479068E0BB
:1029500076E0CE014C960E94386C6EE478E1CE01B0
:102960004C960E94286BBC01CE0101960E94306CEF
:1029700060ED77E0CE0101960E940D7CCE010196BC
:102980000E94A86BCE014C960E94A86B0C94602903
:102990006DE076E0CE0101960E94386CBE016F5F5B
:1029A0007F4FCE018F5B9F4F0E94633E182FCE0159
:1029B00001960E94A86B112309F441C047E050E042
:1029C00069E076E1CE0101960E948C36BE016F5F10
:1029D0007F4F8BEE95E10E94C56ACE0101960E9461
:1029E000A86B60E477E0CE0101960E94386CBE01CE
:1029F0006F5F7F4F8BEE95E10E94633E182FCE01F3
:102A000001960E94A86B111110923D0B67E179E0CD
:102A1000CE0101960E94386CBE016F5F7F4F8BEE36
:102A200095E10E94633E182FCE0101960E94A86B8B
:102A3000112309F462C781E080933D0B5EC765E115
:102A400076E0CE0101960E94386CBE016F5F7F4F29
:102A5000CE018F5B9F4F0E94633E182FCE010196DF
:102A60000E94A86B112301F146E050E069E076E195
:102A7000CE0101960E948C36BE016F5F7F4F8BEEB8
:102A800095E10E94C56ACE0101960E94A86B8BEE6B
:102A900095E10E948F916093181870931918809394
:102AA0001A1890931B1834C06CE176E0CE010196A1
:102AB0000E94386CBE016F5F7F4FCE018F5B9F4FCE
:102AC0000E94633E182FCE0101960E94A86B11232D
:102AD00081F148E050E069E076E1CE0101960E9484
:102AE0008C36BE016F5F7F4F8BEE95E10E94C56A09
:102AF000CE0101960E94A86B8BEE95E10E948F910A
:102B000060931E1870931F188093201890932118BB
:102B100084EF91E09093AC028093AB0264E177E1A3
:102B20000E94479064E670E080E090E00E9441825D
:102B3000E4C665E276E0CE0101960E94386CBE01E3
:102B40006F5F7F4FCE018F5B9F4F0E94633E182FB8
:102B5000CE0101960E94A86B112301F149E050E0DB
:102B600069E076E1CE0101960E948C36BE016F5F6E
:102B70007F4F8BEE95E10E94C56ACE0101960E94BF
:102B8000A86B8BEE95E10E948F9160932218709351
:102B900023188093241890932518BACF6FE276E01B
:102BA000CE0101960E94386CBE016F5F7F4FCE014F
:102BB0008F5B9F4F0E94633E182FCE0101960E94AB
:102BC000A86B1123F1F049E050E069E076E1CE0115
:102BD00001960E948C36BE016F5F7F4F8BEE95E1B0
:102BE0000E94C56ACE0101960E94A86B8BEE95E10A
:102BF0000E948F910E945DB37093291860932818EA
:102C000087CF69E376E0CE0101960E94386CBE0161
:102C10006F5F7F4FCE018F5B9F4F0E94633E182FE7
:102C2000CE0101960E94A86B1123F1F04AE050E01A
:102C300069E076E1CE0101960E948C36BE016F5F9D
:102C40007F4F8BEE95E10E94C56ACE0101960E94EE
:102C5000A86B8BEE95E10E948F910E945DB37093FB
:102C600027186093261854CF64E476E0CE010196CD
:102C70000E94386CBE016F5F7F4FCE018F5B9F4F0C
:102C80000E94633E182FCE0101960E94A86B11236B
:102C900011F14BE050E069E076E1CE0101960E942F
:102CA0008C36BE016F5F7F4F8BEE95E10E94C56A47
:102CB000CE0101960E94A86B8BEE95E10E948F9148
:102CC0000E945DB360932A1870932B1880932C1880
:102CD00090932D181DCF60E576E0CE0101960E94FD
:102CE000386CBE016F5F7F4FCE018F5B9F4F0E949C
:102CF000633E182FCE0101960E94A86B1123E1F0CC
:102D000045E050E069E076E1CE0101960E948C3604
:102D1000BE016F5F7F4F8BEE95E10E94C56ACE01C9
:102D200001960E94A86B8BEE95E10E94344C709343
:102D30001D1860931C18ECCE66E576E0CE01019676
:102D40000E94386CBE016F5F7F4FCE018F5B9F4F3B
:102D50000E94633E182FCE0101960E94A86B11239A
:102D600009F440C20E94254E60939E0C70939F0C04
:102D70008093A00C9093A10C26E030E045E050E059
:102D800069E076E1CE0101960E944C6CBE016F5F56
:102D90007F4F8BEE95E10E94C56ACE0101960E949D
:102DA000A86B8BEE95E10E94344C4B015C016B01EA
:102DB00081E08093131880933E0B0E94254E609310
:102DC000A90C7093AA0C8093AB0C9093AC0C81145B
:102DD000910481F580912E1890912F18FC01EE0F2F
:102DE000FF1FE158FD4F11821082880F991F880F35
:102DF000991FFC01EF5FFD4F108211821282138236
:102E00008091301890913118FC01EE0FFF1FE158AE
:102E1000FD4F11821082880F991F880F991FFC01A6
:102E2000EF5FFD4F108211821282138248E7E42E79
:102E3000F12C43C141E08416910409F061C08091F6
:102E40000D1690910E160897C0F047E050E069E02B
:102E500076E1CE0101960E948C36CE0101960E9449
:102E60008F91609318187093191880931A18909383
:102E70001B18CE0101960E94A86B00912E1810918C
:102E80002F18F801EE0FFF1FE158FD4F81E090E091
:102E900091838083000F111F000F111FF801E3576A
:102EA000FD4F84E893E0A0E0B0E080839183A283AB
:102EB000B3830E94254EF801E75EFD4F6083718366
:102EC000828393838091301890913118FC01EE0F2A
:102ED000FF1FE158FD4F11821082880F991F880F44
:102EE000991FFC01E75EFD4F10821182128213824E
:102EF000FC01EF5FFD4F1082118212821382DBC052
:102F000052E08516910409F0ACC080910D169091A5
:102F10000E160897C0F047E050E069E076E1CE0178
:102F200001960E948C36CE0101960E948F9160938B
:102F30001E1870931F188093201890932118CE01AB
:102F400001960E94A86B40901E1850901F18609028
:102F5000201870902118A30192016091221870919D
:102F6000231880912418909125180E94F5B087FFAE
:102F700010C020E030E040EA50E4C301B2010E94FA
:102F800091B2609322187093231880932418909321
:102F9000251880911C1890911D18019797FD23C04A
:102FA000880F991F880F991F8C0101511D4F20E038
:102FB00030E040E251E46091181870911918809146
:102FC0001A1890911B180E9491B29B01AC01D80174
:102FD0006D917D918D919C910E948EB318161CF479
:102FE00000E010E002C004EB10E080912E189091F8
:102FF0002F18FC01EE0FFF1FE158FD4F11821082C8
:10300000880F991F880F991FFC01EF5FFD4F1082F9
:10301000118212821382E0903018F0903118F7017B
:10302000EE0FFF1FE158FD4F81E090E09183808318
:10303000EE0CFF1CEE0CFF1CF701E357FD4F80EB7D
:1030400094E0A0E0B0E080839183A283B3830E94E8
:10305000254EF701E75EFD4F608371838283938382
:1030600026C0B3E08B16910431F5809189029091CE
:103070008A028A3591051CF004EB10E002C000E0E2
:1030800010E080912E1890912F18FC01EE0FFF1F79
:10309000E158FD4F11821082880F991F880F991FE8
:1030A000FC01EF5FFD4F1082118212821382F8E75C
:1030B000EF2EF12C04C0E12CF12C04EB10E0E8E041
:1030C0008E1A9108F2E08F16910408F05AC0809190
:1030D000890290918A028A35910514F400E010E08B
:1030E00080912E1890912F18FC01EE0FFF1FE158D0
:1030F000FD4F11821082880F991F880F991FFC01C4
:10310000EF5FFD4F1082118212821382E09030181F
:10311000F0903118F701EE0FFF1FE158FD4F81E0ED
:1031200090E091838083EE0CFF1CEE0CFF1CF701F6
:10313000EF5FFD4F8CE291E0A0E0B0E080839183EF
:10314000A283B383F701E357FD4F88E592E0A0E047
:10315000B0E080839183A283B3830E94254EF70160
:10316000E75EFD4F608371838283938328E0C216FC
:10317000D10421F41092131810923E0B48E7E42E6C
:10318000F12CC8010E945D7190938A02809389029C
:10319000801B910B97FF03C091958195910903972F
:1031A0003CF0C8010E945D7190938A02809389026D
:1031B000C7010E94DB7090938C0280938B028E1962
:1031C0009F0997FF03C091958195910903973CF062
:1031D000C7010E94DB7090938C0280938B026CE598
:1031E00076E08DC364E676E0CE0101960E94386CED
:1031F000BE016F5F7F4FCE018F5B9F4F0E94633E8A
:10320000182FCE0101960E94A86B112389F143E08B
:1032100050E0BE016F5B7F4FCE0101960E948C365D
:10322000BE016F5F7F4F8BEE95E10E94C56ACE01B4
:1032300001960E94A86B8091EF159091F015892B53
:1032400041F08BEE95E10E94344C7093DE02609366
:10325000DD028091DD029091DE020197029708F471
:103260004CC381E090E09093DE028093DD0245C381
:103270006DE376E0CE014C960E94386CBE01645E30
:103280007F4FCE018F5B9F4F0E94633E811117C01D
:1032900065E976E0CE0101960E94386CBE016F5F51
:1032A0007F4FCE018F5B9F4F0E94633E11E08111E3
:1032B00001C010E0CE0101960E94A86B01C011E090
:1032C000CE014C960E94A86B112309F462C06DE3F5
:1032D00076E0CE0101960E94386CBE016F5F7F4F91
:1032E000CE018F5B9F4F0E94633E182FCE01019647
:1032F0000E94A86B1123A1F046E050E0BE016F5B75
:103300007F4FCE0101960E948C36BE016F5F7F4FCA
:103310008BEE95E10E94C56ACE0101960E94A86BD2
:1033200065E976E0CE0101960E94386CBE016F5FC0
:103330007F4FCE018F5B9F4F0E94633E182FCE01BF
:1033400001960E94A86B1123A1F042E050E0BE015B
:103350006F5B7F4FCE0101960E948C36BE016F5F7E
:103360007F4F8BEE95E10E94C56ACE0101960E94C7
:10337000A86B8091EF159091F015892B09F4BDC2CF
:103380006BEE75E1CE0101960E94306C61E070E059
:10339000ACC261E776E0CE018A960E94386CBE012D
:1033A000665D7F4FCE018F5B9F4F0E94633E811110
:1033B0000C94992968E676E0CE014C960E94386C10
:1033C000BE01645E7F4FCE018F5B9F4F0E94633EC4
:1033D000811118C060E776E0CE0101960E94386C3A
:1033E000BE016F5F7F4FCE018F5B9F4F0E94633E98
:1033F000FF24F394811101C0F12CCE0101960E94AB
:10340000A86B02C0FF24F394CE014C960E94A86BD7
:10341000CE018A960E94A86BFF2009F4E5C061E7FF
:1034200076E0CE0101960E94386CBE016F5F7F4F3F
:10343000CE018F5B9F4F0E94633E182FCE010196F5
:103440000E94A86B1123A9F046E050E0BE016F5B1B
:103450007F4FCE0101960E948C36BE016F5F7F4F79
:103460008BEE95E10E94C56ACE0101960E94A86B81
:103470004AC047E050E0BE016F5B7F4FCE0101962E
:103480000E948C36BE016F5F7F4F8BEE95E10E94EC
:10349000C56ACE0101960E94A86B65EA7AE0CE016A
:1034A00001960E94386CBE016F5F7F4FCE018F5B2B
:1034B0009F4F0E94633E182FCE0101960E94A86B79
:1034C000112331F081E090E09093DE028093DD02E1
:1034D0006EE775E0CE0101960E94386CBE016F5F09
:1034E0007F4FCE018F5B9F4F0E94633E182FCE010E
:1034F00001960E94A86B112331F082E090E0909336
:10350000DE028093DD028BEE95E10E948F916B01CC
:103510007C0120E030E0A9010E948EB318169CF4D3
:10352000A701960160E070E08AE794E40E94F5B29A
:103530000E945DB36093C9027093CA028093CB026C
:103540009093CC020CC081E090E0A0E0B0E08093CA
:10355000C9029093CA02A093CB02B093CC0280918F
:10356000C9029091CA02A091CB02B091CC02181668
:1035700019061A061B0664F081E090E0A0E0B0E0B6
:103580008093C9029093CA02A093CB02B093CC025D
:103590008091DD029091DE028130910589F4809165
:1035A000C9029091CA02A091CB02B091CC02809343
:1035B000CD029093CE02A093CF02B093D0029DC1D2
:1035C000029709F09AC18091C9029091CA02A09114
:1035D000CB02B091CC028093B3029093B402A0933B
:1035E000B502B093B60289C168E776E0CE01C39612
:1035F0000E94386CBE016D5C7F4FCE018F5B9F4F88
:103600000E94633E8E01045E1F4F81110C94B72906
:103610006BED76E0CE018A960E94386CBE01665D45
:103620007F4FCE018F5B9F4F0E94633E81112CC064
:103630006AED76E0C8010E94386CB801CE018F5B5C
:103640009F4F0E94633E811118C06FE776E0CE0164
:1036500001960E94386CBE016F5F7F4FCE018F5B79
:103660009F4F0E94633EEE24E394811101C0E12C40
:10367000CE0101960E94A86B02C0EE24E394CE0115
:103680004C960E94A86B02C0EE24E394CE018A9669
:103690000E94A86BCE01C3960E94A86BEE2009F48D
:1036A00044C168E776E0CE0101960E94386CBE0105
:1036B0006F5F7F4FCE018F5B9F4F0E94633EE82E6E
:1036C000CE0101960E94A86BEE2019F046E050E072
:1036D00017C06BED76E0CE0101960E94386CBE01FA
:1036E0006F5F7F4FCE018F5B9F4F0E94633EE82E3E
:1036F000CE0101960E94A86BEE20A9F042E050E0B6
:10370000BE016F5B7F4FCE0101960E948C36BE01D9
:103710006F5F7F4F8BEE95E10E94C56ACE010196E7
:103720000E94A86B4AC043E050E0BE016F5B7F4F30
:10373000CE0101960E948C36BE016F5F7F4F8BEEEB
:1037400095E10E94C56ACE0101960E94A86B65EAC8
:103750007AE0CE0101960E94386CBE016F5F7F4F08
:10376000CE018F5B9F4F0E94633EE82ECE010196F3
:103770000E94A86BEE2031F081E090E09093DE0291
:103780008093DD026EE775E0CE0101960E94386CF1
:10379000BE016F5F7F4FCE018F5B9F4F0E94633EE4
:1037A000E82ECE0101960E94A86BEE2031F082E057
:1037B00090E09093DE028093DD028091EF1590916E
:1037C000F015892B09F499C068E27AE0CE014C9695
:1037D0000E94386CBE01645E7F4F8BEE95E10E94C3
:1037E000633E811115C068E27AE0CE0101960E9425
:1037F000386CBE016F5F7F4F8BEE95E10E94633E98
:10380000FF24F3948111F12CCE0101960E94A86B44
:10381000C8010E94A86BFF2009F45FC08BEE95E100
:103820000E948F9120E030E0A9010E948EB387FDB5
:1038300015C066ED77E0CE0101960E94386C6BEE04
:1038400075E1CE0101960E94286BBC018BEE95E1DB
:103850000E94936BCE0101960E94A86B8BEE95E1BE
:103860000E948F9120E030E0A9010E94F5B087FF0F
:1038700034C08BEE95E10E948F9120E030E0A901E9
:103880000E948EB318163CF48BEE95E10E948F9146
:10389000AB01BC0107C08BEE95E10E948F91AB019B
:1038A000BC01705822E0C8010E94AD6B68E27AE06A
:1038B000CE0101960E94386CB801CE0101960E949B
:1038C000286BBC018BEE95E10E94936BCE010196B3
:1038D0000E94A86BC8010E94A86B6BEE75E1CE0137
:1038E00001960E94306C62E070E0CE0101960E9469
:1038F000929ACE0101960E94A86B66ED76E0CE0109
:1039000001960E94386C69E076E1CE0101960E9432
:10391000286BBC01CE014C960E94306CCE014C96B7
:103920000E94DA83CE014C96FBC564E876E0CE01B6
:103930008A960E94386CBE01665D7F4FCE018F5B18
:103940009F4F0E94633E81110C949F2963E876E0AB
:10395000C8010E94386CB801CE018F5B9F4F0E9456
:10396000633E811118C06AE876E0CE0101960E949C
:10397000386CBE016F5F7F4FCE018F5B9F4F0E94FF
:10398000633EFF24F394811101C0F12CCE01019616
:103990000E94A86B02C0FF24F394C8010E94A86B88
:1039A000CE018A960E94A86BFF2009F48DC0CE013B
:1039B0008F5B9F4F0E94FE6964E876E0CE0101961E
:1039C0000E94386CBE016F5F7F4FCE018F5B9F4FAF
:1039D0000E94633EF82ECE0101960E94A86BFF2044
:1039E000A9F045E050E0BE016F5B7F4FCE0101962C
:1039F0000E948C36BE016F5F7F4F8BEE95E10E9477
:103A0000C56ACE0101960E94A86B4AC046E050E00C
:103A1000BE016F5B7F4FCE0101960E948C36BE01C6
:103A20006F5F7F4F8BEE95E10E94C56ACE010196D4
:103A30000E94A86B65EA7AE0CE0101960E94386C7C
:103A4000BE016F5F7F4FCE018F5B9F4F0E94633E31
:103A5000F82ECE0101960E94A86BFF2031F081E084
:103A600090E09093DE028093DD026EE775E0CE0178
:103A700001960E94386CBE016F5F7F4FCE018F5B55
:103A80009F4F0E94633EF82ECE0101960E94A86BC4
:103A9000FF2031F082E090E09093DE028093DD021F
:103AA0008091EF159091F015892B09F425C56BEEE7
:103AB00075E1CE0101960E94306C63E070E0CE01AA
:103AC00001960E94929AC8C562E976E0CE018A9674
:103AD0000E94386CBE01665D7F4FCE018F5B9F4FA9
:103AE0000E94633E81110C94A52961E976E0C8012A
:103AF0000E94386CB801CE018F5B9F4F0E94633EDD
:103B0000811118C068E976E0CE0101960E94386CF8
:103B1000BE016F5F7F4FCE018F5B9F4F0E94633E60
:103B2000FF24F394811101C0F12CCE0101960E9473
:103B3000A86B02C0FF24F394C8010E94A86BCE01B9
:103B40008A960E94A86BFF2009F427C162E976E0FB
:103B5000CE0101960E94386CBE016F5F7F4FCE018F
:103B60008F5B9F4F0E94633EF82ECE0101960E940C
:103B7000A86BFF20A9F045E050E0BE016F5B7F4FCE
:103B8000CE0101960E948C36BE016F5F7F4F8BEE97
:103B900095E10E94C56ACE0101960E94A86B4AC0B9
:103BA00046E050E0BE016F5B7F4FCE0101960E9460
:103BB0008C36BE016F5F7F4F8BEE95E10E94C56A28
:103BC000CE0101960E94A86B65EA7AE0CE010196CB
:103BD0000E94386CBE016F5F7F4FCE018F5B9F4F9D
:103BE0000E94633EF82ECE0101960E94A86BFF2032
:103BF00031F081E090E09093DE028093DD026EE789
:103C000075E0CE0101960E94386CBE016F5F7F4F58
:103C1000CE018F5B9F4F0E94633EF82ECE0101962E
:103C20000E94A86BFF2031F082E090E09093DE02CA
:103C30008093DD028091EF159091F015892B61F052
:103C40008BEE95E10E948F9160935B1170935C11F4
:103C500080935D1190935E11C0905B11D0905C11C8
:103C6000E0905D11F0905E1120E030E044EB53E411
:103C7000C701B6010E948EB387FD0BC020E030E083
:103C800044EB53E4C701B6010E9490B26B017C0182
:103C9000EBCF20E030E0A901C701B6010E94F5B0EA
:103CA00087FF0BC020E030E044EB53E4C701B601CE
:103CB0000E9491B26B017C01ECCFC0925B11D0925B
:103CC0005C11E0925D11F0925E118091DD029091A5
:103CD000DE02019771F4C0925F11D0926011E09200
:103CE0006111F09262116FE976E081EF95E10E9437
:103CF0007E6B8091DD029091DE020297B1F480919B
:103D00005B1190915C11A0915D11B0915E11809357
:103D1000571190935811A0935911B0935A1169EA11
:103D200076E081EF95E10E947E6B61E080E00E9489
:103D3000FD7840915B1150915C1160915D11709123
:103D40005E1121E0C8010E94AD6B61EF75E1CE010B
:103D500001960E94306CB801CE0101960E94286B3A
:103D600060EB76E00E94116BBC0181EF95E10E944F
:103D7000936BCE0101960E94A86BC8010E94A86BAC
:103D800061EF75E18EEB98E10E94366D6DE273E0B4
:103D90008EEB98E10E94576DAFC366EB76E0CE01E3
:103DA0008A960E94386CBE01665D7F4FCE018F5BA4
:103DB0009F4F0E94633E81110C94AB2965EB76E026
:103DC000C8010E94386CB801CE018F5B9F4F0E94E2
:103DD000633E811118C06BEB76E0CE0101960E9424
:103DE000386CBE016F5F7F4FCE018F5B9F4F0E948B
:103DF000633EFF24F394811101C0F12CCE010196A2
:103E00000E94A86B02C0FF24F394C8010E94A86B13
:103E1000CE018A960E94A86BFF2009F409C2409047
:103E2000C9025090CA026090CB027090CC0261EC43
:103E300076E0CE0101960E94386CBE016F5F7F4F25
:103E4000CE018F5B9F4F0E94633EF82ECE010196FC
:103E50000E94A86BFF20A9F044E050E0BE016F5B18
:103E60007F4FCE0101960E948C36BE016F5F7F4F5F
:103E70008BEE95E10E94C56ACE0101960E94A86B67
:103E80004AC045E050E0BE016F5B7F4FCE01019616
:103E90000E948C36BE016F5F7F4F8BEE95E10E94D2
:103EA000C56ACE0101960E94A86B65EA7AE0CE0150
:103EB00001960E94386CBE016F5F7F4FCE018F5B11
:103EC0009F4F0E94633EF82ECE0101960E94A86B80
:103ED000FF2031F081E090E09093DE028093DD02DC
:103EE0006EE775E0CE0101960E94386CBE016F5FEF
:103EF0007F4FCE018F5B9F4F0E94633EF82ECE0115
:103F000001960E94A86BFF2031F082E090E0909330
:103F1000DE028093DD028091DD029091DE0281302D
:103F20009105A9F44090CD025090CE026090CF024E
:103F30007090D00281E090E0A0E0B0E08093CD02EC
:103F40009093CE02A093CF02B093D00216C00297F6
:103F5000A1F44090B3025090B4026090B50270900A
:103F6000B60281E090E0A0E0B0E08093B3029093CD
:103F7000B402A093B502B093B6028091EF15909170
:103F8000F015892BB1F466EC76E08BEE95E10E949A
:103F90007E6B8091EF159091F015892B09F42CC15F
:103FA0006BEE75E1CE0101960E94306C60E070E02E
:103FB00047C06CEC76E0CE0101960E94386CBE01E1
:103FC0006F5F7F4F8BEE95E10E942363F82ECE0149
:103FD00001960E94A86BFF2009F40EC18BEE95E1BB
:103FE0000E948F9120E030E0A9010E94F5B081117C
:103FF00030C08091DD029091DE02019731F46FECC8
:1040000076E08BEE95E10E947E6B8091DD029091CF
:10401000DE02029731F466EC76E08BEE95E10E94C9
:104020007E6B8091EF159091F015892B09F4E4C017
:104030006BEE75E1CE0101960E94306C61E070E09C
:10404000CE0101960E94929ACE0101960E94A86B21
:10405000D3C06DE175E0CE0101960E94386CBE01BF
:104060006F5F7F4F8BEE95E10E942363F82ECE01A8
:1040700001960E94A86BFF2009F4BEC041E050E009
:104080006BEE75E1CE0101960E948C36CE01019651
:104090000E948F916B017C01CE0101960E94A86B5A
:1040A00020E030E0A901C701B6010E94F5B0181662
:1040B00034F0C12CD12C30E8E32E3FE3F32EA09056
:1040C000DD02B090DE0231E0A316B10409F5A701CC
:1040D000960160E070E48CE995E40E94F5B260938B
:1040E000BB027093BC028093BD029093BE026093AA
:1040F0003218709333188093341890933518609366
:10410000BF027093C0028093C1029093C20224C088
:1041100042E0A416B10401F5A701960160E070E445
:104120008CE196E40E94F5B26093BB027093BC02EE
:104130008093BD029093BE02609336187093371837
:1041400080933818909339186093AD027093AE0243
:104150008093AF029093B002B501C8010E94E97A42
:1041600064ED76E0CE0101960E94386CB801CE0174
:1041700001960E94286BBC01CE018A960E94306C89
:10418000CE018A960E943B7CCE018A960E94A86B43
:10419000CE0101960E94A86BC8010E94A86B6BE13A
:1041A00073E0CE0101960E94286CCE0101960E9418
:1041B0003B7CCE0101960E94A86B4091BB025091BE
:1041C000BC026091BD027091BE0225E0CE01019655
:1041D0000E94AD6BCE0101960E94DA83CE0101965A
:1041E0000E94A86B84EF91E09093AC028093AB02A5
:1041F00064E177E10E9447908091DD029091DE02B8
:104200008130910549F44092CD025092CE026092E5
:10421000CF027092D00270C1029709F06DC1409236
:10422000B3025092B4026092B5027092B60264C1B9
:1042300069ED76E0CE018A960E94386CBE01665D1B
:104240007F4FCE018F5B9F4F0E94633E81110C9484
:10425000B12968ED76E0C8010E94386CB801CE0142
:104260008F5B9F4F0E94633E811118C06EED76E018
:10427000CE0101960E94386CBE016F5F7F4FCE0168
:104280008F5B9F4F0E94633EFF24F394811101C016
:10429000F12CCE0101960E94A86B02C0FF24F3947A
:1042A000C8010E94A86BCE018A960E94A86BFF20CD
:1042B00009F43CC127968EAD9FAD2797059708F46A
:1042C0001BC144E050E0BE016F5B7F4FCE01019601
:1042D0000E948C36BE016F5F7F4F8BEE95E10E948E
:1042E000C56ACE0101960E94A86B69ED76E0CE0109
:1042F00001960E94386CBE016F5F7F4FCE018F5BCD
:104300009F4F0E94633EF82ECE0101960E94A86B3B
:10431000FF20A9F044E050E0BE016F5B7F4FCE016B
:1043200001960E948C36BE016F5F7F4F8BEE95E148
:104330000E94C56ACE0101960E94A86B4AC045E062
:1043400050E0BE016F5B7F4FCE0101960E948C361C
:10435000BE016F5F7F4F8BEE95E10E94C56ACE0173
:1043600001960E94A86B65EA7AE0CE0101960E9450
:10437000386CBE016F5F7F4FCE018F5B9F4F0E94F5
:10438000633EF82ECE0101960E94A86BFF2031F00B
:1043900081E090E09093DE028093DD026EE775E0AD
:1043A000CE0101960E94386CBE016F5F7F4FCE0137
:1043B0008F5B9F4F0E94633EF82ECE0101960E94B4
:1043C000A86BFF2031F082E090E09093DE028093B2
:1043D000DD028BEE95E10E948F9120E030E0A90193
:1043E0000E948EB318160CF087C08BEE95E10E94E8
:1043F0008F916093BB027093BC028093BD02909337
:10440000BE022091DD023091DE022130310589F4B7
:104410006093321870933318809334189093351842
:104420006093BF027093C0028093C1029093C20256
:1044300013C02230310581F4609336187093371819
:1044400080933818909339186093AD027093AE0240
:104450008093AF029093B002B901C8010E94E97A3B
:1044600064ED76E0CE0101960E94386CB801CE0171
:1044700001960E94286BBC01CE018A960E94306C86
:10448000CE018A960E943B7CCE018A960E94A86B40
:10449000CE0101960E94A86BC8010E94A86B69E03A
:1044A00073E0CE0101960E94286CCE0101960E9415
:1044B0003B7CCE0101960E94A86B4091BB025091BB
:1044C000BC026091BD027091BE0225E0CE01019652
:1044D0000E94AD6BCE0101960E94DA83CE01019657
:1044E0000E94A86B84EF91E09093AC028093AB02A2
:1044F00064E177E10E94479066ED76E0CE01019697
:104500000E94386C69E076E1CE0101960E94286B2A
:10451000BC01C8010E94306CC8010E94DA83C80146
:104520000E94A86BCE0101960C94C41468EA74E052
:10453000C8010E94386CB801CE018F5B9F4F0E946A
:10454000633E811118C064EE76E0CE0101960E94B0
:10455000386CBE016F5F7F4FCE018F5B9F4F0E9413
:10456000633EFF24F394811101C0F12CCE0101962A
:104570000E94A86B02C0FF24F394C8010E94A86B9C
:10458000FF2009F46EC068EA74E0CE0101960E9433
:10459000386CBE016F5F7F4FCE018F5B9F4F0E94D3
:1045A000633EF82ECE0101960E94A86BFF2099F081
:1045B00042E050E069E076E1CE0101960E948C363F
:1045C000BE016F5F7F4F8BEE95E10E94C56ACE0101
:1045D00001960E94A86B64EE76E0CE0101960E94DF
:1045E000386CBE016F5F7F4FCE018F5B9F4F0E9483
:1045F000633EF82ECE0101960E94A86BFF2099F031
:1046000043E050E069E076E1CE0101960E948C36ED
:10461000BE016F5F7F4F8BEE95E10E94C56ACE01B0
:1046200001960E94A86B8BEE95E10E94344C653B8D
:10463000710540F4CB010E945D7190938A028093D2
:1046400089025ACF66EF72E0CE0101960E94286C73
:10465000CE0101960E943B7CCE0101960E94A86B80
:104660004BCF68EE76E0CE0101960E94386CBE0119
:104670006F5F7F4FCE018F5B9F4F0E94633EF82E8E
:10468000CE0101960E94A86BFF2009F4FAC226E031
:1046900030E044E050E069E076E1CE0101960E940E
:1046A0004C6CBE016F5F7F4F8BEE95E10E94C56A37
:1046B000CE0101960E94A86B8BEE95E10E94344CCE
:1046C0006B017C011B016DE175E0CE0101960E943A
:1046D000386C40910D1650910E168D819E81481BAD
:1046E000590BBE016F5F7F4F89E096E10E94CA9926
:1046F000AC014F5F5F4F69E076E1C8010E948C36E4
:10470000B8018BEE95E10E94C56AC8010E94A86BB2
:10471000CE0101960E94A86B8BEE95E10E948F91CD
:104720004B015C01C60101972D969FAF8EAF2D976F
:104730008091FA188823C1F165E772E0CE010196F5
:104740000E94286CCE0101960E943B7CCE0101960E
:104750000E94A86BB601CE0101960E94E97ACE01B3
:1047600001960E943B7CCE0101960E94A86B6AE1F3
:1047700075E0CE0101960E94386CCE0101960E9430
:104780003B7CCE0101960E94A86B22E0B501A401FA
:10479000CE0101960E94AD6BCE0101960E94DA8394
:1047A000CE0101960E94A86B60E088E30E94E08140
:1047B000E7EAF8E0E491EC8FEDEEF8E0E491F0E068
:1047C000EE0FFF1FE554F64F859194919E8F8D8FCC
:1047D0001FA219A618A6FE01B796CE014F96DF01BB
:1047E0001E928A179B07E1F718870F831D821E828E
:1047F000198229E02A8321E02B832C831C8A1B8ABF
:104800001292E817F907E1F711E0BE01665D7F4FEC
:104810008F8198850E94F3A8882309F45BC067E024
:10482000CE018A960E94539899A98913EECF898167
:1048300081111DC08F8198850E940E99BE01665D11
:104840007F4F8F8198850E94F19840E064EB8F81C3
:1048500098850E94BE988F8198850E946B98082F3A
:104860008F8198850E940E99002309F458C50A810A
:104870008AA5803109F459C5BE01665D7F4FCE011E
:1048800001960E949D99801710F48A810CC08AA518
:10489000803111F48CE007C0BE01665D7F4FCE0110
:1048A00001960E949D998A838D818F5F8D838AA551
:1048B000883209F436C538F4803109F432C58232C1
:1048C00009F0A3CF2EC58B3309F42BC5823409F030
:1048D0009CCF27C58F8198850E940E9940E06CEC93
:1048E0008F8198850E94BE98498164E48F81988564
:1048F0000E94BE988B81882309F442C0EA81E95066
:10490000E33040F4F0E0EE0FFF1FE751FD4F008170
:10491000118102C00EEE12E08C81882359F1898149
:10492000811128C00E9479822B013C019801110F4E
:10493000440B550B61962CAF3DAF4EAF5FAF619707
:104940008F8198850E946B988130D1F00E94798286
:10495000DC01CB0161962CAD3DAD4EAD5FAD6197F5
:10496000821B930BA40BB50B84159505A605B70503
:1049700038F306C0B801110F880B990B0E944182D1
:104980008CE08A8300E010E0AFE74A2EBFE15B2EA7
:104990008FE3682E8D8190E0081719070CF097C0FF
:1049A000402FBE016D5C7F4FCE0101960E9475A91C
:1049B0008A81893038F0782E3CE0381728F4FCE002
:1049C0007F2E02C0E9E07E2E8BA9803141F0BE012E
:1049D0006D5C7F4FCE0101960E949D9901C08CE0D5
:1049E000781609F471C0AE01465D5F4FBE016D5C83
:1049F0007F4FCE0101960E944599882309F464C037
:104A00008BA9803109F460C04BE0741651F05CE072
:104A1000751629F08AE0781207C06EA606C04EA669
:104A200004C09FE59EA701C05EA68F8198850E9465
:104A30000E99BE016D5C7F4F8F8198850E94F19821
:104A400040E06EE48F8198850E94BE9840E06CA59E
:104A50008F8198850E94BE9840E06DA58F819885D2
:104A60000E94BE988BA9803131F040E06EA58F8105
:104A700098850E94BE988F8198850E940E99BE01EC
:104A80006D5C7F4F8F8198850E94F198498168E421
:104A90008F8198850E94BE9864E170E080E090E08C
:104AA0000E9441828981882331F06AE070E080E0D1
:104AB00090E00E9441828F8198850E940E998A81A0
:104AC000871508F4872D8A830F5F1F4F63CF0E81F0
:104AD00010E00B30110514F00AE010E0ABE5CA1647
:104AE000D10408F44CC072EEC72E7AE0D72E5601DE
:104AF000412C512C3201E12CF12CE016F106BCF4D2
:104B00006E2DCE0101960E94AFA99B01AC01F5016B
:104B100061937193819391935F01C301B2010E94EC
:104B200091B22B013C01FFEFEF1AFF0AE6CFB8016B
:104B3000012E000C880B990B0E94FBB09B01AC016D
:104B4000C301B2010E94F5B24B015C01E12CF12CD2
:104B5000E016F1060CF05EC0D6012D913D914D910D
:104B60005C91C501B4010E9490B2F601619371930A
:104B7000819391936F01FFEFEF1AFF0AE9CF1214AF
:104B8000130444F5021513053CF498012150310932
:104B90002D963FAF2EAF2D972C966FAD2C97CE0153
:104BA00001960E94AFA99B01AC012D960EAD1FADE1
:104BB0002D97000F111F000F111F0E51154FC5012A
:104BC000B4010E9490B2D8016D937D938D939C9314
:104BD000139720C02328F1F422EEC22E2AE0D22E11
:104BE000E12CF12CE016F106ACF46E2DCE0101960D
:104BF0000E94AFA99B01AC01C501B4010E9490B213
:104C0000F60161937193819391936F01FFEFEF1A16
:104C1000FF0AE8CF88E2E2EEFAE0ABEEB7E10190FE
:104C20000D928A95E1F784EF91E09093AC02809326
:104C3000AB0264E177E10E94479065ED72E081EF9D
:104C400095E10E94396B44E050E069E076E1CE01E5
:104C500001960E948C36BE016F5F7F4F81EF95E118
:104C60000E94BF6ACE0101960E94A86B61EF75E1B8
:104C7000CE0101960E94306CCE0101960E94DA832B
:104C80001BC36CEE76E0CE0101960E94386CBE012B
:104C90006F5F7F4FCE018F5B9F4F0E94633EF82E68
:104CA000CE0101960E94A86BFF2009F441C047E0A5
:104CB00050E069E076E1CE0101960E948C36BE019B
:104CC0006F5F7F4F8BEE95E10E94C56ACE01019622
:104CD0000E94A86B60E477E0CE0101960E94386CD8
:104CE000BE016F5F7F4F8BEE95E10E94633EF82E11
:104CF000CE0101960E94A86BF11010923D0B67E166
:104D000079E0CE0101960E94386CBE016F5F7F4F43
:104D10008BEE95E10E94633EF82ECE0101960E9433
:104D2000A86BFF2009F4E8CB81E080933D0BE4CB36
:104D300064EF76E0CE0101960E94386CBE016F5F91
:104D40007F4FCE018F5B9F4F0E94633EF82ECE01B6
:104D500001960E94A86BFF20A1F141E068E572E096
:104D6000CE0101960E944E8FBE016F5F7F4F8CE691
:104D700098E10E94157B8CE698E10E94AA7C811143
:104D80000BC069E872E0CE0101960E94286CCE014A
:104D900001960E94DA83B3C08CE698E10E946844D1
:104DA000892B51F08CE698E10E947446682F89EBBC
:104DB00093E10E941469F0CF8CE698E10E946B7C2D
:104DC00081C26BEF76E0CE0101960E94386CBE0185
:104DD0006F5F7F4FCE018F5B9F4F0E94633EF82E27
:104DE000CE0101960E94A86BFF20E1F02DB73EB7DF
:104DF000265231400FB6F8943EBF0FBE2DBFADB75F
:104E0000BEB7119686E291E0E4E1F7E101900D92E0
:104E10000197E1F70E94E58A0FB6F894DEBF0FBE56
:104E2000CDBF50C264E077E0CE0101960E94386C9D
:104E3000BE016F5F7F4FCE018F5B9F4F0E94633E2D
:104E4000F82ECE0101960E94A86BFF2009F45AC0EB
:104E50008DB79EB7865291400FB6F8949EBF0FBE95
:104E60008DBFADB7BEB7119686E291E0E4E1F7E100
:104E700001900D920197E1F70E9452890FB6F894C4
:104E8000DEBF0FBECDBF64EC72E0CE0101960E9482
:104E9000286CEDB7FEB7E652F1400FB6F894FEBFAE
:104EA0000FBEEDBFADB7BEB7119686E291E0E4E16B
:104EB000F7E101900D920197E1F70E94A3870FB6E9
:104EC000F894DEBF0FBECDBF4DB75EB7465251401E
:104ED0000FB6F8945EBF0FBE4DBFADB7BEB711960B
:104EE00086E291E0E4E1F7E101900D920197E1F7AC
:104EF0000E94E58A0FB6F894DEBF0FBECDBFCE018B
:104F000001962FC166E077E0CE0101960E94386CD1
:104F1000BE016F5F7F4FCE018F5B9F4F0E94633E4C
:104F2000F82ECE0101960E94A86BFF20E1F062EB03
:104F300072E0CE0101960E94286CBE016F5F7F4F28
:104F4000C8010E94306CC8010E94DA83C8010E9427
:104F5000A86BADB7BEB7A652B1400FB6F894BEBFAE
:104F60000FBEADBFBCCF6AE077E0CE0101960E94D4
:104F7000386CBE016F5F7F4FCE018F5B9F4F0E94E9
:104F8000633EF82ECE0101960E94A86BFF2009F423
:104F9000EBC066E972E0CE018A960E94286CBE01E1
:104FA000665D7F4FCE0101960E94306CAE014F5F6F
:104FB0005F4F62E070E082E392E00E942441F82EAD
:104FC000CE0101960E94A86BF1101FC0BE01665D64
:104FD0007F4FC8010E94306C6EE077E0C8010E94EC
:104FE000116B6CE376E10E94286BBC01CE01019647
:104FF0000E94306CCE0101960E94DA83CE010196A8
:105000000E94A86BC8010E94A86B68EE73E080E064
:1050100090E00E944182BE01665D7F4FCE01019605
:105020000E94306CAE014F5F5F4F63E070E085E23D
:1050300092E00E942441F82ECE0101960E94A86BB6
:10504000F1101FC0BE01665D7F4FC8010E94306C29
:105050006EE177E0C8010E94116B6CE376E10E947B
:10506000286BBC01CE0101960E94306CCE010196E6
:105070000E94DA83CE0101960E94A86BC8010E94AB
:10508000A86B68EE73E080E090E00E94418260E3EC
:1050900076E1CE0101960E94306CAE014F5F5F4F0A
:1050A00061E070E082E792E00E942441F82ECE0198
:1050B00001960E94A86BF1101EC060E376E1C80162
:1050C0000E94306C6EE177E0C8010E94116B6CE3C6
:1050D00076E10E94286BBC01CE0101960E94306CE3
:1050E000CE0101960E94DA83CE0101960E94A86B40
:1050F000C8010E94A86B68EE73E080E090E00E9417
:10510000418280913D0B882351F143E162E772E0D7
:10511000CE0101960E944E8FBE016F5F7F4F82EAE3
:1051200098E10E94157B82EA98E10E94AA7C88237C
:10513000B1F060E376E182EA98E10E94446D66E9AD
:1051400070E080E090E00E94418282EA98E10E9453
:105150006B7C62E370E080E090E00E944182CE01CF
:105160008A960E94A86BAEC06AE277E0CE010196F3
:105170000E94386CBE016F5F7F4FCE018F5B9F4FE7
:105180000E94633E182FCE0101960E94A86B112346
:10519000F9F096EDE92E9AE0F92E01E010E0809109
:1051A000850290918602801791070CF48BC0D7017D
:1051B0008C91B2E0EB0EF11C60E00E9482816CE207
:1051C00071E080E090E00E9441820F5F1F4FE7CFC7
:1051D0006EE277E0CE0101960E94386CBE016F5FEF
:1051E0007F4FCE018F5B9F4F0E94633E182FCE01F1
:1051F00001960E94A86B1123F9F086EDE82E8AE053
:10520000F82E01E010E080918502909186028017CF
:1052100091070CF457C0F7018081F2E0EF0EF11C0A
:1052200061E00E9482816CE271E080E090E00E9487
:1052300041820F5F1F4FE7CF63E377E0CE01019616
:105240000E94386CBE016F5F7F4FCE018F5B9F4F16
:105250000E94633E182FCE0101960E94A86B112375
:1052600089F127E030E046E050E069E076E1CE01E8
:1052700001960E944C6CBE016F5F7F4F8BEE95E1F3
:105280000E94C56ACE0101960E94A86B8BEE95E143
:105290000E94344C672B19F41092FA1803C081E075
:1052A0008093FA1869E076E1CE0101960E94306C95
:1052B000CE0101960E94C38DCE0101960E94A86B7B
:1052C0001092000280910002882309F456C069E020
:1052D00076E1CE0101960E94306CCE0101960E94CB
:1052E000C38DCE0101960E94A86B47C06AE377E0A8
:1052F000CE0101960E94386CBE016F5F7F4FCE01D8
:10530000C3960E94633E082FCE0101960E94A86BAF
:1053100011E0002311F40C94B3120C94B21219830F
:10532000A6CA8E818F5F8E8370CA0D3008F0ADCA19
:10533000B1CACE018A960E94A86B0C940F1ACE01B6
:105340008A960E94A86B0C94D71CCE018A960E9464
:10535000A86B0C94A61DCE018A960E94A86B0C9493
:105360000F1FCE018A960E94A86B0C945A21CE0181
:10537000C3960E94A86B0C94511BCE018F5B9F4F6C
:105380000E94A86B81E0C05BDF4F0FB6F894DEBFD0
:105390000FBECDBFDF91CF911F910F91FF90EF9086
:1053A000DF90CF90BF90AF909F908F907F906F9045
:1053B0005F904F903F902F9008952F923F924F9281
:1053C0005F926F927F928F929F92AF92BF92CF9295
:1053D000DF92EF92FF920F931F93CF93DF93CDB79E
:1053E000DEB7C554D1090FB6F894DEBF0FBECDBFEE
:1053F00040E052EC61E070E089EB93E10E94287993
:1054000040E855E260E070E08CE193E10E94287989
:1054100040E855E260E070E08FE792E10E94287971
:1054200040E855E260E070E082EE91E10E94287968
:1054300061E088E00E94E08161E089E00E94E08113
:1054400060E08AE30E94E08161E088E00E9482815E
:1054500060E089E00E94828161E08AE00E94E08150
:1054600061E08BE00E94E08160E08BE30E94E081DC
:1054700061E08AE00E94828160E08BE00E9482818C
:105480000E94B08101E00093331112E51093551191
:10549000109234111092561180EF90E00E94E7783C
:1054A00085E590E00E94E77881E00E948B78009388
:1054B00033111093551110923411109256118BEF35
:1054C00090E00E94E77880E090E00E94E77881E039
:1054D0000E948B7884EF91E09093AC028093AB02B2
:1054E00068EE73E080E090E00E94418289EB93E1F6
:1054F0000E94A068182FAAE0EA2EF12C11110BC00F
:1055000089EB93E10E94A068182F6EE170E080E0C3
:1055100090E00E94418221E0E21AF10879F780913F
:10552000AB029091AC02EAE3AE2EE8E1BE2EF4E1CC
:10553000EF2EF7E1FF2EFC01E451F7416F01C601A8
:105540008E0D9F1D0E940EB2F70181937F01AE1652
:10555000BF06A9F760912E1870912F18072E000C26
:10556000880B990B0E94FBB09B01AC010E9492B387
:10557000882331F081E090E090932F1880932E18CB
:105580006091301870913118072E000C880B990B20
:105590000E94FBB09B01AC010E9492B3882331F0C2
:1055A00082E090E09093311880933018153709F419
:1055B000E8C360912A1870912B1880912C18909153
:1055C0002D180E94FBB09B01AC010E9492B3811187
:1055D000D8C38091141790911517819708F0D1C303
:1055E0002DB73EB7265231400FB6F8943EBF0FBEDE
:1055F0002DBFADB7BEB7119686E291E0E4E1F7E1C9
:1056000001900D920197E1F70E94A3870FB6F894DD
:10561000DEBF0FBECDBF153711F01337D9F4EDB78C
:10562000FEB7E652F1400FB6F894FEBF0FBEEDBFD5
:10563000ADB7BEB7119686E291E0E4E1F7E10190E3
:105640000D920197E1F70E94E58A0FB6F894DEBF4C
:105650000FBECDBF6FE974E082E496E10E94396B22
:1056600069E874E08CE396E10E94396B0E94B08196
:1056700062E477E089EB93E10E94206DE12CF12C4C
:1056800007E2DD24D394D092331100935511109288
:1056900034111092561181E00E948B78811118C04C
:1056A0006EE477E089EB93E10E94346D802F0E94D5
:1056B00040800093C2186AE677E089EB93E10E948C
:1056C000346D802F0E9440803FEFE31AF30A0BC035
:1056D000843049F464E877E089EB93E10E94346D0B
:1056E000802F0E9440800F5F003469F6EF2819F484
:1056F0006FE977E002C065EB77E089EB93E10E9408
:10570000206D0E94B0811092C3188091C71882301A
:1057100018F098E09093C3189091C818992339F025
:10572000813029F48091C31884608093C31862E3A8
:1057300070E080E090E00E9441826091C9188EEB99
:1057400098E10E94C04D68EE73E080E090E00E9416
:10575000418260E38EEB98E10E94D34D4BE4E42E4E
:1057600046E4F42EC7010197F1F760E38EEB98E170
:105770000E94D34DC7010197F1F760E38EEB98E1EA
:105780000E94D34D83E592E00197F1F760E28EEB42
:1057900098E10E94D34D8091C31880620E94EC78FA
:1057A00084E08093C4188CE00E94EC7881E00E9431
:1057B000EC785BE3E52E5FE1F52EC7010197F1F789
:1057C00082E08093C51886E00E94EC7882E00E9417
:1057D000EC78C7010197F1F780E40E94EC786CE463
:1057E000E62E62E0F62E74E5C72E72E0D72EF701A2
:1057F00061917F018EEB98E10E94E94DCE14DF04A8
:10580000B1F70E9401840E94F18364E670E080E0B9
:1058100090E00E94418261E774E0CE0101960E940F
:10582000286CCE0101960E94DA83CE0101960E9477
:10583000A86B61E085E30E94E08161E085E30E945E
:10584000828161E08AE00E94E08161E08AE00E945A
:10585000828161E089E30E94E08169E370E08BE48A
:1058600095E10E94566F68EC70E080E090E00E9445
:1058700041828FEF9FEF90938C0280938B029093E5
:105880008A028093890268EE73E080E090E00E94D3
:10589000418260E674E0CE0101960E94286C4AE0E5
:1058A00050E06FEF7FEFCE0101960E946C85CE0134
:1058B00001960E94A86B10926D1410926B141092B6
:1058C00068141092671484E0809366140E947982B1
:1058D0007B0161E0809166140E94E08182E694E1A0
:1058E0000E949F4560E082E30E94E08161E083E3E3
:1058F0000E94E08161E084E30E94E08161E085E351
:105900000E94E08161E085E30E94828183E58CBD95
:105910008DB58E7F8DBD0AE08FEF0E94A4450150AA
:10592000D9F760E0809166140E94828120E030E027
:10593000A90160E082E694E10E94AD45082F8093C2
:105940006C14813049F00E9479826E197F09613DA3
:10595000774060F381E054C02AEA31E040E050E053
:1059600068E082E694E10E94AD4582FF03C00093A7
:105970006D140EC004E00E94A94580936C14015080
:10598000D1F78A3A11F082E03BC082E080936D1437
:1059900080916D14823021F0812C912C540105C02E
:1059A000812C912CA12C30E4B32E20E030E0A90111
:1059B00067E382E694E10E94AD45A501940169E2A6
:1059C00082E694E10E94AD4580936C14882349F0EF
:1059D0000E9479826E197F09613D774030F388E03B
:1059E0000FC080916D14823001F520E030E0A901F4
:1059F0006AE382E694E10E94AD45882341F086E0A7
:105A00008093671482E694E10E949F457CC50E94C2
:105A1000A945807C803C19F483E080936D140E943A
:105A2000A9450E94A9450E94A94582E694E10E94E9
:105A30009F458DB58E7F8DBD8CB58C7F8CBD8CB513
:105A40008CBD81E00E94127F882329F080919114FF
:105A5000882341F058C580E00E94127F882309F412
:105A600052C5F4CF80918514803109F582E080938E
:105A700091141092A3141092A4141092A5141092D1
:105A8000A6148091861490918714A0E0B0E025E0E0
:105A9000880F991FAA1FBB1F2A95D1F780939F14C7
:105AA0009093A014A093A114B093A2141FC08032AD
:105AB00009F029C583E08093911440918814509196
:105AC000891460918A1470918B144093A31450939D
:105AD000A4146093A5147093A6142FE934E18EE604
:105AE00094E10E94717D882309F40DC58EE694E14E
:105AF0009093A8148093A71481E08093901410923F
:105B0000921410929314109294141092951410926F
:105B1000961410929714109298141092991410924F
:105B20009A1410929B1410929C1410929D1410922F
:105B30009E1465E374E0CE0101960E94286CCE01AC
:105B400001960E94DA83CE0101960E94A86B41E083
:105B500069E874E0CE0101960E944E8FBE016F5F2E
:105B60007F4F87E898E10E94157B8091891890917A
:105B70008A189C838B8380918B1890918C18A091AC
:105B80008D18B0918E188D839E83AF83B8878091D6
:105B90008F1890919018A0919118B09192188987C0
:105BA0009A87AB87BC878FEB93E09A8389838DE0DC
:105BB000E3E9F8E1DE011D9601900D928A95E1F787
:105BC0008091A0189091A1189B8F8A8F60E070E05F
:105BD000CE0101960E94EF8D6FE274E0CE01019636
:105BE0000E94286CCE0101960E94DA83CE010196B4
:105BF0000E94A86B68EE73E080E090E00E94418212
:105C000043E162E772E0CE0101960E944E8FBE0131
:105C10006F5F7F4F82EA98E10E94157B67EF73E028
:105C200080E396E10E94396B6CEE73E080E396E1CD
:105C30000E946F6A82EA98E10E94AA7C8823B9F1E7
:105C400069E175E482E792E00E94617E811122C0E1
:105C50006CEB77E0CE0101960E94386CCE01019684
:105C60000E943B7CCE0101960E94A86B62E772E025
:105C7000CE0101960E94386CCE0101960E94DA8313
:105C8000CE0101960E94A86B60E376E182EA98E17A
:105C90000E94446D82EA98E10E946B7C66E970E0A4
:105CA00080E090E00E9441826EEC77E010C067EDEA
:105CB00073E0CE0101960E94286CCE0101960E94ED
:105CC0003B7CCE0101960E94A86B62E772E0CE0198
:105CD00001960E94386CCE0101960E94DA83CE01B3
:105CE00001960E94A86B10923C0B69EC73E0CE0108
:105CF00001960E94286CCE0101960E94DA83CE01A3
:105D000001960E94A86B0E947B666C0168EE73E0AE
:105D100080E090E00E944182E12CF12CCD2809F036
:105D200050C03AE0E316F10409F448C0B701CE01CF
:105D300001960E94E97ACE0101960E94DA83CE0193
:105D400001960E94A86B60ED77E080E090E00E94F1
:105D500041820E947B666C0168EE73E080E090E017
:105D60000E944182CE0101960E946858BE016F5F79
:105D70007F4F89EB93E10E9443638FEFE81AF80AA3
:105D8000CDCF2DB73EB7265231400FB6F8943EBF67
:105D90000FBE2DBFADB7BEB7119686E291E0E4E12C
:105DA000F7E101900D920197E1F70E9452890FB639
:105DB000F894DEBF0FBECDBF15E712CC6DEB73E0DC
:105DC00002C060EB73E0CE0101960E94286CCE0108
:105DD00001960E94DA83CE0101960E94A86B68EEBC
:105DE00073E080E090E00E94418269E175E48FE316
:105DF00092E00E94617E882331F069ED74E48FE3C4
:105E000092E00E94617E66E970E080E090E00E948E
:105E1000418243E16FE372E0CE0101960E944E8F12
:105E2000BE016F5F7F4F82EA98E10E94157B81E09F
:105E300080933C0BCE0101960E946858BE016F5FB3
:105E40007F4F82EA98E10E94436382EA98E10E94D0
:105E50006B7C62E370E080E090E00E9441821092EF
:105E60003C0B0E94067668EE73E080E090E00E94B2
:105E700041820E945D7794E6E92EF12C11110BC04E
:105E800089EB93E10E94A068182F64E170E080E044
:105E900090E00E94418291E0E91AF10879F760EA06
:105EA00073E0CE0101960E94286CCE0101960E94FB
:105EB000DA7DCE0101960E94A86B123711F481E0C1
:105EC00001C080E0DCD566E973E08AE596E10E94D6
:105ED000396BCE010196DED7BE016F5F7F4F8AE539
:105EE00096E10E94BF6ACE0101960E94A86B63E80A
:105EF00073E08AE596E10E946F6A61E773E0CE0184
:105F000001960E94286CCE0101960E94DA7DCE0196
:105F100001960E94A86B67E370E0809187029091E0
:105F200088026BD390930B0B80930A0B6AE576E1A2
:105F3000CE0101960E94306CAE014F5F5F4F62E070
:105F400070E082E392E00E942441182FCE01019676
:105F50000E94A86B111121C06AE576E1CE0101967D
:105F60000E94306C6EE177E0CE0101960E94116BC9
:105F70006CE376E10E94286BBC01CE014C960E9436
:105F8000306CCE014C960E94DA83CE014C960E9472
:105F9000A86BCE0101960E94A86B6AE576E1CE015E
:105FA00001960E94306CAE014F5F5F4F63E070E07E
:105FB00085E292E00E942441182FCE0101960E94B2
:105FC000A86B111121C06AE576E1CE0101960E940D
:105FD000306C6EE177E0CE0101960E94116B6CE3AC
:105FE00076E10E94286BBC01CE014C960E94306C79
:105FF000CE014C960E94DA83CE014C960E94A86B8B
:10600000CE0101960E94A86B68EE73E080E090E0FC
:106010000E9441826E01E0E4CE0ED11C62ED7AE076
:10602000C6010E94386C62ED7AE0CE01CA960E94E9
:10603000386C62ED7AE0CE01C4960E94386C809094
:10604000850290908602B1E8AB2EB2E0BB2E10E341
:10605000E12E17E1F12E01E9602E02E0702E8DE1B4
:10606000282E82E0382E210101E010E080169106F2
:106070000CF45CC0F501119211925F0160E277E1CE
:10608000CE0188960E94386CB701CE0182960E949C
:10609000386CB801CE014C960E94E97A64ED77E045
:1060A000CE0101960E94386CBE01645E7F4FCE0126
:1060B00001960E94286B66E076E00E94116BBE019B
:1060C0006E5D7F4F0E94286B6DE175E00E94116B41
:1060D000BE01685D7F4F0E94286BBC01C6010E9413
:1060E000BF6ACE0101960E94A86BCE014C960E9419
:1060F000A86BCE0182960E94A86BCE0188960E9462
:10610000A86BF30111921192119211923F01F201C9
:1061100011921192119211922F01C8010E94858251
:106120000F5F1F4FF8E0EF0EF11CA0CF7FE0A72E0E
:1061300072E0B72EEDE8EE2EE2E0FE2EF5E1CF2E76
:10614000F2E0DF2E01E010E0A8EE4A2EA3E05A2E86
:10615000612C712C24E0E20EF11C8091850290915B
:106160008602801791070CF4AAC0F5016191719124
:106170005F01CE0188960E94E97A42E050E0BE01BC
:10618000685D7F4FCE018E960E943E78B801CE01A9
:106190004C960E94E97A42E050E0BE01645E7F4F77
:1061A000CE0182960E943E7866ED76E0CE010196A1
:1061B0000E94386CBE016E5D7F4FCE0101960E9439
:1061C000286BBE01625D7F4F0E94286BBC01CE012F
:1061D000C4960E94936BCE0101960E94A86BCE01DB
:1061E00082960E94A86BCE014C960E94A86BCE01AD
:1061F0008E960E94A86BCE0188960E94A86BF7012C
:106200006081718182819381A30192010E9455B2C4
:10621000BA01A90120E0CE0101960E94DC6B48E0A2
:1062200050E0BE016F5F7F4FCE014C960E943E78DA
:10623000BE01645E7F4FCE01C4960E94BF6ACE014C
:106240004C960E94A86BCE0101960E94A86BF601A5
:10625000619171916F01CE0101960E94E97A43E04C
:1062600050E0BE016F5F7F4FCE014C960E943E789A
:10627000BE01645E7F4FCE01C4960E94BF6ACE010C
:106280004C960E94A86BCE0101960E94A86BBE019D
:106290006C5C7F4FCE01CA960E94BF6AF7011082E4
:1062A000118212821382F1011192119211921192B4
:1062B0001F01C8010E9485820F5F1F4F4BCFCE0187
:1062C0004C96E8D568ED77E0CE0101960E94386CD7
:1062D000BE01645E7F4FCE0101960E94286B6AE189
:1062E00075E00E94116BBE01605C7F4F0E94286BBD
:1062F000BC018AE596E10E94936BCE0101960E9453
:10630000A86BCE014C960E94A86BCE010196C2D517
:1063100046E150E0BE016F5F7F4FCE014C960E9478
:106320003E78BE01645E7F4FCE0182960E94306C43
:10633000BE01665C7F4FCE0182960E94286BBC0135
:10634000CE01CA960E94936BCE0182960E94A86BE2
:10635000CE014C960E94A86BCE0101960E94A86BBC
:106360006AE576E1CE0101960E94306CCE0101967D
:106370000E94DA83CE0101960E94A86B6AE576E15D
:10638000CE0101960E94306CAE014F5F5F4F62E01C
:1063900070E082E392E00E942441182FCE01019622
:1063A0000E94A86B111121C06AE576E1CE01019629
:1063B0000E94306C6EE177E0CE0101960E94116B75
:1063C0006CE376E10E94286BBC01CE014C960E94E2
:1063D000306CCE014C960E94DA83CE014C960E941E
:1063E000A86BCE0101960E94A86BBE01665C7F4F30
:1063F000CE0101960E94306CAE014F5F5F4F63E0AB
:1064000070E085E292E00E942441CE0101960E9454
:10641000A86BCE01C4960E94A86BCE01CA960E94BA
:10642000A86BCE01805C9F4F0E94A86B86E990E725
:106430009093C3158093C2152091E415822F022EEC
:10644000000C990B88309105C8F4FC01EE0FFF1F7A
:10645000EE0FFF1FEC53FA4E42EE57E0518340839C
:106460002F5F2093E415880F991F880F991FFC0157
:10647000EA53FA4E8DED91E7918380832091E415E4
:10648000822F022E000C990B88309105C8F4FC0174
:10649000EE0FFF1FEE0FFF1FEC53FA4E48EE57E0D2
:1064A000518340832F5F2093E415880F991F880F35
:1064B000991FFC01EA53FA4E8EE195E791838083A0
:1064C00082E595E10E949C560E94254E60939E0CA9
:1064D00070939F0C8093A00C9093A10C1092A20C2F
:1064E0000E940F868091131880933E0B882331F110
:1064F0000E94254E6093A90C7093AA0C8093AB0C5C
:106500009093AC0C1BC062E574E0CE0101960E9432
:10651000286CCE0101960E94DA83CE0101960E947A
:10652000A86B61E474E0CE0101960E94286C6AE0D9
:1065300070E0CE0101960E940D7C58CBCB5BDF4F03
:106540000FB6F894DEBF0FBECDBFDF91CF911F9184
:106550000F91FF90EF90DF90CF90BF90AF909F9002
:106560008F907F906F905F904F903F902F90089505
:10657000FC01768765870895DC01ED91FC91068C1E
:10658000F78DE02D199591E089270895862F0895BC
:1065900081E08627089521E0FC018485883008F099
:1065A00020E0822F0895FC01848595850895FC01E3
:1065B00084899589089523E534E0FC0131832083A3
:1065C000FB014089518962897389FC0142835383AD
:1065D000648375830895DC01ED91FC91048CF58D45
:1065E000E02D199480E0089580E090E008950A96E7
:1065F0000C9490540A960C94CA528F929F92AF9228
:10660000BF92CF92DF92EF92FF920F931F93CF939F
:10661000DF938C01862F0B30110509F06FC090912C
:106620004718992309F0F89462E10E94887B209131
:106630004718222309F07894009709F072C0E0907F
:106640004218F09043186F2D70E080E090E00E94B7
:10665000FBB02DEC3CEC4CEC5DE30E945AB14B01DD
:106660005C016E2D70E080E090E00E94FBB09B0129
:10667000AC01C501B4010E9491B260933A187093C5
:106680003B1880933C1890933D18C0914418D091CA
:1066900045186C2F6F7770E080E090E00E94FBB0AF
:1066A0004B015C016D2F70E080E090E00E94FBB038
:1066B0002DEC3CEC4CEC5DE30E945AB19B01AC012B
:1066C000C501B4010E9491B2C7FD09C060933E1894
:1066D00070933F1880934018909341180BC0DC01D1
:1066E000CB01B05880933E1890933F18A093401868
:1066F000B0934118FE0CCF0DCD0F71C006311105BE
:1067000009F0B4C090914718992309F0F89461E01A
:106710000E94887B20914718222309F078940097E3
:10672000A9F040E050EC69E774EC40933A185093BC
:106730003B1860933C1870933D1840933E1850935B
:106740003F18609340187093411895C0F09043181B
:10675000D0914218609142187091431876276727AC
:10676000762780E090E00E94F9B02DEC3CEC4CECF8
:106770005DE30E945AB160933A1870933B1880937E
:106780003C1890933D18E0904518C09144188C2F08
:106790008F776E2D70E0782B80E090E00E94F9B04A
:1067A0002DEC3CEC4CEC5DE30E945AB1C7FD09C0F6
:1067B00060933E1870933F1880934018909341184F
:1067C0000BC0DC01CB01B05880933E1890933F186A
:1067D000A0934018B0934118DF0DED0ECE0D8091BF
:1067E0004618C81346C0C0903A18D0903B18E090A5
:1067F0003C18F0903D1820E030E048EC52E4C7012E
:10680000B6010E948EB318161CF0C0E0D0E002C0A2
:10681000CBEFDFEF20E030E0A901C701B6010E9415
:10682000F5B087FF02C0CAEFDFEFC0903E18D090EE
:106830003F18E0904018F090411820E030E048EC1C
:1068400052ECC701B6010E94F5B087FF02C0C9EF44
:10685000DFEF20E030E040EF52E4C701B6010E94D4
:106860008EB31816ACF4C8EFDFEF12C0CFEFDFEF36
:106870000FC08FEF9FEF8F3FFFEF9F0709F4E2C03C
:10688000009709F4B0CF029609F4E8C0CCEFDFEF2F
:106890000C30110509F0E5C081E0809333118CE5DF
:1068A00080935511109234111092561180E090E0AF
:1068B0000E94E77881E00E948B7865E08CE50E9479
:1068C000467B1092CD118093CC11C82FD0E0209739
:1068D000A1F0C530D105A4F000ED11E186E594E109
:1068E0000E94834CF80180870F5F1F4FC801805DB5
:1068F00091418C179D0794F306C0CEEFDFEFB1C036
:10690000CDEFDFEFAEC0C091D8110091D911602F4B
:1069100070E080E090E00E94FBB02DEC3CEC4CEC91
:106920005DE30E945AB16B017C016C2F70E080E046
:1069300090E00E94FBB09B01AC01C701B6010E9430
:1069400091B26093D0117093D1118093D211909332
:10695000D311D091DA111091DB116D2F6F7770E0A8
:1069600080E090E00E94FBB06B017C01612F70E041
:1069700080E090E00E94FBB02DEC3CEC4CEC5DE341
:106980000E945AB19B01AC01C701B6010E9491B2AD
:10699000D7FF5BC0DC01CB01B0588093D41190933A
:1069A000D511A093D611B093D7118C2F800FC82F7B
:1069B000CD0FC10F8091DC11C81344C0C090D0111D
:1069C000D090D111E090D211F090D31120E030E0BE
:1069D00048EC52E4C701B6010E948EB318161CF0B1
:1069E000C0E0D0E002C0CBEFDFEF20E030E040EAD3
:1069F00050E4C701B6010E94F5B087FF02C0CAEF9C
:106A0000DFEFC090D411D090D511E090D611F09066
:106A1000D71120E030E040EF51ECC701B6010E94F1
:106A2000F5B087FF02C0C9EFDFEF20E030E040EFB4
:106A300052E4C701B6010E948EB3181694F4C8EF51
:106A4000DFEF0FC0CFEFDFEF0CC06093D411709376
:106A5000D5118093D6119093D711A7CFCEEFDFEF4A
:106A600017CFCE01DF91CF911F910F91FF90EF9043
:106A7000DF90CF90BF90AF909F908F900895DF925E
:106A8000EF92FF920F931F93CF93DF93D82EC4ED15
:106A9000DAE08E01EE24E394F12C0E5F1F4F80911B
:106AA0008502909186028E159F05ACF061E0D801B9
:106AB0008C910E94E0816091DE11F80180810E943A
:106AC000828164EF71E080E090E00E944182FFEFFC
:106AD000EF1AFF0AE2CFDD2009F45AC001E010E00E
:106AE000229680918502909186020817190724F555
:106AF0006091E01188810E94828168EE73E080E0FD
:106B000090E00E9441820F5F1F4F6091E0118A81E7
:106B10000E94828168EE73E080E090E00E944182F2
:106B20006091DE1188810E94828168EE73E080E0CE
:106B300090E00E944182D4CF68EE73E080E090E064
:106B40000E9441822FE0E22E22E0F22E06ED1AE0B2
:106B5000C1E0D0E080918502909186028C179D075C
:106B6000BCF0D701ED91FD917D01D8018C910E5FB4
:106B70001F4FEE0FFF1FE252FE4E60810E94828186
:106B800068EC70E080E090E00E9441822196E2CFC4
:106B9000DF91CF911F910F91FF90EF90DF900895BB
:106BA000CF92DF92EF92FF920F931F93CF93DF93D9
:106BB000CDB7DEB7A0970FB6F894DEBF0FBECDBF3E
:106BC0006C018B0140E050E07C018AE0E80EF11C92
:106BD000CA010196F8012491E1E0F0E0EC0FFD1FFD
:106BE000E40FF51F2083222391F08032910521F0DC
:106BF0000F5F1F4FAC01ECCF40E250E0BE016F5F72
:106C00007F4FC7010E94905480E090E0F1CF02973F
:106C100038F0BE016F5F7F4FC6010A960E94905404
:106C2000A0960FB6F894DEBF0FBECDBFDF91CF9117
:106C30001F910F91FF90EF90DF90CF900895EF920A
:106C4000FF920F931F93CF93DF93EC018B017A0197
:106C50006FE075E0A5DFB801CE010E94346D8E01B2
:106C6000065F1F4F42E050E060EB79E0C8010E94F0
:106C70009054E114F10421F0B701CE010E94346D6B
:106C800042E050E060EB79E0C801DF91CF911F91C5
:106C90000F91FF90EF900C94905461EB74E080CFD3
:106CA000FC01138212828FE594E09183808388EE49
:106CB00093E0A0E0B0E084839583A683B783089532
:106CC000CF93DF93EC01ECDF8DE193E09983888330
:106CD00083E594E09F878E87188A198A1A8A1B8A0F
:106CE00088E0888FDF91CF9108956115710579F063
:106CF000FB0101900020E9F73197AF01461B570BCC
:106D0000DC01ED91FC910280F381E02D199480E08B
:106D100090E008950A96E9CFCF93DF93EC01FB0151
:106D2000248135810E944C6CCE01DF91CF91089572
:106D3000EF92FF920F931F93CF93DF9300D000D079
:106D4000CDB7DEB78C017B0162ED7AE00E94386C32
:106D50008AE0E816F1042CF460E477E0C8010E94B0
:106D6000B16AB701CE0101960E94E97ABE016F5F58
:106D70007F4FC8010E94BF6ACE0101960E94A86B96
:106D8000C80126960FB6F894DEBF0FBECDBFDF91C7
:106D9000CF911F910F91FF90EF9008950F931F9344
:106DA000CF93DF93CDB7DEB72C970FB6F894DEBF45
:106DB0000FBECDBF8C010E94884FBC01C801B8DF57
:106DC0000E94824FBC01CE010796B2DF66E076E0FA
:106DD000CE0101960E94386CBE01695F7F4FCE01E3
:106DE00001960E94286BBC01C8010E94BF6ACE01B7
:106DF00001960E94A86BCE0107960E94A86B6AE1DB
:106E000075E0C8010E94B16A0E947C4FBC01CE01AE
:106E100001968EDFBE016F5F7F4FC8010E94BF6A7F
:106E2000CE0101960E94A86B6CEE77E0C8010E942B
:106E3000B16A0E94764FBC01CE01019679DFBE0196
:106E40006F5F7F4FC8010E94BF6ACE0101960E940A
:106E5000A86B6CEE77E0C8010E94B16A0E946E4F89
:106E6000BC01CE01019664DFBE016F5F7F4FC80198
:106E70000E94BF6ACE0101960E94A86BC8012C96A1
:106E80000FB6F894DEBF0FBECDBFDF91CF911F913B
:106E90000F9108950F931F93CF93DF93CDB7DEB774
:106EA0002C970FB6F894DEBF0FBECDBF8C010E94A9
:106EB000884FBC01C8013CDF0E94824FBC01CE015B
:106EC000079636DF66E076E0CE0101960E94386CC8
:106ED000BE01695F7F4FCE0101960E94286BBC0105
:106EE000C8010E94BF6ACE0101960E94A86BCE0124
:106EF00007960E94A86B0E94254E0E946B4E6091DF
:106F0000480D70E0CE01079613DF66E076E0CE0113
:106F100001960E94386CBE01695F7F4FCE010196D9
:106F20000E94286BBC01C8010E94BF6ACE01019675
:106F30000E94A86BCE0107960E94A86B6AE175E0DB
:106F4000C8010E94B16A0E947C4FBC01CE0101962B
:106F5000EFDEBE016F5F7F4FC8010E94BF6ACE01A6
:106F600001960E94A86B6CEE77E0C8010E94B16A9E
:106F70000E94764FBC01CE010196DADEBE016F5F42
:106F80007F4FC8010E94BF6ACE0101960E94A86B84
:106F90006CEE77E0C8010E94B16A0E946E4FBC019E
:106FA000CE010196C5DEBE016F5F7F4FC8010E9412
:106FB000BF6ACE0101960E94A86BC8012C960FB63D
:106FC000F894DEBF0FBECDBFDF91CF911F910F911F
:106FD00008956F927F928F929F92AF92BF92CF92BD
:106FE000DF92EF92FF920F931F93CF93DF93CDB772
:106FF000DEB7A0970FB6F894DEBF0FBECDBF62ED2F
:107000007AE084E596E10E947E6B62ED7AE088E4A6
:1070100096E10E947E6B3FE0C32E32E0D32E40E328
:10702000842E47E1942E0FE712E054EDA52E5AE08E
:10703000B52E65E0662E62E0762EEE24E394F12C08
:1070400080918502909186028E159F050CF47BC07D
:10705000F30181919191A191B1913F01892B8A2BEB
:107060008B2BF9F4F80182819381F6012081318123
:1070700082179307B1F0880F991FFC01E252FE4E70
:107080006081F50182810E948281F8018281938171
:10709000F6019183808364E670E080E090E00E94D6
:1070A0004182F601619171916F01CE0145960E9476
:1070B000E97AB701CE010F960E94E97AB401CE01B8
:1070C00009960E94386C6AE175E0CE0101960E9433
:1070D000386CBE01675F7F4FCE0101960E94286B1E
:1070E0006EEE77E00E94116BBE01615F7F4F0E94E0
:1070F000286B6DE175E00E94116BBE016B5E7F4FE6
:107100000E94286BBC0184E596E10E94BF6ACE0113
:1071100001960E94A86BCE0109960E94A86BCE0131
:107120000F960E94A86BCE0145960E94A86BFFEFB8
:10713000EF1AFF0A88E0880E911C0E5F1F4FE2E0F5
:10714000AE0EB11C7DCFE0912E18F0912F18EE0FEE
:10715000FF1FE35FFD4F60817181CE0101960E94A8
:10716000E97A46E050E0BE016F5F7F4FCE0109969D
:107170000E943E78BE01675F7F4F88E496E10E94DF
:10718000BF6ACE0109960E94A86BCE0101960E94AB
:10719000A86BE0913018F0913118EE0FFF1FE35FFC
:1071A000FD4F60817181CE0101960E94E97A46E02F
:1071B00050E0BE016F5F7F4FCE0109960E943E787E
:1071C000BE01675F7F4F88E496E10E94BF6ACE01EF
:1071D00009960E94A86BCE0101960E94A86B6AE1F5
:1071E00075E0CE0145960E94386C0E94798228EEA7
:1071F00033E040E050E00E9433B269017A0162ED71
:107200007AE0CE014B960E94386C62ED7AE08AE516
:1072100096E10E947E6BCE0101963CDE44E150E097
:10722000BE016F5F7F4FCE0109960E943E78BE017E
:10723000675F7F4F8AE596E10E94C56ACE01099695
:107240000E94A86BCE0101960E94A86B2AE0B701AC
:10725000A601CE0109960E94DC6B48E050E0BE0119
:10726000675F7F4FCE010F960E943E786AE576E118
:10727000CE0101960E94306CBE01615F7F4FCE014E
:1072800001960E94286BBC018EE496E10E94936BEC
:10729000CE0101960E94A86BCE010F960E94A86BAA
:1072A000CE0109960E94A86B2AE0B701A601CE0183
:1072B00009960E94DC6B61EF77E0CE0101960E9497
:1072C000386CBE01675F7F4FCE0101960E94286B2C
:1072D000BE016B5E7F4F0E94286BBC018AE596E180
:1072E0000E94BF6ACE0101960E94A86BCE0109964A
:1072F0000E94A86B40915F115091601160916111E3
:107300007091621121E0CE0101960E94AD6BBE0129
:107310006F5F7F4FCE014B960E94C56ACE010196EA
:107320000E94A86B68EF77E0CE0101960E94386C4E
:10733000BE01655E7F4FCE0101960E94286BBE01A3
:107340006B5E7F4F0E94286BBC018AE596E10E942C
:10735000BF6ACE0101960E94A86BBE01655E7F4F99
:10736000CE0101960E94306C46E050E0BE016F5F96
:107370007F4FCE0109960E943E78BE01675F7F4F26
:107380008EE496E10E94BF6ACE0109960E94A86B26
:10739000CE0101960E94A86B40915711509158114F
:1073A0006091591170915A1121E0CE0101960E940D
:1073B000AD6BBE016F5F7F4FCE014B960E94C56AD9
:1073C000CE0101960E94A86B66E078E0CE0101969E
:1073D0000E94386CBE01655E7F4FCE0101960E940F
:1073E000286BBE016B5E7F4F0E94286BBC018AE553
:1073F00096E10E94BF6ACE0101960E94A86BBE0171
:10740000655E7F4FCE0101960E94306C46E050E0F1
:10741000BE016F5F7F4FCE0109960E943E78BE018C
:10742000675F7F4F8EE496E10E94BF6ACE010996A6
:107430000E94A86BCE0101960E94A86B80910A0B56
:1074400090910B0B892B59F067E370E080918702D4
:1074500090918802D2D890930B0B80930A0B809165
:107460000A0B90910B0B892B09F0A7C00E944B8649
:1074700029833A834B835C836D837E838F839887D4
:1074800049815A816B817C8121E0CE0109960E945D
:10749000AD6BBE01675F7F4FCE014B960E94C56A00
:1074A000CE0109960E94A86B60E178E0CE010996B2
:1074B0000E94386CBE01655E7F4FCE0109960E9426
:1074C000286BBE016B5E7F4F0E94286BBC018AE572
:1074D00096E10E94BF6ACE0109960E94A86BBE0188
:1074E000655E7F4FCE0109960E94306C46E050E009
:1074F000BE01675F7F4FCE010F960E943E78BE01AE
:10750000615F7F4F8EE496E10E94BF6ACE010F96C5
:107510000E94A86BCE0109960E94A86B4D815E81E6
:107520006F81788521E0CE0109960E94AD6BBE0186
:10753000675F7F4FCE014B960E94C56ACE010996C8
:107540000E94A86B6BE178E0CE0109960E94386C2E
:10755000BE01655E7F4FCE0109960E94286BBE0179
:107560006B5E7F4F0E94286BBC018AE596E10E940A
:10757000BF6ACE0109960E94A86BBE01655E7F4F6F
:10758000CE0109960E94306C46E050E0BE01675F74
:107590007F4FCE010F960E943E78BE01615F7F4F04
:1075A0008EE496E10E94BF6ACE010F960E94A86BFE
:1075B000CE0109960E94A86B18C061E278E08AE5C6
:1075C00096E10E94B16A60E378E08EE496E10E9461
:1075D000B16A67E378E08AE596E10E94B16A60E308
:1075E00078E08EE496E10E94B16A64E576E18AE58E
:1075F00096E10E94BF6A6AE175E0CE0101960E94A1
:10760000386C68E476E1CE0101960E94286BBC01DB
:107610008EE496E10E94BF6ACE0101960E94A86B9B
:107620006EE476E1CE0101960E94306CCE010196A7
:107630000E94DA83CE0101960E94A86B6AE070E096
:1076400080E090E00E944182CE014B960E94A86BA0
:10765000CE0145960E94A86BA0960FB6F894DEBFA7
:107660000FBECDBFDF91CF911F910F91FF90EF9093
:10767000DF90CF90BF90AF909F908F907F906F9052
:107680000895CF93DF9300D000D0CDB7DEB768EB7D
:1076900072E28FE096E10E94725480E3ECE0FBE03E
:1076A000DF011D928A95E9F783EE80930C0B86E04B
:1076B00080930E0B8CEE80930F0B81E38093180B5D
:1076C0009EE49093190B80931A0B84E380931B0B19
:1076D00064E572E0CE0101960E947B6D4BE750E0BD
:1076E000BE016F5F7F4F8FE096E10E947C5540E3C3
:1076F00050E06CE07BE08FE096E10E9428548FE040
:1077000096E10E94DB5668EE73E080E090E00E9414
:1077100041828FE096E10E94CC53892BB1F140E386
:1077200050E06CE07BE08FE096E10E94585360915E
:10773000340B7091350B762767277627CB01A0E0B5
:10774000B0E0BC01552744278091360B9091370B50
:10775000982789279827A0E0B0E0842B952BA62BAB
:10776000B72BBC01CD017E508A4A93480E94FE4D42
:107770000E94254E6093970C7093980C8093990CFF
:1077800090939A0C81E090E002C080E090E0269611
:107790000FB6F894DEBF0FBECDBFDF91CF91089535
:1077A0004F925F926F927F928F929F92AF92BF9211
:1077B000CF92DF92EF92FF920F931F93CF93DF93BD
:1077C000CDB7DEB763970FB6F894DEBF0FBECDBF5F
:1077D0007C015B013A01FB0120E080E090E06AE07F
:1077E0003191332309F140ED430F4A3080F4689F13
:1077F000A001699F500D1124CA01C097830F911DEC
:1078000037FD9A958F3F910559F350F313C03E32DF
:1078100089F4233079F0D301A20FB11D12968C9315
:107820002F5F80E090E0DCCF233021F4F3018583EB
:1078300081E021C0F701428153816481758180918B
:10784000B3149091B414A091B514B091B614481724
:1078500059076A077B0709F491C10E947982870161
:10786000085F1F4F6F7077277C5FC8010E947254BA
:10787000813019F080E090E0D9C183E594E09A83EB
:107880008983F70182819381A481B5818B839C8355
:10789000AD83BE8345E350E0BE016F5F7F4FC801FB
:1078A0000E947C55892B19F4C12CD12C62C10E94F5
:1078B0007982F7017783668342E050E0B7016A5F1F
:1078C0007F4FC8010E94285481E090E09A83898309
:1078D00042E050E0BE016F5F7F4FC8010E94285414
:1078E00080E091E09A83898342E050E0BE016F5FBF
:1078F0007F4FC8010E9428541A82198242E050E04A
:10790000BE016F5F7F4FC8010E94285442E050E0E3
:10791000BE016F5F7F4FC8010E94285442E050E0D3
:10792000BE016F5F7F4FC8010E9428544501F501D9
:107930008081882301F164015601F60181912F01B4
:10794000882321F08E3211F06201F6CFC818D908D1
:107950001C141D0474F4CD8641E050E0BE01635F49
:107960007F4FC8010E942854A601B401C8010E949B
:1079700028544201DCCF1D8641E050E0BE01635F28
:107980007F4FC8010E942854C12CDD24D394DA8291
:10799000C98242E050E0BE016F5F7F4FC8010E9484
:1079A0002854DA82C98242E050E0BE016F5F7F4F07
:1079B000C8010E942854C8010E94DB56892B09F493
:1079C00073CFE3E0AE2EB12C230122E0420E511C16
:1079D0000E9479823B014C01C8010E94CC531816C9
:1079E0001906A4F00E947982DC01CB01861997095F
:1079F000A809B90989389341A105B105D0F462E31A
:107A000070E080E090E00E944182E6CFF701428181
:107A1000538164817581808D918DA28DB38D4817BE
:107A200059076A077B0749F4848D958DC59729F41A
:107A300009C0CC24CA94DC2C93C05EEFC52EDD2493
:107A4000DA948EC0F70181A192A10C970CF4E9C0E1
:107A50004CE050E0BE016F5F7F4FC8010E94585359
:107A60008B819C819827892798279A8B898BF7018E
:107A70004681578129813A814217530709F0C2C0D4
:107A800097FFC0C08F709270892B09F0C0C06F80C3
:107A900078847624672476246114710409F4BCC0C8
:107AA000C12CD12C8D819E81982789279827C816B3
:107AB000D90608F466C0812C912C41E050E0BE014B
:107AC0006D5E7F4FC8010E9458534B89842F807C84
:107AD00009F076C0442331F050E060E070E0C80166
:107AE0000E9458538B898111E8CF42E050E0BE01DB
:107AF000615F7F4FC8010E94585342E050E0BE01D1
:107B0000635F7F4FC8010E94585344E050E060E03B
:107B100070E0C8010E94585342E050E0BE016F5E21
:107B20007F4FC8010E9458538F85988949895A8987
:107B30008115914009F04DC0CD84DE84DC24CD2434
:107B4000DC2481E0C816D10409F043C0411554403B
:107B500009F053C044E050E0B201C8010E945853FC
:107B600021E0A21AB10829F0FFEFCF16DF0609F4D1
:107B70002FCFC8010E942153C60158C08EEF9FEF3E
:107B800055C041E050E0BE01635F7F4FC8010E94D5
:107B900058534D85442331F050E060E070E0C80157
:107BA0000E9458538D858111ECCF44E050E060E095
:107BB00070E0C8010E945853FFEFCF1ADF0A72CF5E
:107BC00041E050E060E070E0C8010E9458531B8A19
:107BD00089CF54274527542760E070E0C8010E94F0
:107BE0005853FFEF8F1A9F0A6814790409F065CF84
:107BF00096EFC92EDD24DA94B3CF77EFC72EDD24BC
:107C0000DA94AECF4CEFC42EDD24DA94A9CF3BEF4B
:107C1000C32EDD24DA94A4CF2AEFC22EDD24DA9419
:107C20009FCF8DEFC82EDD24DA949ACF63960FB6DE
:107C3000F894DEBF0FBECDBFDF91CF911F910F91A2
:107C4000FF90EF90DF90CF90BF90AF909F908F907C
:107C50007F906F905F904F9008950F931F93CF93F5
:107C6000DF9341155105E1F061157105C9F0FC0183
:107C7000C481D581209719F4FB01108211C04150B5
:107C800051094C175D0708F4EA018B01FC01608182
:107C90007181AE01C8010E943CB6C00FD11F18828D
:107CA000DF91CF911F910F910895CF93DF93EC0156
:107CB0000E949E6A811103C0CE010E94FF6ACE011C
:107CC000DF91CF910895FB0144815581FC0124810E
:107CD00035812417350778F080819181009759F01C
:107CE000FB01608171816115710529F00E942EB63A
:107CF00021E0892B09F020E0822F089544E050E034
:107D0000BC018FE090E00C9442472F923F924F923B
:107D10005F926F927F928F929F92AF92BF92CF921B
:107D2000DF92EF92FF920F931F93CF93DF93CDB724
:107D3000DEB7AC970FB6F894DEBF0FBECDBF8C0197
:107D400062ED7AE08AE296E10E947E6B67E370E082
:107D500080918702909188020E94FD321C0166E3A7
:107D600076E0C8010E94D03561E478E0C8010E9445
:107D7000346D68E478E1CE0101960E94306CBE015A
:107D80006F5F7F4FC8010E94366DCE0101960E9441
:107D9000A86B6AE478E0C8010E94346D0E94798281
:107DA00028EE33E040E050E00E9433B229013A016E
:107DB000CE0109966FD860E578E0CE010F960E945B
:107DC000386CBE01675F7F4FCE010F960E94286B13
:107DD000BC01CE0101960E94306CBE016F5F7F4FE7
:107DE000C8010E94366DCE0101960E94A86BCE019B
:107DF0000F960E94A86BCE0109960E94A86BC30142
:107E0000B20120E13EE040E050E00E9455B24B015B
:107E10005C01B901CE0187960E9498364CE3C42ECE
:107E2000D12CE12CF12CC501B401A70196010E94CF
:107E300055B2B901CE0101960E94983666E076E00F
:107E4000CE0109960E94386CBE016F5F7F4FCE0154
:107E500009960E94286BBC01CE0187960E94BF6ADA
:107E6000CE0109960E94A86BCE0101960E94A86BD4
:107E7000C301B201A70196010E9455B2CE0101963D
:107E80000E94983666E076E0CE0109960E94386C32
:107E9000BE016F5F7F4FCE0109960E94286BBC0127
:107EA000CE0187960E94BF6ACE0109960E94A86BF8
:107EB000CE0101960E94A86B6AE578E0CE01099692
:107EC0000E94386CBE01695D7F4FCE0109960E9409
:107ED000286B6DE578E00E94116BBC01CE01019624
:107EE0000E94306CBE016F5F7F4FC8010E94366DEB
:107EF000CE0101960E94A86BCE0109960E94A86B44
:107F00006BE678E0C8010E94346DCE0101960E94B4
:107F10006858B801CE0101960E94D86C66E678E0F8
:107F2000C8010E94206D0E944B8629833A834B83AF
:107F30005C836D837E838F83988749815A816B81AF
:107F40007C8121E0CE010F960E94AD6BBE01615F86
:107F50007F4FCE0109960E94306C63E778E0CE0136
:107F600009960E94116BBC018AE296E10E94936B14
:107F7000CE0109960E94A86BCE010F960E94A86BB5
:107F80006AE778E0CE010F960E94386C6AE276E1EB
:107F9000CE010F960E94286BBC01CE0109960E946B
:107FA000306CBE01675F7F4FC8010E94366DCE0105
:107FB00009960E94A86BCE010F960E94A86B4D8176
:107FC0005E816F81788521E0CE0109960E94AD6BBC
:107FD000BE01675F7F4F8AE296E10E94C56ACE01CB
:107FE00009960E94A86B6CE878E0CE010F960E947B
:107FF000386C6AE276E1CE010F960E94286B6DE93B
:1080000078E00E94116BBC01CE0109960E94306C91
:10801000BE01675F7F4FC8010E94366DCE01099691
:108020000E94A86BCE010F960E94A86B40915F1131
:1080300050916011609161117091621122E0CE0146
:108040000F960E94AD6B64EA78E0CE0145960E94DF
:10805000386CBE01615F7F4FCE0145960E94286B50
:1080600066EB78E00E94116BBC01CE0109960E947C
:10807000306CBE01675F7F4FC8010E94366DCE0134
:1080800009960E94A86BCE0145960E94A86BCE016E
:108090000F960E94A86B4091571150915811609112
:1080A000591170915A1122E0CE010F960E94AD6BCA
:1080B0006FEB78E0CE0145960E94386CBE01615F9F
:1080C0007F4FCE0145960E94286B66EB78E00E94B8
:1080D000116BBC01CE0109960E94306CBE01675F36
:1080E0007F4FC8010E94366DCE0109960E94A86B91
:1080F000CE0145960E94A86BCE010F960E94A86BF8
:1081000086EF28168FEF38062CF461E176E0C8017F
:108110000E94D03561EF75E0C8010E94D03591E82A
:10812000A92E92E0B92E20E3C22E27E1D22EEE2412
:10813000E394F12C80918502909186028E159F0523
:108140000CF465C0F501619171915F01660F771FB5
:10815000660F771F605E784ECE0109960E94386CDC
:10816000B601CE010F960E94386CB701CE014B9636
:108170000E94E97A66ED76E0CE0181960E94386C25
:10818000BE01655E7F4FCE0181960E94286B6AE139
:1081900075E00E94116BBC01CE0145960E94306CC7
:1081A000BE016B5E7F4FC8010E94366DBE01615FEC
:1081B0007F4FC8010E94366D6DEC78E0C8010E94C7
:1081C000346DBE01675F7F4FC8010E94366D62ED5E
:1081D00078E0C8010E94346DCE0145960E94A86BDC
:1081E000CE0181960E94A86BCE014B960E94A86B8F
:1081F000CE010F960E94A86BCE0109960E94A86B33
:10820000FFEFEF1AFF0A88E0C80ED11C93CFCE0112
:1082100087960E94A86BAC960FB6F894DEBF0FBE8F
:10822000CDBFDF91CF911F910F91FF90EF90DF9025
:10823000CF90BF90AF909F908F907F906F905F9006
:108240004F903F902F9008959F92AF92BF92CF9200
:10825000DF92EF92FF920F931F93CF93DF93CDB7EF
:10826000DEB7C859D1090FB6F894DEBF0FBECDBF37
:108270005C017B016A016CE677E1CE018D569F4F70
:108280000E94386C69E874E08E010F5F1F4FC801CF
:108290000E94386CB801CE018D569F4F14DD982E88
:1082A000C8010E94A86B911014C069E874E0C8016D
:1082B0000E94386CBE016D567F4FC8010E94286B2A
:1082C000BC01CE018D569F4F0E94936BC8010E9446
:1082D000A86BB501CE0183579F4F0E94386C21E0F7
:1082E000E216F10419F467ED78E00DC032E0E31610
:1082F000F10419F462EE78E006C083E0E816F104B8
:1083000039F46AEE78E0CE018D569F4F0E94B16A33
:1083100060E0CE018D569F4F0E949E6AB601C80153
:108320000E94306C6AE0C801C0DCBC01CE018957F4
:108330009F4F0E94306CC8010E94A86BC956DF4F46
:1083400048815981C759D040B801CE018D569F4F01
:1083500084DC8091D20B882399F162EF78E0CE0122
:108360008F579F4F0E94386CCE018F579F4F0E94AE
:108370003B7CCE018F579F4F0E94A86BBE016D566C
:108380007F4FCE018F579F4F0E94306CCE018F5789
:108390009F4F0E943B7CCE018F579F4F0E94A86B3E
:1083A000B801CE018F579F4F0E94386CCE018F5776
:1083B0009F4F0E943B7CCE018F579F4F0E94A86B1E
:1083C000C857DF4F8881C858D0408F93C957DF4FB7
:1083D0008881C758D0408F93C257DF4F8881CE58CD
:1083E000D0408F93C357DF4F8881CD58D0408F93B3
:1083F00082E099E09F938F9383EDE82E8BE0F82E37
:10840000FF92EF920E9465B640E550E062EC7BE09F
:1084100083EF96E10E9495580FB6F894DEBF0FBE29
:10842000CDBF019709F05AC01F930F9388E099E0E0
:108430009F938F9302E41BE01F930F930E9465B6F6
:10844000B80183EF96E10E94206D82EC9BE09F9340
:108450008F9389E199E09F938F931F930F930E94CD
:1084600065B6B80183EF96E10E94206D62E975E080
:1084700083EF96E10E94576D60EB79E083EF96E120
:108480000E947536F70101900020E9F73197E35D0E
:10849000FB40FF93EF9382E299E09F938F931F93AA
:1084A0000F930E9465B6B80183EF96E10E94206D9C
:1084B000B70183EF96E10E94346D62E370E080E0E3
:1084C00090E00E94418283EF96E10E94FF540FB634
:1084D000F894DEBF0FBECDBF11E034C065ED75E08E
:1084E000CE018F579F4F0E94286CCE018F579F4F10
:1084F0000E94DA83CE018F579F4F0E94A86B61EED6
:1085000075E0CE018F579F4F0E94286CCE018F5788
:108510009F4F0E943B7CCE018F579F4F0E94A86BBC
:1085200063ED7BE0CE018F579F4F0E94386CCE01E8
:108530008F579F4F0E94DA83CE018F579F4F0E9423
:10854000A86B10E0CE0189579F4F0E94A86BCE0107
:1085500083579F4F0E94A86BCE018D569F4F0E945C
:10856000A86B812FC856DF4F0FB6F894DEBF0FBE41
:10857000CDBFDF91CF911F910F91FF90EF90DF90D2
:10858000CF90BF90AF909F9008950F931F93CF937C
:10859000DF93CDB7DEB7AD970FB6F894DEBF0FBE51
:1085A000CDBF8091410B882309F440C180915E16B4
:1085B00090915F16892B09F439C162ED7AE0CE0102
:1085C00088960E94386C8091D20B8823E1F061E894
:1085D00075E0CE0101960E94286CCE0101960E94A2
:1085E0003B7CCE0101960E94A86B68E572E0CE014B
:1085F00001960E94386CCE0101960E94DA83CE016A
:1086000001960E94A86B8091410B811105C0809159
:108610003E0B811109C051C080915E1690915F168A
:10862000892B09F006C1F3CF809152169091531611
:10863000892B09F442C065E675E0CE0188960E9458
:10864000396B6EE476E1CE0101960E94306CAE018A
:108650004F5F5F4F62E070E082E792E0F5DD182F38
:10866000CE0101960E94A86B111127C0BE01685D62
:108670007F4FCE014C960E94306C6CE376E1CE01C8
:108680004C960E94286BBC01CE0101960E94306C72
:10869000CE0101960E94DA83CE0101960E94A86B5A
:1086A000CE014C960E94A86B80913F0B9091400B9D
:1086B00001969093400B80933F0B80913D0B882354
:1086C00009F499C00FE110E080913C0B882359F028
:1086D0000150110909F49BC064E170E080E090E072
:1086E0000E944182F1CF43E165E672E0CE0101963E
:1086F0000E944E8FBE016F5F7F4F82EA98E10E9419
:10870000157B81E080933C0B82EA98E10E94AA7C71
:108710008823E1F16AE576E182EA98E10E94446DFE
:1087200082EA98E10E946B7C62E370E080E090E076
:108730000E94418210923C0B8091D20B882331F130
:10874000CE014C960E944A3767E379E0CE018296CB
:108750000E94386CBE01645E7F4FCE0182960E94FB
:10876000286BBC01CE0101960E94306CCE010196AF
:108770000E94DA83CE0101960E94A86BCE018296F8
:108780000E94A86BCE014C960E94A86B82EA98E1E9
:108790000E946B7C62E370E080E090E00E94418286
:1087A00010923C0B43E162E772E0CE0101960E9419
:1087B0004E8FBE016F5F7F4F82EA98E10E94157B6A
:1087C00081E080933C0B82EA98E10E94AA7C882396
:1087D00031F06EE476E182EA98E10E94446D82EA2B
:1087E00098E10E946B7C62E370E080E090E00E9480
:1087F000418210923C0B62ED7AE08EE496E10E9499
:108800007E6B62ED7AE08AE596E10E947E6BCE0196
:1088100088960E94A86BAD960FB6F894DEBF0FBE87
:10882000CDBFDF91CF911F910F9108950E94E9373D
:10883000C4CE64E170E080E090E00E94418263E792
:1088400075E0CE0188960E94396B6AE576E1CE012B
:1088500001960E94306CAE014F5F5F4F63E070E0A5
:1088600088E592E0F1DC182FCE0101960E94A86BFA
:10887000111127C0BE01685D7F4FCE014C960E944A
:10888000306C6CE376E1CE014C960E94286BBC0103
:10889000CE0101960E94306CCE0101960E94DA83CF
:1088A000CE0101960E94A86BCE014C960E94A86B47
:1088B00080913F0B9091400B01969093400B8093D9
:1088C0003F0B1092410B80913E0B8111A0CE9FCFA8
:1088D000DC015996ED91FC915A973097B9F0838954
:1088E0009489A589B6894285538564857585841BDD
:1088F000950BA60BB70B811520E89207A105B105D2
:1089000038F08FEF9FE7A0E0B0E0089580E090E0BE
:108910000895CF93DF931F92CDB7DEB76983DC0153
:10892000ED91FC910280F381E02D41E050E0BE0129
:108930006F5F7F4F19950F90DF91CF910895FC01E4
:1089400020812EBD9B012150310941F051810DB490
:1089500007FEFDCF4EB55EBD4193F5CF6150710965
:10896000FC01E60FF71F0DB407FEFDCF8EB5808327
:108970000895E0917A0EF0917B0E90818091790EAE
:1089800080958923808308958EBD00000DB407FE75
:10899000FDCF8EB5089520917C0E90E0233311F425
:1089A0000C9601C04896982F990F990F990F80E067
:1089B0000895CF93DF93CDB7DEB76D970FB6F894D8
:1089C000DEBF0FBECDBF442351F1AB01BC011C8201
:1089D0001B8283EB93E09A8389831E8222E0CE017F
:1089E00001960E94C85E811102C090E013C0CE01C2
:1089F00001960E94E47C8823C1F3CE0101960E9477
:108A0000527C009791F325EEFC0120831E820E9488
:108A10000E5D982F81E0911103C080E001C081E0DC
:108A20006D960FB6F894DEBF0FBECDBFDF91CF912C
:108A300008951F93CF93DF93CDB7DEB76D970FB631
:108A4000F894DEBF0FBECDBFAB011C821B8223EBAF
:108A500033E03A8329831E8221E0BC01CE010196D6
:108A60000E94C85E11E0811102C010E004C0CE0176
:108A700001960E94BD5E812F6D960FB6F894DEBF01
:108A80000FBECDBFDF91CF911F910895FC01818D65
:108A9000928D009711F00C94915E0895CF93DF931F
:108AA000EC01898D9A8D009739F481E090E09B83E9
:108AB0008A8380E090E00BC0FC01138212820E9446
:108AC0007060E98DFA8D22813381232B71F7DF915C
:108AD000CF910895FF920F931F93CF93DF931F922F
:108AE0001F92CDB7DEB7F82E22E030E0AE014F5F27
:108AF0005F4F66E270E00E94F45709811A811027E7
:108B00000127102722E030E0AE014F5F5F4F66E2A1
:108B100070E08F2D0E94F45789819A8198278927C8
:108B200098270817190711F08C01ECCFC8010F9096
:108B30000F90DF91CF911F910F91FF90089561E009
:108B4000FC0184810C9482818EBD0DB407FEFDCFA3
:108B500008958FEFF9DF8EB508958F929F92AF92AF
:108B6000BF92FF920F931F93CF93DF93EC01F62EEA
:108B700049015A018E81882319F0CE010E94BE5B03
:108B800060E08C810E9482816CE271E0CE010E94E3
:108B9000855C8F2D8064D8DF08E110E0D501C40129
:108BA000002E04C0B695A795979587950A94D2F79D
:108BB000CBDF08501109083F8FEF180779F7FF2026
:108BC00029F088E0F81204C087E803C085E901C0F5
:108BD0008FEFBADF10E0BDDF8A8787FF04C01F3F39
:108BE00011F01F5FF8CFDF91CF911F910F91FF9090
:108BF000BF90AF909F908F900895FC01DB0112967B
:108C00008D919C9113979383828383EB93E091835F
:108C1000808314968C911497848315968C91159764
:108C2000858316964D915D916D917C911997468340
:108C30005783608771871A964D915D916D917C91F4
:108C40001D9742875387648775871E964D915D9166
:108C50006D917C91519746875787608B718B5296A7
:108C60008C915297828B53964D915D916D917C9131
:108C70005697438B548B658B768B57964D915D91B0
:108C80006D917C915A97478B508F618F728F5B9655
:108C90008D919C915C97948F838F0895CF93DF93F0
:108CA000EC010E9450368FEB93E0998388831A8EF3
:108CB000198E1C86DF91CF910895CF93DF931F9279
:108CC000CDB7DEB741E050E0BE016F5F7F4F0E943D
:108CD0008E5D019719F4898190E002C08FEF9FEFBC
:108CE0000F90DF91CF910895FC01818D928D0097B7
:108CF00009F0E3CF8FEF9FEF08950F931F93CF936A
:108D0000DF93FC01818D928D0097B1F0EF01D5DFEB
:108D10008C010F3F8FEF180791F0898D9A8DFC0120
:108D200042855385648575854150510961097109F2
:108D30000E94275BC80105C080E090E002C08FEF71
:108D40009FEFDF91CF911F910F910895CF93C82F7F
:108D5000462F61E070E00E945D5661E070E08C2F6C
:108D60000E947B568111F9CFCF910895E0917A0E40
:108D7000F0917B0E90818091790E892B80830895EC
:108D8000AF92BF92CF92DF92EF92FF920F931F9319
:108D9000CF93DF9300D01F92CDB7DEB78C016B016C
:108DA0007A0180917C0E8333C1F45B016801C40EAB
:108DB000D51E0C151D0509F455C0DBDD8FE0E4DD83
:108DC000812FE2DD802FE0DD0F5F1F4F80E0DCDDD3
:108DD000F50181935F01CADFECCF8433D1F4C9DDA3
:108DE00019830A838F2D8F778B83EC8264E070E088
:108DF000CE010196A4DDA70160E070E0C6010E94EB
:108E00000CB6E114F10419F0B701C60198DDAEDF2C
:108E100029C0AFDD0F3F110509F020F419820A8344
:108E20001B821DC017FD0BC019820A8333E0169503
:108E300007953A95E1F7007E08600B8310C0C801E2
:108E400026E0969587952A95E1F719830A83807E17
:108E50000115104C10F4806101C088618B8363E0C0
:108E600070E0C6CFC7010F900F900F900F90DF9169
:108E7000CF911F910F91FF90EF90DF90CF90BF9017
:108E8000AF900895AF92BF92CF92DF92EF92FF9290
:108E90000F931F93CF93DF93CDB7DEB728970FB60D
:108EA000F894DEBF0FBECDBF8C017B016A018091BB
:108EB0007C0E8333B1F45801A40EB51E0A151B05B0
:108EC00009F47DC056DD80EF5FDD812F5DDD802FF1
:108ED0005BDD0F5F1F4FF70181917F0155DD46DF9D
:108EE000EDCF8433F9F445DD19830A838D2D806835
:108EF0008B83CC8264E070E0CE01019620DD870197
:108F00000C0D1D1DE016F10659F0F70181917F014E
:108F10003BDDF8CFB6016D5F7F4FCE0101960FDDCF
:108F200025DF4DC026DD0F3F110509F020F4198221
:108F30000A8384E01CC017FD0BC019820A8333E04A
:108F4000169507953A95E1F7007E0C600B8310C0EB
:108F5000C80126E0969587952A95E1F719830A833B
:108F6000807E0115104C10F4846101C08C618B83EC
:108F700026E0C216D10498F420E0822F90E08C15F0
:108F80009D0540F6E4E0F0E0EC0FFD1FE80FF91F4F
:108F9000D701A80FB91F8C9180832F5FEECF63E0BC
:108FA00070E0CE010196CBDC87010C0D1D1DF70191
:108FB00081917F01E9DCE016F106C9F7B1CFC60166
:108FC00028960FB6F894DEBF0FBECDBFDF91CF91CC
:108FD0001F910F91FF90EF90DF90CF90BF90AF90D7
:108FE0000895CF93DF931F92CDB7DEB741E050E0F5
:108FF000BE016F5F7F4F80E090E0C2DE89810F90FD
:10900000DF91CF910895CF93DF931F92CDB7DEB755
:10901000898341E050E0BE016F5F7F4F80E090E0C8
:1090200031DF0F90DF91CF910895CF93DF9380E8E8
:10903000EADFC4E1D0E0D5DF882351F061E070E0E1
:1090400080E090E00E9441822197A9F780E001C072
:1090500081E0DF91CF9108957F928F929F92AF929E
:10906000BF92CF92DF92EF92FF920F931F93CF9315
:10907000DF931F921F92CDB7DEB7782E8B014A0186
:10908000590122E030E0AE014F5F5F4F64E270E0D3
:109090000E94F457E980FA80FE24EF24FE24E00EBB
:1090A000F11E9701377040917C0E072D10E0C8012A
:1090B000433311F4089601C04096982F8827990FE2
:1090C000990F990F820F931F473319F4A501B4012B
:1090D0001FC0A9014A0D5B1D41305840B8F360E044
:1090E00078E06B01C21AD30AA601B401CBDEA50158
:1090F0004C195D09B4016C0D7D1D80917C0E83338C
:1091000031F5085F1F4F902F990F990F990F80E04D
:10911000B9DEEA0CFB1CF982EA8222E030E0AE0103
:109120004F5F5F4F64E270E0872D0E9455550F90AE
:109130000F90DF91CF911F910F91FF90EF90DF90F3
:10914000CF90BF90AF909F908F907F900895005FD9
:109150001F4FD9CFEF92FF921F93CF93DF931F92B0
:109160001F92CDB7DEB7182F22E030E0AE014F5F7F
:109170005F4F60E270E00E94F457E980FA80FE24BD
:10918000EF24FE2422E030E0AE014F5F5F4F60E24B
:1091900070E0812F0E94F45789819A81982789274E
:1091A0009827E816F90611F07C01ECCF87E0189FAC
:1091B000F0011124E058FE4EF582E482C7010F90C1
:1091C0000F90DF91CF911F91FF90EF900895FF9244
:1091D0000F931F93CF93DF931F921F92CDB7DEB7EC
:1091E000F82ECE0101960E94857889819A810E948D
:1091F00044908F2DAFDF8C018F2D0E949956F82E51
:109200000E94439087E1F81631F08CE1F81619F0CE
:1092100080E090E001C0C8010F900F90DF91CF91E6
:109220001F910F91FF900895AF92BF92CF92DF925E
:10923000EF92FF920F931F93CF93DF931F921F9292
:10924000CDB7DEB7F82E6B018A014130584010F0DF
:1092500000E018E0CE0101960E94857889819A810C
:109260000E9444908F2D76DF5C018F2D0E949956CD
:10927000E82E0E94439087E1E81619F08CE1E8128D
:1092800004C0A016B10630F302C000E010E0CE0129
:1092900001960E94857889819A810E944490980164
:1092A000A60160E070E08F2DD7DE60E270E08F2DC8
:1092B0004DDD62E070E08F2D0E947B5684FD15C06D
:1092C0008F2D0E949956811105C00E94439080E025
:1092D00090E014C00E944390CE0101960E948578D0
:1092E00089819A810E944490E4CF40E162E070E07D
:1092F0008F2D0E945D560E944390C8010F900F90E1
:10930000DF91CF911F910F91FF90EF90DF90CF9061
:10931000BF90AF9008951F93CF93DF931F921F923A
:10932000CDB7DEB7182FCE0101960E9485788981CE
:109330009A810E944490812F2EDB27E0129FF0013A
:109340001124E058FE4E22813381377041E050E015
:10935000BE016F5F7F4F820F931F12DD0E9443900B
:1093600089810F900F90DF91CF911F910895EF9217
:10937000FF920F931F93CF93DF931F921F92CDB74E
:10938000DEB7482F87E0489F90011124F901E0588B
:10939000FE4E7F01808191810097B1F4142FCE01A0
:1093A00001960E94857889819A810E944490812F3C
:1093B00091DB8C010E944390F70186819801281B64
:1093C0003109C901318320830F900F90DF91CF9134
:1093D0001F910F91FF90EF9008954F925F927F92AF
:1093E0008F929F92AF92BF92CF92DF92EF92FF92B5
:1093F0000F931F93CF93DF931F921F92CDB7DEB7CA
:10940000782E6B014A01A82EB12C27E0829FC00163
:109410001124AC0140585E4E7A01FA01008111819D
:10942000CE0101960E94857889819A810E9444909C
:10943000081519054CF4872D4DDBF70126818C01A9
:10944000021B1109118300830115110599F4872D61
:109450000E949956843109F47BC0882309F478C0AE
:1094600001E010E08C3111F400E010E0119501955D
:1094700011096EC0801691060CF4840187E08A9D64
:10948000F0018B9DF00D1124E058FE4EE280F38038
:10949000C114D10439F12701F7E05F22872D7BDA6F
:1094A000840D951D20917C0E273319F4A801B60177
:1094B00018C09801240D351D21303840B8F320E044
:1094C00038E0490184189508A401B60159DC260149
:1094D000480C591C6801C818D908872D5CDAA60108
:1094E000B2014EDCE00EF11E87E08A9DF0018B9DFB
:1094F000F00D1124E058FE4EF382E28280819181CA
:10950000801B910B918380832681A801420F511DFE
:109510004A3F510510F4892BD1F487E08A9DF00170
:109520008B9DF00D1124E058FE4E1682F982EA82DE
:1095300022E030E0AE014F5F5F4F68E270E0872DC0
:109540000E94555560E470E0872D00DC01C0468321
:109550000E944390C8010F900F90DF91CF911F910F
:109560000F91FF90EF90DF90CF90BF90AF909F90C2
:109570008F907F905F904F9008951F93CF93DF93CC
:109580001F921F92CDB7DEB7182FCE0101960E9411
:10959000857889819A810E94449068E070E0812FEB
:1095A000D5DB0E9443900F900F90DF91CF911F91D8
:1095B00008951F93CF93DF931F921F92CDB7DEB70D
:1095C000182FCE0101960E94857889819A810E9488
:1095D000449060E170E0812FB9DB0E9443900F90CE
:1095E0000F90DF91CF911F9108951F93CF93DF9339
:1095F0001F921F92CDB7DEB7182FCE0101960E94A1
:10960000857889819A810E944490812F0E94995681
:10961000182F0E944390812F0F900F90DF91CF91D0
:109620001F9108958F929F92BF92CF92DF92EF92F7
:10963000FF920F931F93CF93DF93CDB7DEB72A9797
:109640000FB6F894DEBF0FBECDBF90917C0E99236C
:1096500009F495C0933319F028E0B22E02C094E0CB
:10966000B92E6B01082FCE0101960E948578898161
:109670009A810E9444909E012F5F3F4F79014901DA
:1096800010E0812F0E949956F40181934F018823A5
:10969000C1F01F5FB112F5CF10E0F70191917F018A
:1096A0009D3159F0983149F09A51923030F01F5F56
:1096B000B112F3CF0E94439062C060E170E0812F4D
:1096C00045DBE12EF12CF701EE0FFF1FE854FE4EB3
:1096D0001182108283EE93E00197F1F7402F60E052
:1096E00070E0812F0E945D564FEF62E070E0812FA5
:1096F0000E945D56C114D10411F0B60113C08091CF
:10970000A1029091A20201968115F0EC9F0710F43E
:1097100080E090EC9093A2028093A1026091A1025C
:109720007091A202812F0E94675561E070E0812F45
:109730000DDB27E02E9DC0012F9D900D11249C0173
:1097400020583E4E7901F9011182108222E030E06A
:10975000AE01475F5F4F68E270E0812F0E94F457CF
:1097600089859A85982789279827F701938382838B
:109770001682158214820E944390812F01C088E0D6
:109780002A960FB6F894DEBF0FBECDBFDF91CF9102
:109790001F910F91FF90EF90DF90CF90BF909F901F
:1097A0008F900895CF93DF931F921F92CDB7DEB7AE
:1097B00079836A8322E030E0AE014F5F5F4F60E162
:1097C00070E00E9455550F900F90DF91CF91089552
:1097D0000E94D9B51F920F920FB60F9211242F93AA
:1097E0003F938F939F93AF93BF9380917811909104
:1097F0007911A0917A11B0917B113091420D23E043
:10980000230F2D3720F40196A11DB11D05C026E8B8
:10981000230F0296A11DB11D2093420D8093781154
:1098200090937911A0937A11B0937B1180917C1160
:1098300090917D11A0917E11B0917F110196A11D93
:10984000B11D80937C1190937D11A0937E11B093F4
:109850007F11BF91AF919F918F913F912F910F9069
:109860000FBE0F901F901895FC0180819181009789
:1098700011F00C9472AC60E070E0CB01089585EDBE
:109880008093BC008091BC0084FDFCCF109232110B
:10989000089540916F0D262F30E0240F311D2132A5
:1098A0003105DCF4209132112430C9F4FC0180E050
:1098B00090E0861758F430916F0D2191DC01A15B87
:1098C000B24FA30FB11D2C930196F3CF80916F0D72
:1098D000680F60936F0D80E0089581E0089582E045
:1098E0000895089508950895E091CD118091CC11C7
:1098F000E81730F4F0E0E451FF4E808190E00895E5
:109900008FEF9FEF08959091CD118091CC11981712
:1099100050F4E92FF0E0E451FF4E208130E09F5FEA
:109920009093CD1102C02FEF3FEFC90108958091B0
:10993000CC1190E02091CD11821B91090895CF9216
:10994000DF92EF92FF920F931F93CF93DF937C01EF
:10995000CB018A0120913311222389F0EB016B01A5
:10996000C40ED51ECC15DD0561F06991D701ED91CE
:10997000FC910190F081E02DC7011995F3CF642F80
:1099800088DFC801DF91CF911F910F91FF90EF9079
:10999000DF90CF900895CF93DF931F92CDB7DEB7BE
:1099A0006983209133112223D1F020915611203266
:1099B00040F021E030E0FC013383228380E090E03E
:1099C00014C080913411E82FF0E0EB5CFE4E9981D9
:1099D00090838F5F809334118093561104C061E0AF
:1099E000CE01019656DF81E090E00F90DF91CF919C
:1099F0000895CF92DF92EF92FF920F931F93CF9330
:109A0000DF936C018B017A01EC01CB58D14F888137
:109A100087FF04C0FB011182108224C02CE02C9D22
:109A2000C0012D9D900D11242881AC01420F511DC4
:109A300027FD5A952091471530E04217530794F4BB
:109A40002881AC01420F511D27FD5A959A01FA0158
:109A5000EE0FFF1F2E0F3F1FF901E954FB4E20812F
:109A600026FD19C088818F5F88832CE02C9DC00162
:109A70002D9D900D11242881AC01420F511D27FD11
:109A80005A952091471530E042175307BCF42881BE
:109A90002C3044F113C02881820F911D27FD9A9527
:109AA000FC01EE0FFF1F8E0F9F1FFC01E954FB4EC0
:109AB000808160E08F730E948281D4CFF801808121
:109AC0009181049680349C4918F480E49CE904C098
:109AD000F801808191810496F701918380838FEF53
:109AE000888345C0F801408151812881BC01620F03
:109AF000711D27FD7A959B01FB01EE0FFF1F2E0FB5
:109B00003F1FF901E954FB4E21813281240F351F9B
:109B1000F701318320832881AC01420F511D27FDBD
:109B20005A959A01FA01EE0FFF1F2E0F3F1FF90100
:109B3000E954FB4E208126FF1AC02881820F911D17
:109B400027FD9A95FC01EE0FFF1F8E0F9F1FFC0152
:109B5000E954FB4E808161E08F73DF91CF911F91BB
:109B60000F91FF90EF90DF90CF900C948281DF9166
:109B7000CF911F910F91FF90EF90DF90CF900895BC
:109B8000FC01848191E090933311809355111092E0
:109B90003411109256118385862B90E00E94E7784D
:109BA00081E00C948B780F931F93CF938C01C62F79
:109BB000E7DF6C2F6460C801E3DF6C2F6B7FC801A7
:109BC000DFDF83EC90E00197F1F7CF911F910F91C8
:109BD00008950F931F93CF938C01C62F607F616010
:109BE000E2DF80E1C89FB00111246160C801DBDFC2
:109BF00081E090E0CF911F910F9108956093710ED5
:109C00007093720E8093730E9093740EDC01CB01EF
:109C1000845D9E4FAF4FBF4F80936D0E90936E0E3D
:109C2000A0936F0EB093700E82E090E090936C0E54
:109C300080936B0E0E9479826093670E7093680E1A
:109C40008093690E90936A0E0895CF92DF92EF92FF
:109C5000FF920F931F930E9479820091670E1091DB
:109C6000680E2091690E30916A0E6B017C01C01A5A
:109C7000D10AE20AF30A6091710E7091720E80911E
:109C8000730E9091740E48EEC41643E0D406E104BE
:109C9000F104D0F0DC01CB010196A11DB11D809330
:109CA000710E9093720EA093730EB093740E0851C0
:109CB0001C4F2F4F3F4F0093670E1093680E209359
:109CC000690E30936A0EC7CF1F910F91FF90EF90EE
:109CD000DF90CF9008954F925F926F927F928F9214
:109CE0009F92AF92BF92CF92DF92EF92FF920F932B
:109CF0001F93CF93DF934B015C018091630E909192
:109D0000640EA091650EB091660E88159905AA059E
:109D1000BB0509F4D2C08CE3C82ED12CE12CF12C68
:109D2000C501B401A70196010E9433B26093480DAA
:109D3000CA01B901A70196010E9433B26093490D8F
:109D4000C501B40120E13EE040E050E00E9433B2A2
:109D5000CA01B90128E130E040E050E00E9433B28E
:109D600060934A0DC501B40120E831E541E050E0BF
:109D70000E9433B269017A01CA01B9016C5F7F4F59
:109D80008F4F9F4F27E030E040E050E00E9433B219
:109D90006F5F60934B0D412C512C320140E004E683
:109DA00010E0C0E9D1E0242F30E02E54384FF90103
:109DB000E370FF27309789F4C901B8010E94A2B36C
:109DC000892B31F4C901BE010E94A2B3892B29F469
:109DD0008EE691E0A0E0B0E004C08DE691E0A0E066
:109DE000B0E0480E591E6A1E7B1ED301C201AA278D
:109DF000BB27C816D906EA06FB0610F04F5FD3CF83
:109E000040934E0D309799F4C90164E670E00E94CA
:109E1000A2B3892B39F4C90160E971E00E94A2B3B1
:109E2000892B29F48EE691E0A0E0B0E004C08DE635
:109E300091E0A0E0B0E0481A590A6A0A7B0AC41807
:109E4000D508E608F708C90164E670E00E94A2B3ED
:109E5000EC01C90160E971E00E94A2B3A3E4B3E0A0
:109E600020E0213039F4309749F4209729F4009705
:109E700029F402C04C9103C04DE101C04CE150E017
:109E800060E070E0C416D506E606F70640F0C41A96
:109E9000D50AE60AF70A2F5F11962C3011F72F5FCB
:109EA00020934D0DC394C0924C0D8092630E9092FE
:109EB000640EA092650EB092660EDF91CF911F9155
:109EC0000F91FF90EF90DF90CF90BF90AF909F9059
:109ED0008F907F906F905F904F900895B6DEFBDE7D
:109EE00080914E0D90E08E54984F0895AEDEF3DED3
:109EF00080914D0D90E00895A8DEEDDE80914C0D2F
:109F000090E00895A2DEE7DE8091490D90E008958B
:109F10009CDEE1DE80914A0D90E008951F920F9241
:109F20000FB60F9211240BB60F922F933F934F93BE
:109F30005F936F937F938F939F93AF93BF93EF93B1
:109F4000FF938091930D0E945A812091960D30913C
:109F5000970D2F5F3F4F3093970D2093960D909163
:109F6000950D953618F096E09093920D9091920D84
:109F70009430C9F128F4923069F09330D1F05EC08A
:109F8000953009F451C0963009F058C091E0909393
:109F9000620E51C0811152C02091960D3091970DE3
:109FA0002436310508F442C01092620E1092950DCD
:109FB0001CC0813009F042C0E091950D91E09E0FE8
:109FC0009093950DF0E02091960D3091970DEE0F46
:109FD000FF1FE856F24F318320831092970D1092A5
:109FE000960D94E029C0811117C0E091950D91E084
:109FF0009E0F9093950DF0E02091960D3091970D66
:10A00000EE0FFF1FE856F24F318320831092970D19
:10A010001092960D93E010C02091960D3091970DFF
:10A020002536310558F007C0811108C01092970DF0
:10A030001092960D03C095E09093920D9091940D1F
:10A04000992329F0811102C02F9A01C02F98FF9106
:10A05000EF91BF91AF919F918F917F916F915F91A0
:10A060004F913F912F910F900BBE0F900FBE0F900D
:10A070001F9018951F920F920FB60F9211240BB6D6
:10A080000F922F933F934F935F936F937F938F9391
:10A090009F93AF93BF93EF93FF938091B900887F15
:10A0A000803609F49CC068F5883209F45BC090F4EE
:10A0B000803109F454C038F4882309F4F6C088309C
:10A0C00009F44DC0F5C0883109F44CC0803209F460
:10A0D0005DC0EEC0803409F468C048F4803309F4F0
:10A0E00055C0883309F0E4C080933011D8C0803562
:10A0F00009F44FC0883509F45DC0883409F0D8C030
:10A10000D6C0883909F4C7C0A8F4883709F467C0F5
:10A1100038F4883609F463C0803709F460C0C8C0D9
:10A12000883809F4B8C0803909F45FC0803809F074
:10A13000BFC05BC0803B09F486C038F4803A09F4A4
:10A1400066C0883A09F47FC0B3C0803C09F4A7C058
:10A15000883C09F4A4C0883B09F48AC0A9C0809156
:10A160000D1110C090912F1180912E11981770F53C
:10A17000E0912F1181E08E0F80932F11F0E0E25FCC
:10A18000FE4E80818093BB0085EC86C080933011A9
:10A190008EC0E0912F1181E08E0F80932F1180915E
:10A1A000BB00F0E0E25FFE4E808390912F11809122
:10A1B0002E116EC0E0912F1181E08E0F80932F1130
:10A1C0008091BB00F0E0E25FFE4E80838091311110
:10A1D00081116DC081E080930C1184EA61C083E03D
:10A1E000809332111092910DCFCF8091910D8032DA
:10A1F00008F051C0E091910D81E08E0F8093910D98
:10A200008091BB00F0E0EF58F24F8083BDCF85EC2A
:10A210008093BC00109232118091910D803230F405
:10A22000E091910DF0E0EF58F24F10826091910DA6
:10A2300070E0E091C811F091C91181E79DE0199596
:10A240001092910D35C084E0809332111092700D00
:10A2500010926F0DE091CA11F091CB111995809178
:10A260006F0D811105C081E080936F0D10924F0D2D
:10A27000E091700D81E08E0F8093700DF0E0E15B56
:10A28000F24F80818093BB009091700D80916F0D93
:10A29000981708F479CF85E88093BC0009C085EC55
:10A2A0008093BC001092321103C010923011E7DA93
:10A2B000FF91EF91BF91AF919F918F917F916F919E
:10A2C0005F914F913F912F910F900BBE0F900FBE5A
:10A2D0000F901F9018954F925F926F927F928F927E
:10A2E0009F92AF92BF92CF92DF92EF92FF920F9325
:10A2F0001F93CF93DF93EC01423051056105710547
:10A3000010F480E078C089859A85AB85BC8501967C
:10A31000A11DB11D84179507A607B70790F3CB8839
:10A32000DC88ED88FE888F89803129F4BB27A72F30
:10A33000962F852F09C0DB01CA01E7E0B695A795E6
:10A3400097958795EA95D1F7480159012A013B0174
:10A35000C80ED91EEA1EFB1E80919D0290919E029E
:10A36000A0919F02B091A002C816D906EA06FB068A
:10A3700081F48F898031A9F4B301A20155276627A2
:10A380007727440F551FFA01E851F14F91828082DF
:10A3900019C040E0C701B6010E94475D8111E9CFB5
:10A3A000B0CFB301A2014F77552766277727440F17
:10A3B000551F440F551FFA01E851F14F80829182D9
:10A3C000A282B3828091430D81608093430D8A897C
:10A3D000823080F08D819E81AF81B885C80ED91EF4
:10A3E000EA1EFB1EC092440DD092450DE092460D30
:10A3F000F092470D81E0DF91CF911F910F91FF9077
:10A40000EF90DF90CF90BF90AF909F908F907F9014
:10A410006F905F904F9008958F929F92AF92BF92EE
:10A42000CF92DF92EF92FF920F931F93CF93DF9320
:10A43000FC0181859285A385B4850196A11DB11D7E
:10A4400084179507A607B70710F480E05BC08388E0
:10A450009488A588B6888789803129F4BB27A72FDF
:10A46000962F852F09C0DB01CA01C7E0B695A795D5
:10A4700097958795CA95D1F7E9016A017B018F010C
:10A48000BC01CD01680D791D8A1D9B1D80909D0228
:10A4900090909E02A0909F02B090A002681579054E
:10A4A0008A059B0591F4F80187898031A1F4DD24A8
:10A4B000EE24FF24C601880F991FFC01E851F14FDB
:10A4C00080819181A0E0B0E018C040E00E94475D2B
:10A4D0008111E9CFBACFE894C7F8DD24EE24FF2438
:10A4E000C601880F991F880F991FFC01E851F14F91
:10A4F00080819181A281B381BF7088839983AA836F
:10A50000BB8381E0DF91CF911F910F91FF90EF907E
:10A51000DF90CF90BF90AF909F908F900895CF9392
:10A52000DF931F92CDB7DEB76983DC01ED91FC911B
:10A530000280F381E02D41E050E0BE016F5F7F4F6C
:10A5400019950F90DF91CF910895FC01818D928D27
:10A550000895CF93DF931F92CDB7DEB76983DC01F7
:10A56000ED91FC910280F381E02D41E050E0BE01CD
:10A570006F5F7F4F19950F90DF91CF910895FC0188
:10A580009485FB018485981303C081E0983008F01E
:10A5900080E00895CF93DF931F92CDB7DEB7698334
:10A5A000DC01ED91FC910280F381E02D41E050E06F
:10A5B000BE016F5F7F4F19950F90DF91CF91089586
:10A5C000CF92DF92EF92FF920F931F93CF93DF937F
:10A5D00000D000D0CDB7DEB78C016B017A01FC0151
:10A5E000808D883010F40E94D94A83E594E09A83E4
:10A5F0008983F60182819381A481B5818B839C83B9
:10A60000AD83BE83B701CE0101960E945780F80149
:10A61000808F883030F4F586E486128E118E81E0CA
:10A6200001C080E026960FB6F894DEBF0FBECDBF06
:10A63000DF91CF911F910F91FF90EF90DF90CF901E
:10A640000895CF93DF93FC01808D883028F4EF01CB
:10A650000E94D94A88E0888FDF91CF910895FC014C
:10A66000808D883040F4218D328D232B21F00E9483
:10A670008B4990E008958FEF9FEF0895CF93DF937C
:10A68000FC012485283018F08FEF9FEF0EC0EC01FD
:10A690000190F081E02D0084F185E02D1995892B42
:10A6A00099F38C850E948B4990E0DF91CF910895BA
:10A6B000CF93DF93FC01218D328D2115310519F4E3
:10A6C0008FEF9FEF11C0EC014217530708F0A9016B
:10A6D000888D0E94ED491816190694F7298D3A8D38
:10A6E000281B390B3A8F298FDF91CF9108950F9353
:10A6F0001F93CF93DF931F92CDB7DEB7FC01218D5F
:10A70000328D232B61F08C0141E050E0BE016F5F80
:10A710007F4F808D0E94ED49181619061CF08FEFAF
:10A720009FEF08C0F801818D928D0197928F818FE4
:10A73000898190E00F90DF91CF911F910F91089543
:10A74000CF93DF931F92CDB7DEB741E050E0BE015B
:10A750006F5F7F4FFC0184850E94ED491816190632
:10A760001CF4898190E002C08FEF9FEF0F90DF9182
:10A77000CF910895FC018485883010F40C94ED4944
:10A7800080E090E00895FC018485883010F40C94FA
:10A79000B74980E090E008950F931F93CF93DF9324
:10A7A000CDB7DEB728970FB6F894DEBF0FBECDBF8A
:10A7B0008C01D80159964D915C915A9741155105DC
:10A7C00051F0ED91FC91048CF58DE02D60E070E08E
:10A7D000C8011995EECFF801808D0E94B749892BE9
:10A7E00051F148E050E0BE016F5F7F4FD8015896AD
:10A7F0008C910E94ED4918161906FCF4D801509668
:10A8000084E0FE01319601900D928A95E1F78D81E9
:10A8100090E0982F88272E81820F911DF801958B4B
:10A82000848B8F8190E0982F88272885820F911D37
:10A83000928F818F02C080E090E028960FB6F89446
:10A84000DEBF0FBECDBFDF91CF911F910F91089555
:10A850007F928F929F92AF92BF92CF92DF92EF92B0
:10A86000FF920F931F93CF93DF931F921F92CDB749
:10A87000DEB77C014B01742EC52EFC01A688B7887B
:10A88000D08CCE0101960E94857889819A810E94A0
:10A8900044908D2D0E94AA48072D1C2D80179107EA
:10A8A00008F48C019801A401B5018D2D0E942C485B
:10A8B0000E944390F70186899789800F911F978B9B
:10A8C000868BC8010F900F90DF91CF911F910F9150
:10A8D000FF90EF90DF90CF90BF90AF909F908F90C0
:10A8E0007F9008950F931F93CF93DF93EC018B011B
:10A8F000888D883010F40E94D94AB80182E00E9405
:10A90000124B888F883030F41D870C871A8E198E71
:10A9100081E001C080E0DF91CF911F910F910895F8
:10A920000F931F93CF93DF93FC018485883068F4E5
:10A93000C52FD42F8F010E941449009749F421E0BC
:10A9400030E0F8013383228305C080E090E002C04C
:10A950008D2F9C2FDF91CF911F910F910895EF9232
:10A96000FF920F931F93CF93DF937C0180917C0E16
:10A97000833311F4D4E001C0D8E008EB11E1C0E06A
:10A98000F801219131918F01F70184819581281778
:10A99000390729F0CF5FDC13F3CF80E006C08C2F9E
:10A9A0000E94F54A8431B1F781E0DF91CF911F9188
:10A9B0000F91FF90EF900895CF93DF93EC018C857A
:10A9C0008830C8F40E94F54A843181F0882371F000
:10A9D000883161F08C3161F4E881F9810084F1857E
:10A9E000E02DCE01199521E0892B19F420E001C05A
:10A9F00021E0822F01C080E0DF91CF910895CF92B6
:10AA0000DF92EF92FF92CF93DF93EC018C85883039
:10AA100038F50E94BD4A0E9479826B017C018C85C9
:10AA20000E94F54A8823D1F061E070E080E090E078
:10AA30000E9441820E947982AB01BC014C195D09E0
:10AA40006E097F098D859E85A0E0B0E04817590703
:10AA50006A077B0720F38C850E94D94A88E08C879F
:10AA6000DF91CF91FF90EF90DF90CF900895CF933B
:10AA7000DF93EC018C85883060F40E94F54A8731C1
:10AA800011F08C3131F48C850E94E7488115984093
:10AA900088F3DF91CF910895FC018485883010F40C
:10AAA0000C94E74880E090E00895DA0190917D0EE3
:10AAB000E92FF0E0FE2FEE27E60FF71F90E0982F2A
:10AAC0008827A901BD018E0F9F1F0C944247CF9389
:10AAD000DF931F921F92CDB7DEB779836A8322E09E
:10AAE00030E0AE014F5F5F4F64E070E0DEDF0F905B
:10AAF0000F90DF91CF910895DF92EF92FF920F9325
:10AB00001F93CF93DF931F921F92CDB7DEB7FB0148
:10AB1000DC0157961C921E9256972281211109C082
:10AB20002381211106C02481211103C02581222304
:10AB300001F141155105E9F07A018F01FC01D08C3A
:10AB4000CE0101960E94857889819A810E94449065
:10AB5000A8014E5F5F4F24E030E06CE070E08D2D87
:10AB6000A4DFB7018D2D0E94D24B0E94439081E05B
:10AB700001C080E090E00F900F90DF91CF911F9186
:10AB80000F91FF90EF90DF900895AF92BF92CF9218
:10AB9000DF92EF92FF920F931F93CF93DF931F9259
:10ABA0001F92CDB7DEB78C016B015A01FC01848581
:10ABB000883058F40E94F54A882321F0F8018485F2
:10ABC0000E94BD4A88E0F8018487F6018281938162
:10ABD000A481B5810097A105B10509F45CC08F3F40
:10ABE0009F4FAF4FBF4F09F456C060E070E081E265
:10ABF0000E94124BF82EF8018487F7E0F81708F44A
:10AC00004AC0CE0101960E94857889819A810E946E
:10AC10004490A6014E5F5F4F24E030E06CE070E0AE
:10AC20008F2D43DFB5018F2D0E94D24B64E070E081
:10AC30008F2D0E94A6460E9443900E9479826B014C
:10AC40007C01F80184850E94F54A873139F18C3105
:10AC500029F1882301F10E947982AB01BC014C19D2
:10AC60005D096E097F09F80185859685A0E0B0E051
:10AC700084179507A607B70738F061E070E080E019
:10AC800090E00E944182DDCFF80184850E94D94A7C
:10AC900088E0F801848780E090E002C081E090E0E5
:10ACA0000F900F90DF91CF911F910F91FF90EF9038
:10ACB000DF90CF90BF90AF900895CF93DF931F9216
:10ACC000CDB7DEB790917D0E292F30E0322F2227AD
:10ACD000260F371F90E0982F8827498341E050E0E6
:10ACE000BE016F5F7F4F820F931F0E9442470F90FC
:10ACF000DF91CF910895CF93DF931F92CDB7DEB749
:10AD000090917D0E292F30E0322F2227260F371FFA
:10AD100090E0982F882741E050E0BE016F5F7F4FA1
:10AD2000820F931F0E94C04689810F90DF91CF91BF
:10AD3000089563E070E0DFCFEF92FF921F93CF930F
:10AD4000DF931F921F92CDB7DEB77C01FC016481B7
:10AD5000758181E20E94124B182F883020F5CE01B8
:10AD600001960E94857889819A810E944490812F62
:10AD7000E0DF833131F00E944390812F0E94BD4A71
:10AD800012C062E070E0812F0E94A6460E944390AC
:10AD9000F70184819581E12FF0E0EE0FFF1FE85469
:10ADA000FE4E918380830F900F90DF91CF911F9182
:10ADB000FF90EF9008951F93CF93DF931F921F9200
:10ADC000CDB7DEB7FC01108DCE0101960E948578CB
:10ADD00089819A810E94449060E270E0812F0E94F4
:10ADE000A64662E070E0812F86DF84FD1AC062E033
:10ADF00070E0812F80DF83FF09C048E162E070E0EE
:10AE0000812F5BDF0E94439080E013C00E9443903B
:10AE1000CE0101960E94857889819A810E94449092
:10AE2000E0CF40E162E070E0812F47DF0E94439075
:10AE300081E090E00F900F90DF91CF911F910895E6
:10AE40009F92AF92BF92CF92DF92EF92FF920F93B9
:10AE50001F93CF93DF93EC016B0180917C0E8111E6
:10AE60000AC0CE010E9450368DE094E09983888319
:10AE700088E08C874FC0833319F434E0932E02C0EE
:10AE800028E0922E88EBE82E81E1F82E10E098E081
:10AE9000B92EA12CD7012D913C91F6018481958189
:10AEA00028173907F9F4812F0E94F54A082F8731B6
:10AEB00011F08C3159F4812F0E94B749892B71F41C
:10AEC0000C3181F4812F0E94BD4A0CC0843141F0C5
:10AED000811108C0D7011D921C9204C0B12E02C07E
:10AEE000AA24A3941F5FB2E0EB0EF11C9112D2CF03
:10AEF000A11008C0D601ED91FC910084F185E02DF0
:10AF0000C6011995CE010E9450368DE094E09983D8
:10AF10008883BC8688EE93E09E878D87CE01DF9183
:10AF2000CF911F910F91FF90EF90DF90CF90BF9046
:10AF3000AF909F9008958F929F92AF92BF92CF92C1
:10AF4000DF92EF92FF920F931F93CF93DF93CDB7D2
:10AF5000DEB72F970FB6F894DEBF0FBECDBF20919E
:10AF60007C0E222361F1233319F434E0E32E02C076
:10AF700028E0E22E8A015B016C01BC01CE01019642
:10AF80005FDF88EB882E81E1982EF12CF40121916E
:10AF900031914F01F601848195812817390751F4C9
:10AFA0008F2D0E94F54A873129F4A801B5018F2D14
:10AFB0000E941449F394EF10E9CFC80102C080E069
:10AFC00090E02F960FB6F894DEBF0FBECDBFDF9195
:10AFD000CF911F910F91FF90EF90DF90CF90BF9096
:10AFE000AF909F908F900895DA0190917D0EE92F98
:10AFF000F0E0FE2FEE27E60FF71F90E0982F88274E
:10B00000A901BD018E0F9F1F0C94C0460F931F9383
:10B01000CF93DF931F921F92CDB7DEB7FC0124853B
:10B020002830D8F48C01CE0101960E948578898160
:10B030009A810E94449022E030E0AE014F5F5F4F62
:10B0400060E170E0F8018485CFDF09811A81102763
:10B05000012710270E94439002C000E010E0C801C1
:10B060000F900F90DF91CF911F910F9108950F9343
:10B070001F93CF93DF931F921F92CDB7DEB7FC01D2
:10B0800024852830D8F48C01CE0101960E94857861
:10B0900089819A810E94449022E030E0AE014F5FA6
:10B0A0005F4F64E070E0F80184859EDF09811A81BA
:10B0B0001027012710270E94439002C000E010E0F3
:10B0C000C8010F900F90DF91CF911F910F910895BC
:10B0D0000F931F93CF93DF931F921F92CDB7DEB7CD
:10B0E0008C0183E594E0F8019183808312821382BE
:10B0F00014821582CE0101960E94857889819A81F9
:10B100000E944490B8016E5F7F4F44E050E08FE0B2
:10B1100090E00E94C0460E944390C8010F900F909B
:10B12000DF91CF911F910F910895AF92BF92CF926F
:10B13000DF92EF92FF920F931F93CF93DF93CDB7E0
:10B14000DEB7AF970FB6F894DEBF0FBECDBF8C0150
:10B150006B017A0183E5A82E84E0B82EBA82A98219
:10B160001B821C821D821E82CE0109960E946036BF
:10B17000BBA6AAA61CA61DA61EA61FA6D8011C9685
:10B180008C91883060F40E94F54A882321F0F80100
:10B1900084850E94BD4A88E0D8011C968C938091DA
:10B1A000AD149091AE14A091AF14B091B0148EA3D1
:10B1B0009FA3A8A7B9A78B839C83AD83BE83188662
:10B1C0001F82AE01465D5F4FB601CE0101960E941F
:10B1D000D03B0097C1F0D801ED91FC910684F78532
:10B1E000E02D83E594E09DA38CA38CA59DA5AEA541
:10B1F000BFA58EA39FA3A8A7B9A7A701BE016C5D99
:10B200007F4FC8011995AF960FB6F894DEBF0FBEF9
:10B21000CDBFDF91CF911F910F91FF90EF90DF9005
:10B22000CF90BF90AF900895AF92BF92CF92DF9230
:10B23000EF92FF920F931F93CF93DF93CDB7DEB7BB
:10B24000AF970FB6F894DEBF0FBECDBF7C015B0198
:10B250006A0103E514E01A8309831B821C821D82A4
:10B260001E82CE0109960E9460361BA70AA71CA663
:10B270001DA61EA61FA68091AD149091AE14A0919C
:10B28000AF14B091B0148EA39FA3A8A7B9A78B83C6
:10B290009C83AD83BE8318861F82AE01465D5F4FDF
:10B2A000B501CE0101960E94D03B81309105B1F4E9
:10B2B000D701ED91FC910488F589E02D1DA30CA325
:10B2C0008CA59DA5AEA5BFA58EA39FA3A8A7B9A732
:10B2D000A601BE016C5D7F4FC7011995AF960FB6F1
:10B2E000F894DEBF0FBECDBFDF91CF911F910F91BC
:10B2F000FF90EF90DF90CF90BF90AF900895EF92C6
:10B30000FF920F931F93CF93DF9300D01F92CDB77F
:10B31000DEB78C017B01FB018485883050F083E52A
:10B3200094E0F80191838083128213821482158243
:10B330001AC0CE0101960E94857889819A810E9467
:10B34000449024E030E0AE014F5F5F4F6CE070E06E
:10B35000F701848549DE0E944390BE016F5F7F4FF5
:10B36000C8010E947B6DC8010F900F900F900F9045
:10B37000DF91CF911F910F91FF90EF9008951F9350
:10B38000CF93DF93EC0180E2689FF0011124E85134
:10B39000F14F9385917129F0842F827411F080E030
:10B3A0004FC0142F6A8B80919D0290919E02A091B4
:10B3B0009F02B091A0028E879F87A88BB98B44898A
:10B3C000558960E070E0BA0155274427828D938D3E
:10B3D000A0E0B0E0482B592B6A2B7B2B4F8B588F6A
:10B3E000698F7A8F8385887151F4848D958DA68DB0
:10B3F000B78D8B8B9C8BAD8BBE8B81E00CC080316D
:10B4000071F69E012D5E3F4F8B8D9C8D0E94717D4C
:10B41000882329F284E08D83812F8F708C831E8294
:10B420001F82188619861A861B861C861D8616FFA3
:10B4300006C0CE01DF91CF911F910C94E47C81E096
:10B44000DF91CF911F9108953F924F925F926F923B
:10B450007F928F929F92AF92BF92CF92DF92EF92A4
:10B46000FF920F931F93CF93DF93CDB7DEB72C9747
:10B470000FB6F894DEBF0FBECDBF5C01DC015B965A
:10B480008D909C905C971696CD90DD90ED90FC9001
:10B490001997C114D104E104F10439F0BFEFCB1ABC
:10B4A000DB0AEB0AFB0A312C07C0F401C080D18013
:10B4B000E280F38033243394F40181859285A3855F
:10B4C000B4859C01AD012F5F3F4F4F4F5F4F2987E0
:10B4D0003A874B875C87260137011D821E821F82B7
:10B4E0001886F40181859285A385B4852D813E81DE
:10B4F0004F815885281739074A075B0708F063C052
:10B5000089859A85AB85BC858C159D05AE05BF05E3
:10B5100050F482E0C82ED12CE12CF12C92E0492E7F
:10B52000512C612C712C9E012F5F3F4FB701A6015A
:10B53000C4010E940C52882309F445C089819A8174
:10B54000AB81BC81892B8A2B8B2B41F026013701E3
:10B550009FEF491A590A690A790A05C0C414D5042B
:10B56000E604F70491F02D813E814F8158852F5FCD
:10B570003F4F4F4F5F4F2D833E834F8358873FEFA1
:10B58000C31AD30AE30AF30AACCF0FEF1FEF2FEF72
:10B590003FE0B301A201C4010E946B51882399F0DE
:10B5A000D50116964D915D916D917C91199741153C
:10B5B00051056105710549F093018201C4010E94A2
:10B5C0006B51811102C080E02AC0D50116964D92C0
:10B5D0005D926D927C921997332051F0D301C20194
:10B5E0000196A11DB11DF40180839183A283B383D1
:10B5F000F5018789908DA18DB28D892B8A2B8B2B9C
:10B6000069F4D50157964D925D926D927C925A974E
:10B6100014968C911497806814968C9381E02C96E4
:10B620000FB6F894DEBF0FBECDBFDF91CF911F9153
:10B630000F91FF90EF90DF90CF90BF90AF909F90D1
:10B640008F907F906F905F904F903F9008958F9272
:10B650009F92AF92BF92CF92DF92EF92FF920F93A1
:10B660001F93CF93DF93EC018D81811102C080E0A5
:10B6700078C00B891C892D893E8904171507260778
:10B680003707A8F36A017B01823029F4CA86DB867A
:10B69000EC86FD860DC0C114D104E104F10451F41F
:10B6A0001E821F82188619861A861B861C861D8696
:10B6B00081E057C08A849B84AC84BD84EB8DFC8D73
:10B6C000258530E0275F3F4FB501A4014150510966
:10B6D00061097109022E04C07695679557954795C3
:10B6E0000A94D2F7D701C6010197A109B10904C094
:10B6F000B695A795979587952A95D2F784179507BC
:10B70000A607B70720F089288A288B2871F44F896B
:10B71000588D698D7A8D4E835F83688779874C0158
:10B720005D018E010A5F1F4F16C0841B950BA60B8F
:10B73000B70BF5CF4E815F816885798598018B8D38
:10B740009C8D0E940C5291E0891A9108A108B108C1
:10B75000882309F48CCF81149104A104B10451F71A
:10B7600095CFDF91CF911F910F91FF90EF90DF90D8
:10B77000CF90BF90AF909F908F900895CF93DF931D
:10B78000EC018FEF8EBD2FEF8F819885AC014F5F5D
:10B790005F4F58874F838130924028F40DB407FEE5
:10B7A000FDCF2EBDF1CF0DB407FEFDCFCE010E941F
:10B7B0009F451E82DF91CF910895AF92BF92CF92A5
:10B7C000DF92EF92FF920F931F93CF93DF93EC01E1
:10B7D0006901C801820F931F8130924008F084C034
:10B7E0008E81882371F088819981AA81BB81841719
:10B7F0009507A607B70729F48F819885C816D9063B
:10B80000B0F5488359836A837B838B85833039F015
:10B8100089E0440F551F661F771F8A95D1F79A015B
:10B82000AB0161E1CE010E94AD45882319F083E0B0
:10B830008D835AC00E9479825B010E94A9458A8744
:10B840008F3F49F40E9479826A197B096D327140F9
:10B85000A0F38FE003C08E3F31F08DE08D83CE01E9
:10B860000E949F4541C018861F8281E08E838FEF22
:10B870008EBD2FEF8F8198858C159D0550F40DB4EA
:10B8800007FEFDCF2EBD8F819885019698878F8307
:10B89000F1CFC8010197F7012FEFAF014E195F09F2
:10B8A0004817590738F40DB407FEFDCF3EB5319364
:10B8B0002EBDF3CF0DB407FEFDCF2EB5F701E80F77
:10B8C000F91F20838F819885080F191F18870F8310
:10B8D0008985882319F00115124058F08E8188233C
:10B8E00041F0CE014BDF05C0CE010E949F4580E0B4
:10B8F00001C081E0DF91CF911F910F91FF90EF90F8
:10B90000DF90CF90BF90AF9008950F931F93CF9388
:10B91000DF93EB010E9479828B010E94A9458F3F42
:10B9200049F00E947982601B710B6C177D07A8F3A8
:10B9300080E001C081E0DF91CF911F910F910895C8
:10B940000F931F93CF93DF93EC01890141155105AC
:10B950006105710511F482E143C08B85833039F0B4
:10B9600089E0440F551F661F771F8A95D1F79A010A
:10B97000AB0168E1CE010E94AD45882311F084E05F
:10B980002FC08EEF8EBDF801C8019E5F0DB407FE7B
:10B99000FDCF20812EBD0DB407FEFDCF21812EBD30
:10B9A00032968E179F0791F70DB407FEFDCF8FEFEC
:10B9B0000E94A4458FEF0E94A4450E94A9458A8752
:10B9C0008F71853031F081E18D83CE010E949F45DA
:10B9D00008C068E572E0CE0198DF811107C085E1FB
:10B9E0008D83CE010E949F4580E013C020E030E0AF
:10B9F000A9016DE0CE010E94AD45811104C00E94F5
:10BA0000A945882311F084E1EBCFCE010E949F4528
:10BA100081E0DF91CF911F910F9108958091430DA7
:10BA2000882399F140919D0250919E0260919F025E
:10BA30007091A00228EE3EE08091CE119091CF113E
:10BA40007FDF811102C080E008954091440D509144
:10BA5000450D6091460D7091470D411551056105E9
:10BA6000710589F028EE3EE08091CE119091CF11C2
:10BA700067DF882341F31092440D1092450D109218
:10BA8000460D1092470D1092430D81E008958F925C
:10BA90009F92AF92BF92EF92FF920F931F93CF931B
:10BAA0004B015C01C42F80919D0290919E02A09158
:10BAB0009F02B091A00288159905AA05BB05F1F077
:10BAC000ADDF811102C080E01FC088EEE82E8EE05D
:10BAD000F82E00E012E020E030E0B501A4018091F2
:10BAE000CE119091CF1169DE882369F380929D0277
:10BAF00090929E02A0929F02B092A0028091430D6C
:10BB0000C82BC093430D81E0CF911F910F91FF90FF
:10BB1000EF90BF90AF909F908F9008952F923F929B
:10BB20004F925F926F927F928F929F92AF92BF924D
:10BB3000CF92DF92EF92FF920F931F93CF93DF93F9
:10BB4000EC016B014A018D81811103C08FEF9FEFE2
:10BB5000D5C08C8180FFFACF4B885C886D887E8849
:10BB60004A855B856C857D85C401A0E0B0E09301CA
:10BB70008201041B150B260B370B081719072A0720
:10BB80003B0718F44201841A950A54011E0126E06D
:10BB9000220E311CA114B10409F47EC04A855B85D4
:10BBA0006C857D852A0181E05822ED818B8D9C8DED
:10BBB0008A019B01F9E03695279517950795FA9527
:10BBC000D1F7E23061F4FC01828D938DA48DB58DA7
:10BBD000BC01CD01600F711F821F931F3FC0FC018C
:10BBE00074807A94702241145104C9F4711017C002
:10BBF000452B462B472B49F48F89988DA98DBA8DFB
:10BC00008E839F83A887B9870AC04E815F8168852C
:10BC1000798591010E940C52882309F497CFEB8D0E
:10BC2000FC8D8E819F81A885B9850297A109B109F4
:10BC3000058404C0880F991FAA1FBB1F0A94D2F75E
:10BC40004685578560897189840F951FA61FB71F88
:10BC5000BC01CD01670D711D811D911D20E032E0F9
:10BC60002419350935012A153B0508F439012C81C1
:10BC700026FD04C06114F2E07F0681F400919D026C
:10BC800010919E0220919F023091A00260177107CF
:10BC900082079307A9F402C0C40130C040E0F7DE78
:10BCA000882309F453CFF201E851F14FD601CF01B7
:10BCB000860D971D8E179F0781F021912D93FACF46
:10BCC000760183019201AB01BC018091CE1190916C
:10BCD000CF1173DD882309F439CFC60CD71C8A85B0
:10BCE0009B85AC85BD85860D971DA11DB11D8A87DD
:10BCF0009B87AC87BD87A618B7084CCFDF91CF9143
:10BD00001F910F91FF90EF90DF90CF90BF90AF9079
:10BD10009F908F907F906F905F904F903F902F906B
:10BD20000895CF93DF93EC018D81882311F18C81ED
:10BD300087FF1CC0CE010E94527CFC01892BC9F0F8
:10BD40008D81823040F48B899C89AD89BE89848F36
:10BD5000958FA68FB78F8F89988DA98DBA8D938F68
:10BD6000828FB58BA48B8C818F778C83DF91CF9161
:10BD700055CE80E0DF91CF910895CF93DF93EC0112
:10BD8000D0DF882311F01D8281E0DF91CF910895EB
:10BD90002F923F924F925F926F927F928F929F92DB
:10BDA000AF92BF92CF92DF92EF92FF920F931F93C9
:10BDB000CF93DF93CDB7DEB72C970FB6F894DEBFE5
:10BDC0000FBECDBF7C01DC0115962C90211069C1FE
:10BDD000FE013196CE010C966F0130E231938E1741
:10BDE0009F07E1F7DA0130E087E09D91992331F177
:10BDF0009E3231F48A3009F459C138E08AE0F5CF37
:10BE0000EBE2F8E04491442321F031969413FACF09
:10BE10004DC1831708F44AC14FED490F4E3508F064
:10BE200045C141E0430FF601E30FF11D3FE9390F32
:10BE30003A3108F490529083342FD7CF89818032E1
:10BE400009F434C12C878B01FB01838D948DD701BC
:10BE50005C969C938E935B97168217821086118650
:10BE60001286138614861586B12CF8018285938577
:10BE7000A485B58543895489658976898417950792
:10BE8000A607B70708F05BC025E0B695A79597957C
:10BE900087952A95D1F7F82FFF70AF2ED801159608
:10BEA0008C91823008F402C1C8010E945D4697FD62
:10BEB000FDC0F80182859385A485B5854F96A11DA7
:10BEC000B11D82879387A487B587F0E2AF9EB0014A
:10BED00011246851714F6115710509F4E7C0DB0148
:10BEE0008C91882319F0853EC1F4DDC0B1100EC0DD
:10BEF000F701A28A80919D0290919E02A0919F02DB
:10BF0000B091A00286879787A08BB18BDB018C91C3
:10BF1000882399F0BB24B394A8CF4BE050E0C6012E
:10BF20000E94E5B5892B09F0A0CF8C858073803302
:10BF300009F4BCC04C856A2DB0C0BB24B3948C8579
:10BF40008271823109F0B2C0BB2039F0C7010E9472
:10BF5000527C009709F076C0A9C0F8018581823033
:10BF600009F4A4C0C80170DA882309F49FC0D8017D
:10BF70005B96ED91FC915C9716968D909D90AD909F
:10BF8000BC901997B2E08B1A9108A108B1080584FA
:10BF900004C0880C991CAA1CBB1C0A94D2F7868585
:10BFA0009785A089B189880E991EAA1EBB1E348070
:10BFB000E1E08E1A9108A108B108332001F12401B3
:10BFC0003501430C511C611C711C28DD882309F4C8
:10BFD0006DC0E8EEFEE0119220E1E83EF207D9F7ED
:10BFE00040929D0250929E0260929F027092A00227
:10BFF0008091430D81608093430D3A94DECFD80148
:10C000005B96ED91FC915C9780E092E0A0E0B0E05F
:10C01000058404C0880F991FAA1FBB1F0A94D2F77A
:10C02000F8014389548965897689840F951FA61F75
:10C03000B71F838B948BA58BB68BD70152961C921E
:10C0400088EE9EE020E2FC0111922A95E9F72BE0B0
:10C05000F601DC0101900D922A95E1F721E238E228
:10C06000DC0151963C932E93509740E058E01F9688
:10C070005C934E931E9753963C932E9352975996EA
:10C080003C932E93589757965C934E935697C6DCE5
:10C09000882361F04C85F7016289C70170D9282E89
:10C0A00005C0212C03C0B11035CF22CF822D2C9694
:10C0B0000FB6F894DEBF0FBECDBFDF91CF911F91B9
:10C0C0000F91FF90EF90DF90CF90BF90AF909F9037
:10C0D0008F907F906F905F904F903F902F9008953A
:10C0E0002F923F924F925F926F927F928F929F9288
:10C0F000AF92BF92CF92DF92EF92FF920F931F9376
:10C10000CF93DF9300D01F92CDB7DEB78C015B01D8
:10C110001A01DC0115968C9115978130C1F41496A3
:10C120008C9181FF14C082FF1CC0F801438954899F
:10C130006589768982859385A485B5858417950759
:10C14000A607B70771F0C80182DA81110AC081E041
:10C1500090E0D80113969C938E93129780E090E024
:10C1600031C1610182C05B968D919C915C97FC010D
:10C1700074802FEF270D2A013B0139E076946794F4
:10C18000579447943A95D1F7722E74207A01F1E0D2
:10C19000FF22772009F475C080E092E08E199F0994
:10C1A00046018C159D0508F44C01D8015B962D9134
:10C1B0003C915C9716968D919D910D90BC91A02D10
:10C1C0000297A109B109F901058404C0880F991FDC
:10C1D000AA1FBB1F0A94D2F74685578560897189CB
:10C1E000840F951FA61FB71F9C01AD01270D311DA0
:10C1F000411D511D29013A01811432E0930609F0D5
:10C2000086C080919D0290919E02A0919F02B09164
:10C21000A002481659066A067B0659F48FEF9FEF75
:10C22000DC0180939D0290939E02A0939F02B093A5
:10C23000A0029501B301A2018091CE119091CF117E
:10C240007FDB882309F483CF9EEFB91AC818D90879
:10C25000F80182859385A485B585880D991DA11D5A
:10C26000B11D82879387A487B587D8011A964D910F
:10C270005D916D917C911D97C114D10409F073CF2C
:10C2800084C0E114F10409F087CF16964D915D91B9
:10C290006D917C911997411551056105710559F40E
:10C2A00057968D919D910D90BC91A02D0097A10561
:10C2B000B10539F521C09E012F5F3F4F0E940C52FE
:10C2C000882309F44CCF89819A81AB81BC81F80124
:10C2D000238D348DF9012789203129F048EF5FEF54
:10C2E0006FEF7FE004C048EF5FEF60E070E084171D
:10C2F0009507A607B70728F0C801A6D881114CCF2B
:10C3000026CFF80186839783A087B18745CFE114B4
:10C31000F10421F5D8011A964D915D916D917C91B2
:10C320001D9753968D919D910D90BC91A02D48170E
:10C3300059076A077B0790F071DB882309F407CF60
:10C3400040929D0250929E0260929F027092A002C3
:10C350008091430D81608093430D07C041E0C3018C
:10C36000B20195DB882309F4F2CED501F701E8513B
:10C37000F14F9F01280D391D2E173F0719F08D91A0
:10C380008193FACFA80CB91C61CFF80183899489F5
:10C39000A589B68984179507A607B70738F4438B94
:10C3A000548B658B768B848180688483F8018481CB
:10C3B00083FD02C0C10106C0C801B3DC882309F4B3
:10C3C000C6CEF8CF0F900F900F900F90DF91CF91C6
:10C3D0001F910F91FF90EF90DF90CF90BF90AF90A3
:10C3E0009F908F907F906F905F904F903F902F9095
:10C3F0000895CF93DF931F92CDB7DEB7698341E0F5
:10C4000050E0BE016F5F7F4F6BDE0F90DF91CF91E9
:10C41000089520E3FC0120833296862F82958F7049
:10C4200090E1899F601911246A3014F4605D01C0A5
:10C43000695C6293682F8111F0CF08957F928F928B
:10C440009F92AF92BF92CF92DF92EF92FF920F93A3
:10C450001F93CF93DF93CDB7DEB7A6970FB6F894AF
:10C46000DEBF0FBECDBF8C01762E942E852E20E22E
:10C47000B22ECE0101967C01FC012B2D11922A9542
:10C48000E9F783E594E09AA389A38FEF8BA38CA3AC
:10C490008DA38EA3680183E4C80ED11C43E450E051
:10C4A000BE016F5D7F4FC6010E947C55019609F465
:10C4B000B6C081E089838A8386E0A82EAB821C8285
:10C4C000F80164817581868197810E94BDB36D8377
:10C4D0007E838F83988789869A8680E890E09C8700
:10C4E0008B874CE150E0B701C6010E942854F70148
:10C4F0002B2D11922A95E9F7480188E0880E911CAE
:10C50000F401D70101900D92AA94E1F740E150E0C7
:10C51000B701C6010E942854F7011192BA94E9F7B5
:10C5200096E0A92EB12C40E250E0B701C6010E946E
:10C530002854F1E0AF1AB108B1F783E6898392E895
:10C540009A8393E59B838C8385E38D8381E08E833F
:10C550007F829DE3988797E099878A8786E0F40138
:10C56000DE011B9601900D928A95E1F78CE0898B94
:10C570008A8B66E07AE0CE0143960E9427B6F801E6
:10C580006385CE01499645DFF8016485CE014B965F
:10C5900040DFF8016585CE014D963BDF4EE150E06E
:10C5A000B701C6010E942854F3E07F121EC082E347
:10C5B000898384E08A83F80196859B8397859C8391
:10C5C00090899D8391899E8396E39F838887828D3E
:10C5D0008987838D8A87848D8B87858D8C874CE0B6
:10C5E00050E0B701C6010E94285487E3898386E0A2
:10C5F0008A8391E09B8393E09C838D838FE08E837D
:10C600008AE38F838BE388878FEF898749E050E047
:10C61000B701C6010E942854C6010E94DB56A696A7
:10C620000FB6F894DEBF0FBECDBFDF91CF911F9143
:10C630000F91FF90EF90DF90CF90BF90AF909F90C1
:10C640008F907F900895FC0124813581FB01448106
:10C65000558124173507A0F0FC0180819181009756
:10C6600079F0FB01608171816115710549F0241B2E
:10C67000350B820F931F0E941EB621E0892B09F013
:10C6800020E0822F08950F931F93CF93DF93EC0147
:10C69000CB01BE010E94D86C8C0160EB79E0CE0129
:10C6A0000E947536800F911FDF91CF911F910F91DE
:10C6B00008952F923F924F925F926F927F928F9246
:10C6C0009F92AF92BF92CF92DF92EF92FF920F9321
:10C6D0001F93CF93DF93CDB7DEB7E9970FB6F894EA
:10C6E000DEBF0FBECDBF7C014A015B0119010E9474
:10C6F00079822B013C0187010D5B1F4FC8010E940D
:10C70000CC5318161906A4F00E947982DC01CB01E3
:10C7100084199509A609B70988169906AA06BB06C1
:10C72000D8F062E370E080E090E00E944182E6CFC2
:10C7300042E250E0BE016F5F7F4FC8010E94585334
:10C740008981823011F080E035C1F80184899589B2
:10C7500083349105C1F702C08FEF2CC16D817E81BA
:10C760008F8198850E94BDB32B013C01F10160834C
:10C7700071838283938346E050E0B701685F7F4F07
:10C78000CE014D960E94E5B5892BE9F6F70180812F
:10C790009181A281B381481659066A067B0698F2F8
:10C7A00084819581A681B78184159505A605B70575
:10C7B00050F289899A89AB89BC8986879787A08B33
:10C7C000B18B4EEC50E060E070E0C8010E9458531D
:10C7D0001FA66701F2E2CF0ED11CC701869699AB66
:10C7E00088ABF701BA96FBABEAAB4701FAE18F0ED3
:10C7F000911C8D969DAB8CABF7017296FFABEEABA7
:10C80000CD9799AF88AF17019EE1290E311CF80131
:10C81000818D928D181619060CF0CBC0C8010E94AC
:10C8200077538333910509F4A5C0ACF481309105A9
:10C8300069F11CF4892B59F3B6C08330910571F16D
:10C84000069709F0B0C0C8010E9477535C0144E02C
:10C8500050E0B1012BC08A33910509F45FC034F474
:10C860008533910559F0C69771F19DC08B339105C1
:10C8700009F46AC08F3F910551F295C0C8010E942A
:10C880007753C8010E9477538FA7C1CFC8010E9478
:10C89000775344E050E06EA97FA911C0C8010E94FF
:10C8A00077535C0144E050E068AD79ADC8010E9467
:10C8B0005853A50155274450510960E070E0C80164
:10C8C0000E945853A4CFC8010E9477535C01B40161
:10C8D000CE0183960E947B6D8DA19EA1AFA1B8A5CC
:10C8E000892B8A2B8B2BA1F0ECA9FDA940805180CC
:10C8F00062807380B401CE0189960E947B6D8BA506
:10C900009CA5ADA5BEA584159505A605B70521F482
:10C9100044E050E0B401D3CFA50149C0C8010E9452
:10C92000775344E050E068A979A9C8010E945853A0
:10C93000F70166A177A180A591A50E94BDB366A36A
:10C9400077A380A791A763CFC8010E94775344E0E3
:10C9500050E06AA97BA9C8010E945853F70162A55B
:10C9600073A584A595A50E94BDB362A773A784A7EC
:10C9700095A74DCFC8010E94775344E050E0B6011F
:10C98000C8010E945853F70162A173A184A195A127
:10C990000E94BDB362A373A384A395A366A777A7E0
:10C9A00080AB91AB34CFC8010E947753AC015527BF
:10C9B00084CF8FA5E9960FB6F894DEBF0FBECDBF2A
:10C9C000DF91CF911F910F91FF90EF90DF90CF906B
:10C9D000BF90AF909F908F907F906F905F904F909F
:10C9E0003F902F9008952F923F924F925F926F92B7
:10C9F0007F928F929F92AF92BF92CF92DF92EF92EF
:10CA0000FF920F931F93CF93DF9300D000D0CDB749
:10CA1000DEB78C010E94F4AA2FEC37E040E050E032
:10CA20000E9455B2DC01CB010196A11DB11DF80198
:10CA300084839583A683B78380839183A283B38302
:10CA40005801F3E4AF0EB11CC5010E94215364E408
:10CA500070E0C5010E947254882309F431C10E941C
:10CA600079822B013C01812C912CC8018E5B9F4F58
:10CA70009E838D8348EEC42E43E0D42EE12CF12C0E
:10CA800052E0252EAD81BE818C91833009F4FFC028
:10CA900081111FC0F80184819581A681B78101961B
:10CAA000A11DB11D84839583A683B7830E947982DB
:10CAB0006419750986099709A70196010E9433B286
:10CAC000A90161E0C801BADC81E0AD81BE818C932F
:10CAD000C6C08430F1F4F80184819581A681B781C4
:10CAE0000196A11DB11D84839583A683B7830E94FF
:10CAF00079826419750986099709A70196010E9430
:10CB000033B2A90163E0C80199DCAD81BE812C92EA
:10CB1000A6C0813049F5F80142AD53AD64AD75ADA5
:10CB20009E012F5F3F4FC801C4DD382EF2E08F1306
:10CB300090C089819A81AB81BC81F80184839583FF
:10CB4000A683B7830E9479826419750986099709BB
:10CB5000A70196010E9433B2A90163E0C8016EDC0F
:10CB6000AD81BE813C927BC0823009F078C0F80173
:10CB700042AD53AD64AD75AD9E012F5F3F4FC8010F
:10CB800098DD382EF5E08F135DC0E3E0AD81BE8106
:10CB9000EC93F80182A193A1A4A1B5A1892B8A2BC2
:10CBA0008B2B41F484E893E0A0E0B0E082A393A350
:10CBB000A4A3B5A3F80186A197A1A0A5B1A5892B2F
:10CBC0008A2B8B2B61F482A193A1A4A1B5A1B69568
:10CBD000A7959795879586A397A3A0A7B1A7F801D6
:10CBE00082A593A5A4A5B5A5892B8A2B8B2BA9F487
:10CBF00082A193A1A4A1B5A1AC01BD0123E07695CA
:10CC00006795579547952A95D1F7841B950BA60BE9
:10CC1000B70B82A793A7A4A7B5A7F80186A197A1F0
:10CC2000A0A5B1A586A797A7A0ABB1AB82A593A5F8
:10CC3000A4A5B5A582AB93ABA4ABB5AB8824839474
:10CC4000912C0DC0F6E08F1304C0AD81BE811C9203
:10CC500006C0BFEF3B1203C0ED81FE811082F1E000
:10CC60008F16910409F40ECF0E947982DC01CB016A
:10CC700084199509A609B709F80126A937A940AD75
:10CC800051AD281739074A075B0708F0FBCEC501ED
:10CC90000E942153F80184819581A681B781019674
:10CCA000A11DB11D84839583A683B7830E947982D9
:10CCB000F801FE966083718382839383C40102C06E
:10CCC00080E090E026960FB6F894DEBF0FBECDBF91
:10CCD000DF91CF911F910F91FF90EF90DF90CF9058
:10CCE000BF90AF909F908F907F906F905F904F908C
:10CCF0003F902F9008950F931F93CF93DF93CDB75D
:10CD0000DEB728970FB6F894DEBF0FBECDBF809177
:10CD1000E00E811107C085EC9EE00E94603681E044
:10CD20008093E00E82E89EE090937F0E80937E0ECB
:10CD30008091810E811103C160E372E080E090E098
:10CD40000E9441821FB7F8948091800E811127C004
:10CD5000EAEEF8E08491E4EAF8E09491E82FF0E05C
:10CD6000EE0FFF1FEB5AF74FA591B491EC91E92319
:10CD700021F461E085E30E94828161E085E30E9405
:10CD8000E0818CB580618CBD8CB580648CBD61E028
:10CD900084E30E94E08161E083E30E94E08180916E
:10CDA000800E8F5F8093800E1FBFEFEBF8E0E49161
:10CDB000F0E0EE0FFF1FE55CF74F859194919093A3
:10CDC0007B0E80937A0EE9E7F8E0E491E093790E28
:10CDD00061E08AE00E94E0810E94B646CE010196A1
:10CDE0000E94857889819A810E94449084E380938F
:10CDF0007C0E0E941548882309F188E00E940348B0
:10CE00000E94F1478830D1F480E10E9403480E94DB
:10CE1000F147803199F480E00E9403480E94F14775
:10CE200081110CC041E050E0BE016F5F7F4F8FE188
:10CE300090E00E94C0468981833089F187E3809326
:10CE40007C0E0E9415488823F1F188E00E94034877
:10CE50000E94F1478830B9F580E10E9403480E94A2
:10CE6000F147182F803179F580E00E9403480E9435
:10CE7000F147811128C041E050E0BE016F5F7F4F54
:10CE800089E390E00E94C04689818430E1F41093E8
:10CE90007D0E0E94439081E08093810E50C080E41B
:10CEA00080937D0E10E042E06EE170E0812F0E94E1
:10CEB0005D5642E06FE170E0812F0E945D561F5F7A
:10CEC000183089F7E6CF83E380937C0E0E941548E3
:10CED000882371F180E10E9403480E94F14780316C
:10CEE00039F582E10E9403480E94F147823101F541
:10CEF00080E00E9403480E94F147811119C084E03C
:10CF000080937D0E15E5188741E050E0BE01685F13
:10CF10007F4F8BE190E00E9442471F8341E050E049
:10CF2000BE01695F7F4F8AE190E00E944247B1CF26
:10CF300010927C0E0E94439000E010E0BBC0CE0136
:10CF400001960E94857889819A810E94449046E0EA
:10CF500050E063EA72E089E090E00E94424783E596
:10CF600094E09A8389831B821C821D821E82CE01DB
:10CF700003960E947E3E0E94439080917E0E909187
:10CF80007F0EDC0192961D921D921D921C92959728
:10CF9000FC0116A217A210A611A69A961D921D9228
:10CFA0001D921C929D9740E65AEE60E070E046AB01
:10CFB00057AB60AF71AF40EA5FE060E070E0DA96D7
:10CFC0004D935D936D937C93DD973E9624E1DF0155
:10CFD0001D922A95E9F726E0E3EAF2E0DC011896D3
:10CFE00001900D922A95E1F7FC01EE5BFF4F108254
:10CFF000FADC8C01019709F05DC0CE0101960E9418
:10D00000857889819A810E94449060917E0E70910A
:10D010007F0E625F7F4FCE0101966DD5CE010396E4
:10D020000E947E3E60917E0E70917F0E6A5E7F4F01
:10D03000CE01019660D544E050E0BE016D5F7F4FA8
:10D0400081E090E00E94424760917E0E70917F0ED9
:10D050006E5E7F4FCE0101964ED544E050E0BE019A
:10D060006D5F7F4F85E090E00E9442470E944390B1
:10D0700060917E0E70917F0E625E7F4FCE010196B1
:10D080003AD58B819C81AD81BE818093AD14909304
:10D09000AE14A093AF14B093B0140E941C827F739F
:10D0A0008091A1029091A202682779277093A20231
:10D0B0006093A102C80128960FB6F894DEBF0FBE98
:10D0C000CDBFDF91CF911F910F9108950895CF9219
:10D0D000DF92EF92FF920F931F93CF93DF936C0138
:10D0E0007A018B01C0E0D0E0CE15DF0581F0D801D8
:10D0F0006D918D01D601ED91FC910190F081E02DB3
:10D10000C6011995892B11F02196EECF7E01C7013A
:10D11000DF91CF911F910F91FF90EF90DF90CF9013
:10D120000895FC01538D448D252F30E0842F90E02D
:10D13000821B930B541710F0CF9608950197089512
:10D14000FC01918D828D981761F0828DDF01A80F0F
:10D15000B11D5D968C91928D9F5F9F73928F90E031
:10D1600008958FEF9FEF0895FC01918D828D9817A0
:10D1700031F0828DE80FF11D858D90E008958FEFDD
:10D180009FEF0895FC01918D228D892F90E0805CA6
:10D190009F4F821B91098F739927089582EE91E129
:10D1A000F1DF21E0892B09F420E0822F08958FE739
:10D1B00092E1E8DF21E0892B09F420E0822F089535
:10D1C0008CE193E1DFDF21E0892B09F420E0822F5D
:10D1D000089589EB93E1D6DF21E0892B09F420E063
:10D1E000822F0895FC01848DDF01A80FB11DA35A81
:10D1F000BF4F2C91848D90E001968F739927848F77
:10D20000A689B7892C93A089B1898C918370806499
:10D210008C93938D848D981306C00288F389E02D3A
:10D2200080818F7D80830895EF92FF920F931F93EB
:10D23000CF93DF93EC0181E0888F9B8D8C8D9813C9
:10D2400005C0E889F989808185FD25C0F62E0B8D02
:10D2500010E00F5F1F4F0F731127E02E8C8DE81227
:10D260000BC00FB607FCFACFE889F989808185FFEA
:10D27000F5CFCE01B7DFF2CF8B8DFE01E80FF11DA8
:10D28000E35AFF4FF0829FB7F8940B8FEA89FB892E
:10D29000808180620AC09FB7F894EE89FF8960831D
:10D2A000E889F98980818370806480839FBF81E0F1
:10D2B00090E0DF91CF911F910F91FF90EF90089533
:10D2C000CF93DF93EC01888D8823C1F0EA89FB8935
:10D2D000808185FD05C0A889B9898C9186FD0EC025
:10D2E0000FB607FCF5CF808185FFF2CFA889B989F9
:10D2F0008C9185FFEDCFCE0175DFE8CFDF91CF9127
:10D30000089580E090E0892B19F063DF811116C049
:10D3100080E090E0892B19F053DF811112C080E08A
:10D3200090E0892B19F043DF81110EC080E090E07E
:10D33000892B79F033DF81110AC008950E94000023
:10D34000E7CF0E940000EBCF0E940000EFCF0C94CB
:10D35000000008950F931F93CF93DF93EC01888112
:10D360009981009729F02A813B812617370788F495
:10D370008B016F5F7F4F0E94F9B4009761F0998332
:10D3800088831B830A832C813D81232B11F4FC01AC
:10D39000108281E001C080E0DF91CF911F910F9159
:10D3A0000895EF92FF920F931F93CF93DF93611530
:10D3B000710511F480E01BC041155105B9F07B01E6
:10D3C000EC018C819D818A01080F191FB801CE01E3
:10D3D000C1DF882379F3288139818C819D81B70150
:10D3E000820F931F0E9427B61D830C8381E0DF917B
:10D3F000CF911F910F91FF90EF900895AF92BF9240
:10D40000CF92DF92EF92FF920F931F93CF93DF9310
:10D41000DC01CD90DC901197C114D10409F443C014
:10D420001496CD91DC9115972097E9F18C01760146
:10D430005701BFEFAB1ABB0AF7018081082E000C21
:10D44000990B0E9498AC892B11F07501F1CF2197AF
:10D45000CC0DDD1D8881082E000C990B0E9498AC24
:10D46000892B29F0CE15DF0510F02197F3CFAE01FF
:10D470004F5F5F4F4E195F09D80115965C934E932D
:10D480001497CE14DF0420F4B701C6010E94F2B550
:10D49000D801ED91FC91119714968D919C9115975F
:10D4A000E80FF91F1082DF91CF911F910F91FF902C
:10D4B000EF90DF90CF90BF90AF900895FC01248152
:10D4C00035816217730748F480819181009729F0B4
:10D4D000FC01E60FF71F8081089580E00895EF9228
:10D4E000FF920F931F93CF93DF936115710511F492
:10D4F00080E01DC08B01EC01CB010E94A7AC00971E
:10D50000A9F02C813D817C01E20EF31EB701CE0112
:10D5100021DF882369F3288139818C819D81B801BD
:10D52000820F931F0E94A0ACFD82EC8281E0DF910C
:10D53000CF911F910F91FF90EF900895CF93DF93BC
:10D540001F921F92CDB7DEB769831A8241E050E087
:10D55000BE016F5F7F4F25DF0F900F90DF91CF915E
:10D5600008956115710549F0FB0101900020E9F76C
:10D570003197AF01461B570B14CF80E00895FB0194
:10D5800044815581608171810CCF0F931F93CF939C
:10D59000DF938C01EB01FC0180819181009739F0D0
:10D5A0006881798161157105A1F40E9470B4888148
:10D5B0009981F801918380838A819B8193838283FF
:10D5C0008C819D8195838483198218821B821A82A3
:10D5D0000FC0F801428153812C813D8142175307CE
:10D5E00020F30E9427B68C819D81F8019583848366
:10D5F0001D821C82DF91CF911F910F910895CF93CF
:10D60000DF93EC0188819981009711F00E9470B43A
:10D61000198218821D821C821B821A82DF91CF918F
:10D620000895CF93DF93EC016115710559F0FB016B
:10D6300001900020E9F73197AF01461B570BB1DE8F
:10D64000811102C0CE01DBDFCE01DF91CF910895C1
:10D65000CF93DF93EC01FB0144815581608171819F
:10D66000A0DE811102C0CE01CADFCE01DF91CF91D1
:10D670000895EF92FF920F931F93CF93DF93EC01E6
:10D680008B016115710549F0CB010E94A7AC7C01AB
:10D69000BC01CE015FDE811103C0CE01B0DF07C047
:10D6A000FD82EC82B801888199810E94A0ACCE01F4
:10D6B000DF91CF911F910F91FF90EF900895EF921E
:10D6C000FF920F931F93CF93DF93EC017B018A01AD
:10D6D000BA0140DE811103C0CE0191DF07C01D8376
:10D6E0000C83B701888199810E9427B6CE01DF9112
:10D6F000CF911F910F91FF90EF900895CF93DF93FB
:10D70000EC016115710551F0FB0101900020E9F772
:10D710003197AF01461B570BD2DF01C070DFCE013E
:10D72000DF91CF910895CF93DF93EC01FB01861732
:10D73000970751F0608171816115710521F0448175
:10D740005581BDDF01C05BDFCE01DF91CF91089530
:10D75000FC01808191810C9470B4EF92FF920F9341
:10D760001F93CF93DF93CDB7DEB7A1970FB6F89491
:10D77000DEBF0FBECDBF7C01CB01BA01F701118224
:10D780001082138212821582148242E0420F8E01AF
:10D790000F5F1F4F0E948DAABC01C701AFDFA1968A
:10D7A0000FB6F894DEBF0FBECDBFDF91CF911F91B2
:10D7B0000F91FF90EF9008950F931F93CF93DF93F6
:10D7C000CDB7DEB7A2970FB6F894DEBF0FBECDBFC0
:10D7D0008C01CB01BA01F8011182108213821282EE
:10D7E0001582148230E0AE014F5F5F4F0E94BAACE9
:10D7F000BE016F5F7F4FC80181DFA2960FB6F8941C
:10D80000DEBF0FBECDBFDF91CF911F910F91089565
:10D81000CF93DF931F921F92CDB7DEB7FC01118229
:10D820001082138212821582148269831A82BE01C9
:10D830006F5F7F4F63DF0F900F90DF91CF9108955F
:10D84000FC011182108213821282158214829DCEF5
:10D85000FC0111821082138212821582148209CF78
:10D86000FC011182108213821282158214825BCF16
:10D87000FC011182108213821282158214826115BA
:10D88000710549F0FB0101900020E9F73197AF01E4
:10D89000461B570B14CF0895BF92CF92DF92EF92A1
:10D8A000FF920F931F93CF93DF937C016B018A014B
:10D8B000E9012417350720F4812F8901C42FD82FBF
:10D8C00062ED7AE0C701D4DFD60114968D919C9168
:10D8D000159708171907C0F48C179D0708F4EC0179
:10D8E000D601ED91FC911197EC0FFD1FB0801082D5
:10D8F0006D917C91600F711FC70100DFD601ED9122
:10D90000FC91EC0FFD1FB082C701DF91CF911F91F9
:10D910000F91FF90EF90DF90CF90BF9008958F927E
:10D920009F92AF92BF92EF92FF920F931F93CF936C
:10D93000DF93CDB7DEB7A1970FB6F894DEBF0FBE69
:10D94000CDBF7C01FA01CB0119A2223008F42AE0F4
:10D950008E010F5D1F4F822E912CA12CB12CBF0187
:10D96000A50194010E9433B2F901CA0101501109C5
:10D970006A3014F4605D01C0695CD8016C93232B9C
:10D98000242B252B61F7B801C7010E947536A1969B
:10D990000FB6F894DEBF0FBECDBFDF91CF911F91C0
:10D9A0000F91FF90EF90BF90AF909F908F90089550
:10D9B0008F929F92AF92BF92CF92DF92EF92FF929F
:10D9C0000F931F93CF93DF937C01EB016C0182E0F7
:10D9D000C80ED11C4701E5E08E0E911C00E010E05E
:10D9E000F60141916F0150E060E070E02AE0CE0165
:10D9F00096DF5C01E881F9810190F081E02D6EE213
:10DA0000CE0119958A0D9B1D080F191F8C149D04BA
:10DA100039F7F701458150E060E070E02AE0CE017F
:10DA20007EDF800F911FDF91CF911F910F91FF90AB
:10DA3000EF90DF90CF90BF90AF909F908F90089520
:10DA40000F931F93CF93DF93EC010E9475368C01E7
:10DA500060EB79E0CE010E947536800F911FDF9157
:10DA6000CF911F910F9108950C947536DB01149698
:10DA70004D915C9115976D917C91DC01ED91FC913C
:10DA80000280F381E02D19940F931F93CF93DF93BE
:10DA9000EC01ECDF8C0160EB79E0CE010E94753681
:10DAA000800F911FDF91CF911F910F910895EF92F9
:10DAB000FF920F931F93CF93DF938C017B01C0E004
:10DAC000D0E0F701EC0FFD1F6491662361F0D801EF
:10DAD000ED91FC910190F081E02DC8011995892B01
:10DAE00011F02196EECFCE01DF91CF911F910F91D2
:10DAF000FF90EF900895DC0183E594E08D939D9372
:10DB000084E0FB0101900D928A95E1F708951F9240
:10DB10000F920FB60F9211240BB60F922F933F93D3
:10DB20004F935F936F937F938F939F93AF93BF9325
:10DB3000EF93FF9382EE91E155DBFF91EF91BF915F
:10DB4000AF919F918F917F916F915F914F913F9195
:10DB50002F910F900BBE0F900FBE0F901F90189536
:10DB60001F920F920FB60F9211240BB60F922F93A4
:10DB70003F934F935F936F937F938F939F93AF9355
:10DB8000BF93EF93FF9382EE91E10E944181FF9159
:10DB9000EF91BF91AF919F918F917F916F915F9125
:10DBA0004F913F912F910F900BBE0F900FBE0F9092
:10DBB0001F9018951F920F920FB60F9211240BB65B
:10DBC0000F922F933F934F935F936F937F938F9316
:10DBD0009F93AF93BF93EF93FF938FE792E102DBA5
:10DBE000FF91EF91BF91AF919F918F917F916F9135
:10DBF0005F914F913F912F910F900BBE0F900FBEF1
:10DC00000F901F9018951F920F920FB60F9211242C
:10DC10000BB60F922F933F934F935F936F937F9326
:10DC20008F939F93AF93BF93EF93FF938FE792E10F
:10DC30000E944181FF91EF91BF91AF919F918F9190
:10DC40007F916F915F914F913F912F910F900BBEFC
:10DC50000F900FBE0F901F9018951F920F920FB646
:10DC60000F9211240BB60F922F933F934F935F9314
:10DC70006F937F938F939F93AF93BF93EF93FF9394
:10DC80008CE193E1AFDAFF91EF91BF91AF919F915A
:10DC90008F917F916F915F914F913F912F910F9055
:10DCA0000BBE0F900FBE0F901F9018951F920F92F2
:10DCB0000FB60F9211240BB60F922F933F934F93F1
:10DCC0005F936F937F938F939F93AF93BF93EF93E4
:10DCD000FF938CE193E10E944181FF91EF91BF910D
:10DCE000AF919F918F917F916F915F914F913F91F4
:10DCF0002F910F900BBE0F900FBE0F901F90189595
:10DD00001F920F920FB60F9211240BB60F922F9302
:10DD10003F934F935F936F937F938F939F93AF93B3
:10DD2000BF93EF93FF9389EB93E15CDAFF91EF915F
:10DD3000BF91AF919F918F917F916F915F914F9123
:10DD40003F912F910F900BBE0F900FBE0F901F9021
:10DD500018951F920F920FB60F9211240BB60F92C7
:10DD60002F933F934F935F936F937F938F939F93E3
:10DD7000AF93BF93EF93FF9389EB93E10E944181AF
:10DD8000FF91EF91BF91AF919F918F917F916F9193
:10DD90005F914F913F912F910F900BBE0F900FBE4F
:10DDA0000F901F901895CF92DF92EF92FF92CF9332
:10DDB000DF93EC01603282E078070CF03DC077FD24
:10DDC00006C0653B71052CF064EB70E002C060E0BA
:10DDD00070E0898128E830E06901C81AD10887FD20
:10DDE000D394CC0CDD1CCC0CDD1C0D2C000CEE08EF
:10DDF000FF088A8128E532E0281B310987FD339529
:10DE0000220F331F220F331FC901330FAA0BBB0B85
:10DE10009C01AD012C193D094E095F09DB010E94EF
:10DE20007BB224EB30E040E050E00E9455B2C20EDD
:10DE3000D31EE41EF51EB6013881303380F52981EA
:10DE400088E890E0821B910927FD9395880F991F20
:10DE5000880F991F6817790784F08A8148E552E096
:10DE6000481B510987FD5395440F551F440F551FFB
:10DE7000CB01461757070CF4CA010297880F991F68
:10DE80004FB7F894232F30E0F901EE0FFF1F2E0F4C
:10DE90003F1FF901E954FB4E928381834FBFDF910D
:10DEA000CF91FF90EF90DF90CF9008951F93CF9385
:10DEB000DF93EC01162F8881803308F04EC061E0BB
:10DEC000812F0E94E0818881E82FF0E09F01220FDE
:10DED000331FE20FF31FE954FB4E1F739081907CB8
:10DEE000192B108319821A826CE00E9496B39CE071
:10DEF000899FB001112440E050E09B01240F351FA1
:10DF0000F901EE0FFF1F2E0F3F1FF901E954FB4EE1
:10DF1000908196FD16C04F5F5F4F4C30510569F7F9
:10DF2000813001F51092800082E080938100109290
:10DF3000850010928400B19A80916F008260809376
:10DF40006F00E881F0E0CF01880F991FE80FF91FFB
:10DF5000E954FB4E8081806480838881DF91CF917A
:10DF60001F910895823061F4109290008093910087
:10DF7000109295001092940088BB80937100E1CFBD
:10DF8000833069F41092A00082E08093A100109287
:10DF9000A5001092A40089BB80937200D2CF81119A
:10DFA000D0CF1092200182E08093210110922501B0
:10DFB000109224018ABB80937300C3CF1F920F92EB
:10DFC0000FB60F9211240BB60F922F933F934F93DE
:10DFD0005F936F937F938F939F93AF93BF93EF93D1
:10DFE000FF9348E251E064E271E080E090E00E943B
:10DFF000F94CFF91EF91BF91AF919F918F917F91DC
:10E000006F915F914F913F912F910F900BBE0F90A9
:10E010000FBE0F901F9018951F920F920FB60F9280
:10E0200011240BB60F922F933F934F935F936F93EF
:10E030007F938F939F93AF93BF93EF93FF9348EAA0
:10E0400050E064EA70E083E090E00E94F94CFF91B8
:10E05000EF91BF91AF919F918F917F916F915F9160
:10E060004F913F912F910F900BBE0F900FBE0F90CD
:10E070001F9018951F920F920FB60F9211240BB696
:10E080000F922F933F934F935F936F937F938F9351
:10E090009F93AF93BF93EF93FF9348E950E064E9F8
:10E0A00070E082E090E00E94F94CFF91EF91BF9107
:10E0B000AF919F918F917F916F915F914F913F9120
:10E0C0002F910F900BBE0F900FBE0F901F901895C1
:10E0D0001F920F920FB60F9211240BB60F922F932F
:10E0E0003F934F935F936F937F938F939F93AF93E0
:10E0F000BF93EF93FF9348E850E064E870E081E05D
:10E1000090E00E94F94CFF91EF91BF91AF919F91E8
:10E110008F917F916F915F914F913F912F910F90D0
:10E120000BBE0F900FBE0F901F901895FF920F938C
:10E130001F93CF93DF93EC018B018091A30C9091FF
:10E14000A40C01969093A40C8093A30C2091A20C94
:10E15000222339F06AE070E00E94A2B31816190673
:10E1600024F1FF24F394F092A20C1092A40C1092CC
:10E17000A30C40E050E06DE07AE0CE010E941F3633
:10E180000230110531F0CE010E94853EF092410B24
:10E1900005C061E176E0CE010E94D03568E079E00B
:10E1A000CE010E94D0351092A20CDF91CF911F9129
:10E1B0000F91FF9008950F931F93CF93DF938C01DE
:10E1C00080914B1590E0FC01EE0FFF1F8E0F9F1FFB
:10E1D000FC01E954FB4E808186FD07C06091170366
:10E1E000709118038BE495E161DE64E670E080E0F5
:10E1F00090E00E94418280918B0290918C0297FF67
:10E2000004C010928C0210928B02C0918B02D091AC
:10E210008C02BE018BE495E1C6DD64E670E080E02F
:10E2200090E00E94418280918B0290918C020817AD
:10E2300019071CF1C017D1071CF5C53BD10514F017
:10E24000C4EBD0E0BE018BE495E1ADDD6EE170E0A2
:10E2500080E090E00E9441822196ECCFD7FF02C07F
:10E26000C0E0D0E0BE018BE495E19DDD6EE170E0A1
:10E2700080E090E00E94418221970C171D0774F303
:10E28000D7FD06C0C53BD1052CF0C4EBD0E002C0E1
:10E29000C0E0D0E0E0914B15F0E0CF01880F991F6E
:10E2A000E80FF91FE954FB4E80818F7B8083CE01FC
:10E2B000DF91CF911F910F9108950F931F93CF93EB
:10E2C000DF938C018091481590E0FC01EE0FFF1F59
:10E2D0008E0F9F1FFC01E954FB4E808186FD05C017
:10E2E00069E370E088E495E1E1DD64E670E080E0F8
:10E2F00090E00E9441828091890290918A0297FF6A
:10E3000004C010928A0210928902C0918902D091B1
:10E310008A02BE0188E495E146DD64E670E080E0B3
:10E3200090E00E9441828091890290918A020817B0
:10E3300019071CF1C017D1071CF5C43BD10514F017
:10E34000C4EBD0E0BE0188E495E12DDD6DE270E024
:10E3500080E090E00E9441822A96ECCFD7FF02C075
:10E36000C0E0D0E0BE0188E495E11DDD6DE270E023
:10E3700080E090E00E9441822A970C171D0774F3F9
:10E38000D7FD06C0C43BD1052CF0C4EBD0E002C0E1
:10E39000C0E0D0E0E0914815F0E0CF01880F991F70
:10E3A000E80FF91FE954FB4E80818F7B8083CE01FB
:10E3B000DF91CF911F910F9108952F923F924F922D
:10E3C0005F926F927F928F929F92AF92BF92CF9205
:10E3D000DF92EF92FF920F931F93CF93DF93CDB70E
:10E3E000DEB7CA52D1400FB6F894DEBF0FBECDBF24
:10E3F000CB5DDE4F59834883C552D1402091A30C99
:10E400003091A40C2F5F3F4F3093A40C2093A30CAA
:10E410002091A20C2111F8C28B016C0181E0809344
:10E42000A20C1092A40C1092A30C62ED7AE0CE0123
:10E43000875E9E4F1DDA62ED7AE0CE01815E9E4FCF
:10E4400017DA80918502909186028230910594F0CE
:10E4500020910F02309110023093820220938102AA
:10E46000029741F0809111029091120290938402E0
:10E470008093830240E050E06DE07AE0C6010E94A4
:10E480001F360130110509F02AC162ED7AE08AE5F4
:10E4900096E134D9212C312C7E0121E8E20EF11CC9
:10E4A000C701880F991F880F991F9C01205E384E65
:10E4B000C75DDE4F39832883C952D1403AE0432EED
:10E4C000512C612C712C44E6842E912CA12CB12C62
:10E4D000CB5DDE4FE881F981C552D1408081882330
:10E4E00009F478C0A701BE016F5F7F4FCE018B5D3D
:10E4F0009E4FB3D7049761F3BE016F5F7F4FCE018C
:10E500008F5F9E4FB5D9BE016F5F7E4FCE01875E94
:10E510009E4F3BD8CE018F5F9E4F1AD9B701CE01D7
:10E520008F5F9E4FA5D9BE016F5F7E4FCE01815E8A
:10E530009E4F2BD8CE018F5F9E4F0AD98091FA183B
:10E54000882369F1BE01675E7E4FCE018F5F9E4FCB
:10E5500087D96DE175E0CE018F5F9E4F62D8BC0117
:10E56000CE01895F9E4F7CD9CE01895F9E4F0E946C
:10E570003B7CCE01895F9E4FEBD8CE018F5F9E4FD3
:10E58000E7D8B701CE018F5F9E4F72D9CE018F5F62
:10E590009E4F0E94DA83CE018F5F9E4FD9D8C35E13
:10E5A000DE4F88819981CD51D140049708F00FC288
:10E5B00060E070E0CE01875E9E4F0E945E6A823509
:10E5C00009F496C0843509F493C08D7F843409F032
:10E5D000FEC18EC081E080933E0B8091D20B8823D8
:10E5E00019F0C6010E94853E8091D20B882329F044
:10E5F00068E079E0C6010E94D0351092A20C8091AB
:10E600005E1690915F16892B09F469C0CE01895F6F
:10E610009E4F0E944A3769ED77E0CE018F5F9E4F93
:10E6200027D9BE01695F7E4FCE018F5F9E4F10D804
:10E630006AE175E00E94116B6AE576E109D8BC01D8
:10E640008AE596E170D8CE018F5F9E4F81D8CE01CA
:10E65000895F9E4F7DD86AE576E1CE018F5F9E4F40
:10E66000FFD8AE014F5F5E4F62E070E082E392E060
:10E670000E942441182FCE018F5F9E4F69D86AE512
:10E6800076E1CE018F5F9E4F112359F0E9D86EE1FC
:10E6900077E0CE018F5F9E4F0E94116B62E476E1BE
:10E6A0000AC0DED86EE177E0CE018F5F9E4F0E94F8
:10E6B000116B6CE376E10E94286BBC01CE01895F8F
:10E6C0009E4FCED8CE01895F9E4F0E94DA83CE0145
:10E6D000895F9E4F3DD8CE018F5F9E4F39D8CE01C6
:10E6E000815E9E4F35D8CE01875E9E4F31D88CC15A
:10E6F00041E050E0BE01675E7E4FCE018F5F9E4FCE
:10E700000E948C36CE018F5F9E4F0E94344C8B014D
:10E710006130710521F400912E1810912F180330EB
:10E72000110521F4009130181091311810161106BE
:10E730000CF047C180918502909186028017910765
:10E740000CF43FC160E070E0CE01875E9E4F0E94F6
:10E750005E6A823509F070C0C7010E9455AC892BF2
:10E7600039F4F801EE0FFF1FE158FD4F11821082BE
:10E77000C7010E9455AC81309105B9F5F801EE0F43
:10E78000FF1FE158FD4F91838083C801880F991FB7
:10E79000880F991FC95DDE4F99838883C752D14086
:10E7A000FC01E357FD4F80819181A281B38118164E
:10E7B00019061A061B065CF080829182A282B3823F
:10E7C0000730110524F040825182628273820E94D8
:10E7D000254EC95DDE4FE881F981C752D140E75E21
:10E7E000FD4F6083718382839383C75DDE4F6881B1
:10E7F0007981C952D140CE018D5E9E4F39D8B80182
:10E80000E3E0660F771FEA95E1F7685D784ECE0189
:10E81000835F9E4F2DD86AE576E1CE01895F9E4FDA
:10E820001FD8BE01635F7E4FCE01895F9E4F0E945D
:10E83000286B6EEE77E076C0863409F09CC0C70185
:10E840000E9455AC892B39F4F801EE0FFF1FED5EE5
:10E85000FD4F11821082C7010E9455AC8130910595
:10E8600039F4F801EE0FFF1FED5EFD4F91838083B9
:10E870009801220F331F220F331FC95DDE4F3983EA
:10E880002883C752D140F901E357FD4F8081918120
:10E89000A281B381181619061A061B0664F0073008
:10E8A00011052CF480829182A282B38204C040823E
:10E8B0005182628273820E94254EC95DDE4FE881DB
:10E8C000F981C752D140E75EFD4F60837183828337
:10E8D0009383C75DDE4F68817981C952D140CE01F3
:10E8E0008D5E9E4F0E94386CB80143E0660F771F23
:10E8F0004A95E1F7685D784ECE01835F9E4F0E9496
:10E90000386C6AE576E1CE01895F9E4F0E94306CDB
:10E91000BE01635F7E4FCE01895F9E4F0E94286BD0
:10E9200066E27AE00E94116BBE016F5F7E4F0E942B
:10E93000286B6DE175E00E94116BBE016D5E7E4F2C
:10E940000E94286B6AE175E00E94116BBC018AE5A8
:10E9500096E10E94936BCE01895F9E4F0E94A86B47
:10E96000CE01835F9E4F0E94A86BCE018D5E9E4FAD
:10E970000E94A86B26C0843459F4C7010E9472AC6F
:10E98000000F111F000F111FF801EF5FFD4F0CC0AA
:10E990008435B9F4C7010E9472AC000F111F000F3B
:10E9A000111FF801E357FD4F6083718382839383C6
:10E9B0000E94254EF801E75EFD4F608371838283DC
:10E9C0009383CE018F5F9E4F0E94A86B81CD8BE019
:10E9D000281631040CF07CCD86E0829D8001839D59
:10E9E000100D1124BE016F5F7F4FC8018E55994EE7
:10E9F0000E947E6BB701C801805A994E0E947E6BBF
:10EA00003FEF231A330A64CDC65DDE4F0FB6F8948C
:10EA1000DEBF0FBECDBFDF91CF911F910F91FF9051
:10EA2000EF90DF90CF90BF90AF909F908F907F90AE
:10EA30006F905F904F903F902F900895DF92EF92EC
:10EA4000FF920F931F93CF93DF93CDB7DEB7C451DF
:10EA5000D1400FB6F894DEBF0FBECDBFCD5EDE4F06
:10EA600059834883C351D1402091A30C3091A40C09
:10EA70002F5F3F4F3093A40C2093A30C2091A20C46
:10EA80002111B5C08B017C01DD24D394D092A20C5E
:10EA90001092A40C1092A30C62ED7AE0CE01895F73
:10EAA0009E4F0E94386C62ED7AE0CE01835F9E4FEC
:10EAB0000E94386C40E050E06DE07AE0C7010E94AF
:10EAC0001F360130110509F088C062ED7AE08AE551
:10EAD00096E10E947E6BCD5EDE4FE881F981C351E5
:10EAE000D1408081811111C00E94E937D092410B41
:10EAF00074C0AE014F575F4FBE016F5F7F4FCE01B5
:10EB00008D5E9E4FAAD4049751F4CD5EDE4FE8810E
:10EB1000F981C351D14080818111EBCF58C0BE0132
:10EB20006F5F7F4FCE018F5F9E4F0E94386CBE019A
:10EB30006F5F7E4FCE01895F9E4F0E94C56ACE01F6
:10EB40008F5F9E4F0E94A86BBE016F577F4FCE0113
:10EB50008F5F9E4F0E94386CBE016F5F7E4FCE016B
:10EB6000835F9E4F0E94C56ACE018F5F9E4F0E94B9
:10EB7000A86BBE01695F7E4F8AE596E10E94BF6A7D
:10EB8000CF5EDE4F88819981C151D140892B09F434
:10EB9000BCCF6DE175E0CE018F5F9E4F0E94386C57
:10EBA000BE01635F7E4FCE018F5F9E4F0E94286B38
:10EBB0006AE175E00E94116BBC018AE596E10E9452
:10EBC000BF6ACE018F5F9E4F0E94A86B9ECF6AE501
:10EBD00076E186E396E10E94936BCE01835F9E4FC0
:10EBE0000E94A86BCE01895F9E4F0E94A86BCC5EED
:10EBF000DE4F0FB6F894DEBF0FBECDBFDF91CF91D1
:10EC00001F910F91FF90EF90DF9008950F931F9346
:10EC1000CF93DF93CDB7DEB762970FB6F894DEBF20
:10EC20000FBECDBF00E010E00E94413B892B79F47C
:10EC30000A30110509F025C160E679E0CE010196A0
:10EC40000E94386CCE0101960E94DA830BC10A3013
:10EC5000110591F30E94254E6093A90C7093AA0CA4
:10EC60008093AB0C9093AC0C0E94254E6093AD0C3E
:10EC70007093AE0C8093AF0C9093B00CCE010196C4
:10EC80000E944A37CE0101960E94DA83CE01019696
:10EC90000E94A86B0E947C4FBC01CE0107960E9487
:10ECA00098366CEE77E0CE0107960E94B16A0E941A
:10ECB000764FBC01CE0101960E949836BE016F5F6F
:10ECC0007F4FCE0107960E94BF6ACE0101960E9437
:10ECD000A86B6CEE77E0CE0107960E94B16A0E94A5
:10ECE0006E4FBC01CE0101960E949836BE016F5F47
:10ECF0007F4FCE0107960E94BF6ACE0101960E9407
:10ED0000A86B6AE27AE0CE0101960E94386CBE01DF
:10ED1000695F7F4FCE0101960E94286BBC01CE0136
:10ED20000D960E94306C4AE050E06FEF7FEFCE010D
:10ED30000D960E946C85CE010D960E94A86BCE01A7
:10ED400001960E94A86BCE0107960E94A86B68EE00
:10ED500073E080E090E00E9441820E94884FBC01F5
:10ED6000CE010D960E9498360E94824FBC01CE01C2
:10ED700001960E94983666E076E0CE0107960E94E2
:10ED8000386CBE016F5F7F4FCE0107960E94286BE3
:10ED9000BC01CE010D960E94BF6ACE0107960E946B
:10EDA000A86BCE0101960E94A86B0E94254E0E947E
:10EDB0006B4E6091480D70E0CE0101960E9498362E
:10EDC00066E076E0CE0107960E94386CBE016F5F68
:10EDD0007F4FCE0107960E94286BBC01CE010D9695
:10EDE0000E94BF6ACE0107960E94A86BCE010196D1
:10EDF0000E94A86B60E37AE0CE0101960E94386C15
:10EE0000BE01635F7F4FCE0101960E94286BBC015B
:10EE1000CE0107960E94306C4AE050E06FEF7FEF22
:10EE2000CE0107960E946C85CE0107960E94A86BC2
:10EE3000CE0101960E94A86BCE010D960E94A86B90
:10EE400068EE73E080E090E00E944182CE0101967E
:10EE50000E94CE364AE050E06FEF7FEFCE01019680
:10EE60000E946C85CE0101960E94A86B62960FB637
:10EE7000F894DEBF0FBECDBFDF91CF911F910F91F0
:10EE800008950F5F1F4F68EE73E080E090E00E94EE
:10EE900041824091970C5091980C6091990C70911F
:10EEA0009A0CCE01019629D5CE0101960E94DA83F3
:10EEB000CE0101960E94A86BB7CEEF92FF920F93FE
:10EEC0001F93CF93DF93CDB7DEB76E970FB6F8944D
:10EED000DEBF0FBECDBF0E94739060ED77E080E093
:10EEE00090E00E9441820E947B667C0168EE73E0A4
:10EEF00080E090E00E9441820BE010E0EF2899F45E
:10EF00000150110981F060ED77E080E090E00E940F
:10EF100041820E947B667C0168EE73E080E090E0B5
:10EF20000E944182EBCF0E940F8662ED7AE0CE0113
:10EF30000D960E94386C6BEF78E0CE0143960E94EC
:10EF4000286CCE0149960E9468588E8D1F928F932F
:10EF50008D8D1F928F938C8D1F928F938B8D1F920F
:10EF60008F9386E39AE09F938F9382E49BE09F9335
:10EF70008F930E9465B662E47BE0CE0101960E9409
:10EF8000386CBE016F5F7F4FCE010D960E94C56A3F
:10EF9000CE0101960E94A86BBE016D5E7F4FCE012F
:10EFA00001960E94306CBE01635F7F4FCE010196D7
:10EFB0000E94286BBC01CE0107960E94306CCE01E6
:10EFC00007960E94DA83CE0107960E94A86BCE01B5
:10EFD00001960E94A86BBE01635F7F4FCE01019630
:10EFE0000E94306CAE014F5F5F4F63E070E08FE3D3
:10EFF00092E00E942441182FCE0101960E94A86B36
:10F000000FB6F894DEBF0FBECDBF111122C062E46F
:10F010007AE0CE0101960E94386CBE016D5E7F4F92
:10F02000CE0101960E94286B6CE376E10E94286B6A
:10F03000BC01CE0107960E94306CCE0107960E945B
:10F04000DA83CE0107960E94A86BCE0101960E943A
:10F05000A86BCE0143960E94A86BCE010D960E942C
:10F06000A86B6E960FB6F894DEBF0FBECDBFDF91D2
:10F07000CF911F910F91FF90EF900895CF92DF9263
:10F08000EF92FF920F931F93CF93DF9300D000D0A6
:10F09000CDB7DEB77C01FB01848195818A01081B15
:10F0A000190B1016110624F0C7010E94206C1DC018
:10F0B000CE0101960E94306CCC24C394D12C6AE11D
:10F0C00075E0CE0101960E94B16AFFEFCF1ADF0A08
:10F0D0000C151D05A4F7BE016F5F7F4FC7010E948D
:10F0E000206CCE0101960E94A86BC70126960FB630
:10F0F000F894DEBF0FBECDBFDF91CF911F910F916E
:10F10000FF90EF90DF90CF90089520E5FC012083E1
:10F1100021E021830895282F30915611313208F0D3
:10F120004AC0809132118111FCCF9091551142E07B
:10F1300040933211209331112FEF20933011109210
:10F140002F1130932E11E5E3F1E1AEE0B1E120E0C3
:10F15000321721F041914D932F5FFACF10920D118C
:10F1600020910D11990F922B90930D1190910C11EC
:10F17000913061F410920C1190910D119093BB009D
:10F180009091BC0093FDF8CF95EC01C095EE909363
:10F19000BC00909132119230E1F3909130119F3F79
:10F1A00079F080913011803241F0809130118033BC
:10F1B00031F084E005C081E003C082E001C083E05B
:10F1C0001092341110925611109233110895682F35
:10F1D00086E594E10C94CB4CCF93C82F682F607FC9
:10F1E0008EEB98E10E94D34D80E1C89FB0011124BD
:10F1F0008EEB98E1CF910C94D34DCF93DF93CDB7A5
:10F20000DEB728970FB6F894DEBF0FBECDBF98E0EB
:10F21000EFE4F3E0DE01119601900D929A95E1F78B
:10F220009091C718961710F46FEF690FFE01319691
:10F23000E60FF11DE60FF11D9081890F8068289679
:10F240000FB6F894DEBF0FBECDBFDF91CF91C4CF14
:10F25000CF92DF92EF92FF92CF93DF93EC016A019E
:10F260007B01E889F98982E080834115514E61056F
:10F270007105B1F060E079E08DE390E0A7019601BF
:10F280000E9433B2DA01C9010197A109B109B6950B
:10F29000A795979587959C01211580E13807A8F0DF
:10F2A000E889F989108260E874E88EE190E0A701AE
:10F2B00096010E9433B2DA01C9010197A109B1098F
:10F2C000B695A795979587959C01EC85FD8530832C
:10F2D000EE85FF852083188EEC89FD8986E080838A
:10F2E000EA89FB89808180618083EA89FB8980814A
:10F2F00088608083EA89FB89808180688083EA89CD
:10F30000FB8980818F7D8083DF91CF91FF90EF908B
:10F31000DF90CF9008958F3F2FEF920789F0E09113
:10F32000891591E09E0F909389150E2E000CFF0B0E
:10F33000E25BFA4E838F903219F48FE18093891546
:10F340000895CF92DF92EF92FF92809164158830FA
:10F3500008F046C0E0918915E11145C00E9479820C
:10F360006B017C0128EEC20E23E0D21EE11CF11CD1
:10F3700088E595E10E94DC54882391F18091BF15C6
:10F38000882331F080918A1590918B15892B41F15A
:10F3900088E595E10E94A0538F3F2FEF920779F007
:10F3A0002091BF15222349F120918A1530918B15A8
:10F3B0002150310930938B1520938A151EC00E946D
:10F3C0007982C616D706E806F90690F610928915D6
:10F3D00088E595E10E94375588E595E10E94FF5444
:10F3E0008FEF9FEF0AC0E150E09389150E2E000CBD
:10F3F000FF0BE25BFA4E838D90E0FF90EF90DF9081
:10F40000CF900895EF92FF920F931F93CF93DF93C6
:10F410008C017C01EC0189918823A9F092DFF7012E
:10F4200021917F01022E000C330B8217930799F371
:10F4300072DF2197C017D10741F08A91082E000C86
:10F44000990B69DFF7CF81E001C080E0DF91CF91B8
:10F450001F910F91FF90EF9008958F929F92AF921E
:10F46000BF92CF92DF92EF92FF920F931F93CF93B1
:10F47000DF9300D0CDB7DEB74C017B016A01DC0120
:10F48000ED91FC9180E8DB01982F1D929A95E9F7A8
:10F49000DA011D928A95E9F78081882309F466C014
:10F4A00090E8A92EB12C8F010F5F1F4F608166324B
:10F4B00009F456C034F4662309F451C0653239F0BA
:10F4C00059C06B3209F455C06D33D1F053C08181FE
:10F4D0008983882309F444C082818A838F01811142
:10F4E00003C00E5F1F4F3CC00D5F1F4F1B8240E1EA
:10F4F00050E060E070E0CE0101960E9448AB3AC057
:10F500008181882369F180E8E82EF12CF8010F5FF2
:10F510001F4F6081653259F024F461113AC08F01A8
:10F5200036C06632A1F16B32A1F560E232C0818152
:10F530008983882361F182818A838F01811103C0CD
:10F540000E5F1F4F24C00D5F1F4F1B8240E150E034
:10F5500060E070E0CE0101960E9448AB1AC08F01B6
:10F5600081E090E0D4010D931C9323C084E090E0EF
:10F5700020C060E2B2E0AB16B104CCF0F7016083CA
:10F58000F1E0AF1AB108C70101967C0110C083E019
:10F59000E8CFE2E0EE16F1040CF4B8CFD6016C939C
:10F5A000B1E0EB1AF108F60131966F01AFCFF80127
:10F5B0007ACF0F900F900F90DF91CF911F910F9105
:10F5C000FF90EF90DF90CF90BF90AF909F908F9083
:10F5D00008950F931F93CF93DF93CDB7DEB7629754
:10F5E0000FB6F894DEBF0FBECDBF8C01CB01F80182
:10F5F0001182108213821282158214824AE0BE01A7
:10F600006F5F7F4F0E94B0ACBE016F5F7F4FC8013C
:10F610000E947E6B62960FB6F894DEBF0FBECDBF20
:10F62000DF91CF911F910F910895CF93DF93FB014D
:10F6300022813381DC0113963C932E9312974481EF
:10F6400055816681778114964D935D936D937C937C
:10F650001797408551856285738518964D935D9304
:10F660006D937C931B971C96EF012C969C01275E53
:10F670003F4F49914D93A217B307D9F7218D328D92
:10F68000FC01328F218FDF91CF910895909132113B
:10F690009111FCCF91E090933211909331112FEFA3
:10F6A0002093301110922F11260F20932E1190933A
:10F6B0000D1190910D11880F892B80930D11809160
:10F6C0000C11813061F410920C1180910D11809316
:10F6D000BB008091BC0083FDF8CF85EC01C085EEB6
:10F6E0008093BC00809132118130E1F380912F1121
:10F6F000861710F460912F11AEE0B1E1ECEEF0E16D
:10F7000080E0861721F09D9191938F5FFACF089545
:10F71000AF92BF92CF92DF92EF92FF920F931F931F
:10F72000CF93DF93C82FD62F109242181092431810
:10F7300010924418109245181092461861E040D675
:10F7400060E08C2FDFD56D2F70E080E090E099D6DF
:10F7500060E08C2F35D68BE990E00197F1F700E956
:10F7600011E08C2FA7D5892B31F401501109C9F76D
:10F770008EEF9FEF47C000E911E08C2F9BD50197DA
:10F7800009F43BC018E2D0E800E090E9E92EFF243C
:10F79000F3948C2F8FD5892B29F481E0E81AF10896
:10F7A000C1F7E6CF49D66B017C0180E9A82EBB24C6
:10F7B000B3948C2F7FD5019729F481E0A81AB10862
:10F7C000C1F7D6CF39D6DC01CB018C199D09AE0922
:10F7D000BF098997A105B10538F0E02FF0E0E65C9C
:10F7E000F74E80858D2B8087D69511F40F5FD0E87A
:10F7F000115059F680E090E005C00150110909F060
:10F80000BCCFB6CFDF91CF911F910F91FF90EF90BA
:10F81000DF90CF90BF90AF9008950F931F93CF9339
:10F82000DF932091AA02222309F12091A902222329
:10F83000E9F0EB018C0161E080E0DFDCB8018EEBE8
:10F8400098E10E94366D67E479E08EEB98E10E94C2
:10F85000576D61E0F8018481D0DCBE01DD0F880BBB
:10F86000990BDF91CF911F910F910BC6DF91CF9133
:10F870001F910F910895CF93DF93FC01248135816F
:10F88000232B69F0EC01BC0189EB93E10E94366DFA
:10F89000BE0182EE91E1DF91CF910C94366DDF9144
:10F8A000CF910895CF93DF93EC016E857F85888992
:10F8B000998941E00E94475D882341F08A8920E2CE
:10F8C000829FC00111248851914F02C080E090E0D6
:10F8D000DF91CF910895CF93DF93EC01898D9A8DBD
:10F8E000009741F00E94BD5E898D9A8D0E9470B490
:10F8F0001A8E198EDF91CF9108950F931F93CF9396
:10F90000DF93CDB7DEB7A1970FB6F894DEBF0FBE79
:10F91000CDBF8C01CB01BA01F80111821082138294
:10F920001282158214822AE0AE014F5F5F4F0E945F
:10F93000EFACBE016F5F7F4FC8010E947E6BA19646
:10F940000FB6F894DEBF0FBECDBFDF91CF911F91F0
:10F950000F910895DC015996ED91FC915A973097DB
:10F9600021F081E09581911101C080E00895EF922E
:10F97000FF920F931F93CF93DF93EC017B018A01DA
:10F980000E9450368FEB93E0998388838DE190E05D
:10F990000E94D8B39A8F898F009779F02DE1F701F3
:10F9A000DC0101900D922A95E1F74CE050E0B8019E
:10F9B000CE010C960E943CB6188EDF91CF911F911C
:10F9C0000F91FF90EF9008958F929F92AF92BF9208
:10F9D000CF92DF92EF92FF920F931F93CF93DF931B
:10F9E00000D01F92CDB7DEB7FC018581813079F55B
:10F9F000948191FF2CC04389548965897689452B70
:10FA0000462B472B09F45CC07F0140E050E0BA016F
:10FA1000CF010E94275B8823D1F0F7018788908C63
:10FA2000A18CB28CC38CD48C82E090E0A0E0B0E0DA
:10FA3000F60180839183A283B3839E012F5F3F4FA2
:10FA4000B501A401C6010E940C52811102C080E0E0
:10FA500037C000E010E09801B501A401C6010E9482
:10FA60006B518823A1F389809A80AB80BC80F6011A
:10FA70008789803129F088EF9FEFAFEFBFE004C0A6
:10FA800088EF9FEFA0E0B0E088169906AA06BB06B3
:10FA9000A0F2F701178A108E118E128E138A148A23
:10FAA000158A168A848180688483C7010E94915ECA
:10FAB000882369F240E050E0BA01C7010E94275B49
:10FAC0000F900F900F900F90DF91CF911F910F919A
:10FAD000FF90EF90DF90CF90BF90AF909F908F906E
:10FAE00008954F925F926F927F92AF92BF92CF92A2
:10FAF000DF92EF92FF920F931F93CF93DF9300D08B
:10FB00001F92CDB7DEB78C0149835A836B837C8308
:10FB10005901C12CD12C7601412C82E0582E612C48
:10FB2000712C49815A816B817C819E012F5F3F4FEF
:10FB3000C8010E940C52882351F1D301C201F8017F
:10FB4000058404C0880F991FAA1FBB1F0A94D2F70F
:10FB5000C80ED91EEA1EFB1E49815A816B817C8129
:10FB60008789803129F088EF9FEFAFEFBFE004C0B5
:10FB700088EF9FEFA0E0B0E0481759076A077B07BE
:10FB800080F2F501C082D182E282F38281E00F909F
:10FB90000F900F900F90DF91CF911F910F91FF90D9
:10FBA000EF90DF90CF90BF90AF907F906F905F907D
:10FBB0004F9008950F931F93CF93DF9300D000D001
:10FBC000CDB7DEB78C01CE0101960E94CE364AE059
:10FBD00050E06FEF7FEFCE0101967ED7CE01019608
:10FBE0000E94A86BB801CE0101960E94306C6AE0B9
:10FBF00070E0CE01019611DECE0101960E94A86B45
:10FC000026960FB6F894DEBF0FBECDBFDF91CF9121
:10FC10001F910F91089590E0FC013197E231F105B9
:10FC200008F04EC08827EE58FF4F8F4F0C94B5B3A5
:10FC3000809180008F7703C0809180008F7D8093BA
:10FC40008000089580918000877FF9CF84B58F77F9
:10FC500002C084B58F7D84BD08958091B0008F77F8
:10FC600003C08091B0008F7D8093B0000895809193
:10FC700090008F7707C0809190008F7D03C08091A6
:10FC80009000877F8093900008958091A0008F77E7
:10FC900007C08091A0008F7D03C08091A000877F66
:10FCA0008093A0000895809120018F7707C08091F4
:10FCB00020018F7D03C080912001877F80932001E8
:10FCC00008955F926F927F928F929F92AF92BF92B0
:10FCD000CF92DF92EF92FF920F931F93CF93DF9318
:10FCE000CDB7DEB7C754D1090FB6F894DEBF0FBE4B
:10FCF000CDBF5C013B0119A218A283EB93E09F8F5B
:10FD00008E8F1BA21C821B829A8389831E8200E035
:10FD100010E06E018EE1C80ED11C8CE8E82E84E163
:10FD2000F82EF501E00FF11F80818F3211F40F5F83
:10FD30001F4FD501A00FB11FFE01FB9680E090E0A0
:10FD40004F012D912F3249F0222339F001960F5F98
:10FD50001F4F21938C309105A1F7F401E80FF91F93
:10FD60001082F501E00FF11F80818F3211F40F5FD7
:10FD70001F4FF501E00FF11F508041E0511040E0AE
:10FD800020E030E0B401C701F301199581110AC0E8
:10FD9000FCE8EF16F4E1FF0619F0C7010E94BD5E12
:10FDA00080E029C05520B9F021E0A401B701C601C7
:10FDB0000E94C85E982E8CE8E81684E1F806A9F047
:10FDC000C7010E94BD5E992059F39E2D8F2D7601AB
:10FDD000C92ED82EA6CF9CE8E91694E1F90619F0B1
:10FDE000C7010E94BD5E81E006C09920C9F2FE01F4
:10FDF00031967F01EACFC95BDF4F0FB6F894DEBFC3
:10FE00000FBECDBFDF91CF911F910F91FF90EF906B
:10FE1000DF90CF90BF90AF909F908F907F906F902A
:10FE20005F9008958F929F92AF92BF92CF92DF9290
:10FE3000EF92FF92CF93DF93C82F82E694E19093E5
:10FE4000CF118093CE11CC2369F1C53010F080E042
:10FE50000CC140E060E070E0CB010E94475D882368
:10FE6000B1F320E1C29FC00111248852914FFC01DF
:10FE7000E254FE4F20812F7751F73C96408151810B
:10FE800062817381443651056105710500F3349731
:10FE9000C080D180E280F380C114D104E104F10478
:10FEA00021F4D5CFC12CD12C760140E0C701B60199
:10FEB0000E94475D882359F28091F30E9091F40ED1
:10FEC0008115924021F6A091F80EAA2309F4BFCF24
:10FED0006091F60E7091F70E6115710509F4B7CFB8
:10FEE0002091F50E222309F4B2CFA0938014209321
:10FEF000721480E030E041E050E0C82FFA01082E93
:10FF000002C0EE0FFF1F0A94E2F72E173F0739F0E9
:10FF10008F5FC83091F789E080937B1498CF8093EE
:10FF20007B142091FE0E3091FF0E2115310519F042
:10FF300040E050E008C020910C0F30910D0F40912F
:10FF40000E0F50910F0F209373143093741440933D
:10FF500075145093761446015701860E971EA11C06
:10FF6000B11C8092811490928214A0928314B0925A
:10FF70008414E091F90EF091FA0EF0938714E09357
:10FF80008614B0E00E9471B2860E971EA81EB91E9C
:10FF90008092881490928914A0928A14B0928B1443
:10FFA00085E0EE0FFF1F8A95E1F7E150FE4FEF2F3E
:10FFB000FF27E6958E0E9F1EA11CB11C80927C141B
:10FFC00090927D14A0927E14B0927F142091FB0E2B
:10FFD0003091FC0E2115310521F0A90160E070E09F
:10FFE00008C04091080F5091090F60910A0F70915D
:10FFF0000B0FD701C60188199909AA09BB09840FFB
:020000021000EC
:10000000951FA61FB71F04C0B695A795979587950E
:10001000CA95D2F78093771490937814A0937914AB
:10002000B0937A14853F2FE09207A105B10510F433
:100030008CE018C0853F9F4FA105B10510F480E109
:1000400011C08091140F9091150FA091160FB091CF
:10005000170F8093881490938914A0938A14B093F7
:100060008B1480E28093851481E0DF91CF91FF9023
:10007000EF90DF90CF90BF90AF909F908F900895BA
:10008000CF93DF93482F50E060E070E020E189EBF0
:1000900093E10E948F6CEC0160EB79E089EB93E1D6
:1000A0000E9475368C0F9D1FDF91CF9108958F921E
:1000B0009F92AF92BF92CF92DF92EF92FF920F93F7
:1000C0001F93CF93DF93CDB7DEB760970FB6F89449
:1000D000DEBF0FBECDBF7C0190917C0E992309F449
:1000E000BCC0933311F008E001C004E05B01CE0115
:1000F00001960BD889819A810E9444909E012F5FBE
:100100003F4F6901490110E0812F0E949956F40187
:1001100081934F018823C9F01F5F0113F5CF10E0D1
:10012000F60181916F018D3159F0883149F08A5182
:10013000823030F01F5F0113F3CF0E9443908DC0D7
:1001400060E170E0812F0E94A646C12ED12CF601FD
:10015000EE0FFF1FE854FE4E1182108283EE93E0F3
:100160000197F1F742E860E070E0812F0E945D5650
:100170004FEF62E070E0812F0E945D56A114B10440
:1001800011F0B50113C08091A1029091A2020196D5
:100190008115F0EC9F0710F480E090EC9093A202A0
:1001A0008093A1026091A1027091A202812F0E940E
:1001B000675586E0EBE5F3E0DE01199601900D92BC
:1001C0008A95E1F7F70183818F778C8784818D870A
:1001D00085818E87A7014E5F5F4F24E030E06CE0A1
:1001E00070E0812F0E945555B501812F0E94D24B9E
:1001F00026E030E0AE01475F5F4F66E070E0812FA0
:100200000E94555561E070E0812F0E94A64627E0CC
:100210002C9DC0012D9D900D11249C0120583E4E17
:100220007901F9011182108222E030E0AE01415FD4
:100230005F4F68E270E0812F0E94F4578F859889A4
:10024000982789279827F70193838283168215823E
:1002500014820E944390812F01C088E060960FB6FF
:10026000F894DEBF0FBECDBFDF91CF911F910F91EC
:10027000FF90EF90DF90CF90BF90AF909F908F90C6
:100280000895FC01A089B1898C91A689B78982FD66
:100290000FC09C91818D8F5F8F73228D821749F0E3
:1002A000218DDF01A20FB11D5D969C93818F089572
:1002B0008C910895CF93DF93282F30E0F901EB5212
:1002C000F64F8491F901E159F74FD491F901EB54BC
:1002D000F74FC491CC2389F081119DDCEC2FF0E025
:1002E000EE0FFF1FE554F64FA591B491EC91ED236D
:1002F00081E090E021F480E002C080E090E0DF91B6
:10030000CF9108951F93CF93DF93282F30E0F90109
:10031000EB52F64F8491F901E159F74FD491F9016D
:10032000EB54F74FC491CC23B9F0162F811173DC35
:10033000EC2FF0E0EE0FFF1FE55CF74FA591B491B5
:100340009FB7F894111104C08C91D095D82302C0A6
:10035000EC91DE2BDC939FBFDF91CF911F9108952D
:100360001092CD111092CC1110923411109256119E
:100370001092321181E08093311110920C1161E0E2
:1003800084E1C0DF61E085E1BDDFE9EBF0E0808181
:100390008E7F808380818D7F808388E48093B80006
:1003A00085E48093BC0081E79CE49093CB1180931B
:1003B000CA1182E79CE49093C9118093C8110895F3
:1003C000CF93DF9390E0FC01E159F74F2491FC01BA
:1003D000EB54F74F8491882361F190E0880F991FC7
:1003E000FC01EB5AF74FC591D491FC01E55CF74F46
:1003F000A591B491611109C09FB7F89488812095A7
:1004000082238883EC912E230BC0623061F49FB766
:10041000F8948881322F309583238883EC912E2B9A
:100420002C939FBF06C08FB7F894E8812E2B2883AA
:100430008FBFDF91CF9108953FB7F89480917C11E1
:1004400090917D11A0917E11B0917F1126B5A89B4E
:1004500005C02F3F19F00196A11DB11D3FBFBA2F56
:10046000A92F982F8827820F911DA11DB11DBC01B6
:10047000CD0142E0660F771F881F991F4A95D1F77B
:1004800008958F929F92AF92BF92CF92DF92EF9298
:10049000FF926B017C01D0DF4B015C01C114D104E0
:1004A000E104F104E9F0C8DFDC01CB018819990906
:1004B000AA09BB09883E9340A105B10578F321E064
:1004C000C21AD108E108F10888EE880E83E0981E70
:1004D000A11CB11CC114D104E104F10421F7DECF49
:1004E000FF90EF90DF90CF90BF90AF909F908F9054
:1004F00008952FB7F89460917811709179118091D7
:100500007A1190917B112FBF08952F923F924F92B5
:100510005F926F927F928F929F92AF92BF92CF9293
:10052000DF92EF92FF920F931F93CF93DF9300D050
:100530001F92CDB7DEB79C838B834090850250908D
:100540008602EFE0F2E081E090E0212C312C4816A9
:10055000590654F0219131912130310519F42FEFD2
:10056000221A320A0196F3CF8B819C811816190644
:100570002CF4481659063CF02C0109C0E1E0F0E0EB
:10058000FC83EB8304C021E030E03C832B838B8130
:100590009C81880F991FFC01EC52F54F3F019C0193
:1005A0002D5E3D4F4901FC01E35FFD4F7F019C0142
:1005B00021583D4F59018B819C81880F991F880FCD
:1005C000991FFC01EF5FFD4F6F018C01075E1D4F0E
:1005D0009C0123573D4F3A8329838B819C81481688
:1005E00059060CF4D0C0F60180819181A281B381BB
:1005F000181619061A061B0624F50E94254EF80146
:100600002081318142815381DC01CB01821B930B1C
:10061000A40BB50BF601208131814281538128174B
:1006200039074A075B0708F071C0108211821282F5
:1006300013820E94254EF801608371838283938325
:1006400065C0F50180819181F70120813181821798
:100650009307D1F0F3E02F16310414F00097A1F4C2
:10066000880F991FFC01E252FE4E6081F3018081E8
:1006700049DEF50180819181F701918380836CE2ED
:1006800071E080E090E0FDDEF80180819181A2813F
:10069000B381181619061A061B06C4F50E94254ECA
:1006A000F8012081318142815381DC01CB01821B21
:1006B000930BA40BB50BE981FA8120813181428132
:1006C0005381281739074A075B0700F5F8011082A4
:1006D000118212821382F40180819181F7012081BD
:1006E00031818217930791F06091850270918602A3
:1006F000EFE0F2E041E050E020E030E06417750701
:100700000CF5233031053CF1009729F12B813C8118
:100710002F5F3F4F3C832B8332E0630E711C82E0DE
:10072000880E911C92E0E90EF11CE2E0AE0EB11CC5
:10073000F4E0CF0ED11C0C5F1F4F29813A812C5F52
:100740003F4F49CFA191B191119711F42F5F3F4FC6
:100750004F5F5F4FD3CF880F991FFC01E252FE4ECF
:100760006081F3018081CEDDF40180819181F70108
:1007700091838083F501918380836CE271E080E056
:1007800090E07FDEC3CF0F900F900F900F90DF911E
:10079000CF911F910F91FF90EF90DF90CF90BF907E
:1007A000AF909F908F907F906F905F904F903F9011
:1007B0002F900895CF93DF93FC0124813581232B63
:1007C00069F0EC01BC0189EB93E10E94446DBE012C
:1007D00082EE91E1DF91CF910C94446DDF91CF9146
:1007E000089581E08093A9028091AA02882341F0B4
:1007F00088E08093C91860E08EEB98E10C94C04DBE
:1008000008958091AA028823F9F08091A902882393
:10081000D9F081E00E94EC788BE39FE10197F1F73A
:1008200060E080E00E94FD7863ED7AE08EEB98E175
:100830000E94576D61E080E00E94FD7863EC7AE0F1
:100840008EEB98E10C94576D0895DF92EF92FF9232
:100850000F931F93CF93DF93CDB7DEB762970FB699
:10086000F894DEBF0FBECDBF8C011092DD1162ED9A
:100870007AE0CE010D960E94386CFF24F39489EB48
:1008800093E10E94C2682091DD1118161906D4F573
:10089000211138C089EB93E10E94A0688A3041F0B1
:1008A0008D3031F0682FCE010D960E949E6A24C0D3
:1008B00089899A89892B01F1F092DD1161E97AE049
:1008C000CE0101960E94386CBE01635F7F4FCE015E
:1008D00001960E94286BBC01CE0107960E94306CE5
:1008E000CE0107960E94C38DCE0107960E94A86B89
:1008F000CE0101960E94A86B6AE070E080E090E073
:10090000C0DDBDCF211185C0E12CF12CDD24D394B5
:1009100082EE91E10E94C268181619060CF582EE6B
:1009200091E10E94A0688A3079F08D3069F0909151
:10093000DD11911109C0682FCE010D960E949E6AAB
:100940008FEFE81AF80A06C089899A89892B11F075
:10095000D092DD1165E070E080E090E092DDD8CFCC
:1009600064E170E080E090E08CDDEF2809F43DC0A8
:1009700089899A89892BC9F18091FA18882381F194
:1009800066ED76E0CE0101960E94386CBE016F5F85
:100990007F4FCE010D960E94633EF82ECE01019648
:1009A0000E94A86BF1101CC06AE97AE0CE010196A2
:1009B0000E94386CCE0101960E943B7CCE010196CC
:1009C0000E94A86BBE01635F7F4FCE0101960E941B
:1009D000306CCE010196EEDECE0101960E94A86B2E
:1009E00064E170E080E090E04CDD8091DD118111E8
:1009F00010C089899A89892B61F464E670E080E0EF
:100A000090E03FDD76DD62ED7AE0C8010E94386C4F
:100A100050C089899A89019709F045C060E279E060
:100A2000CE0107960E94386CBE01695F7F4FCE01F0
:100A30000D960E94633E811116C061EA7AE0CE01F4
:100A400001960E94386CBE016F5F7F4FCE010D96FC
:100A50000E94633EFF24F3948111F12CCE01019694
:100A60000E94A86B01C0F12CCE0107960E94A86BD2
:100A7000FF20A1F040E050E0BE01635F7F4FCE0158
:100A800001960E948C36BE016F5F7F4F8DEF95E11E
:100A90000E94C56ACE0101960E94A86B64E170E0D5
:100AA00080E090E0EEDCBE01635F7F4FC8010E94F2
:100AB000206CCE010D960E94A86BC80162960FB6FD
:100AC000F894DEBF0FBECDBFDF91CF911F910F9184
:100AD000FF90EF90DF900895BF92CF92DF92EF9258
:100AE000FF920F931F93CF93DF93CDB7DEB762973B
:100AF0000FB6F894DEBF0FBECDBF6C018B017A013B
:100B00008091AA02882309F47AC08091A9028823DF
:100B100009F475C077FF07C00095109560E0802F3D
:100B20000E94FD784DC060E080E00E94FD78E1DC2D
:100B300028EE33E040E050E00E9433B2CA01B90130
:100B400020E831E541E050E00E9455B2AB01BC0124
:100B500020E0CE0101960E94DC6BBE016F5F7F4FEB
:100B6000CE0107960E94306C6FEC78E0CE010796BC
:100B70000E94116BBC01CE010D960E94306CCE011B
:100B800007960E94A86BCE0101960E94A86BBE0139
:100B9000635F7F4F8EEB98E10E94366DB98860E00D
:100BA0008B2D0E94FD780115110511F40B2D04C049
:100BB00060E0802F0E94FD78CE010D960E94A86B08
:100BC000B6018EEB98E10E94366D62EB7AE08EEB17
:100BD00098E10E94576DF601848160E0800F0E94C9
:100BE000FD7887DC6093E8107093E9108093EA1039
:100BF0009093EB10B701FF0C880B990B42DC6296C7
:100C00000FB6F894DEBF0FBECDBFDF91CF911F911D
:100C10000F91FF90EF90DF90CF90BF900895CF930A
:100C2000DF9300D000D0CDB7DEB7EBDDCE0101966B
:100C30000E94CE364AE050E06FEF7FEFCE01019682
:100C40004BDFCE0101960E94A86B61E080E00E941C
:100C5000FD78CE0101960E9468586EEB78E1CE01D6
:100C600001960E94D86C63EA7AE08EEB98E10E94CC
:100C7000346D3FDC6093A50C7093A60C8093A70C99
:100C80009093A80C26960FB6F894DEBF0FBECDBF8A
:100C9000DF91CF9108952F923F924F925F926F9282
:100CA0007F928F929F92AF92BF92CF92DF92EF92FC
:100CB000FF920F931F93CF93DF93CDB7DEB72897A3
:100CC0000FB6F894DEBF0FBECDBF67E370E0809132
:100CD0008702909188020E94FD3284E1482E512CB7
:100CE000612C712C212C312C8FEF281A380AC3016A
:100CF000B201C7DB67E370E08091870290918802C0
:100D00000E94FD328C0183E02816310434F08EE11C
:100D10002816310444F4012B51F084E1480E511C93
:100D2000611C711CE1CF0115110509F082C0809191
:100D30008702909188028B30910589F480903E184B
:100D400090903F18A0904018B0904118C0903A1869
:100D5000D0903B18E0903C18F0903D1815C08631BB
:100D6000910561F30C9781F48090D4119090D51186
:100D7000A090D611B090D711C090D011D090D111C1
:100D8000E090D211F090D31164E670E080E090E042
:100D900078DB6FEA7AE0CE0101960E94286CCE01E2
:100DA00001960E94DA7DCE0101960E94A86B61E057
:100DB00082E00E94FD7821E0B501A401CE010196F8
:100DC0000E94AD6BBE016F5F7F4F8EEB98E10E947A
:100DD000366DCE0101960E94A86B6FED8EEB98E107
:100DE0000E94E94D6AEA7AE08EEB98E10E94576D25
:100DF00020E0B701A601CE0101960E94AD6BBE01B5
:100E00006F5F7F4F8EEB98E10E94366DCE010196A9
:100E10000E94A86B67EA7AE08EEB98E10E94346D3D
:100E200089829A82AB82BC82CD82DE82EF82F88692
:100E300069C00F3F8FEF1807A4F06CE97AE0CE018C
:100E400001960E94286C4AE050E060E070E0CE011C
:100E5000019642DECE0101960E94A86B69E77AE016
:100E600045C00E3F8FEF180771F16BE67AE0CE01B7
:100E700001960E94286C4AE050E060E070E0CE01EC
:100E800001962ADECE0101960E94A86B6CE57AE0FD
:100E900081EF95E10E94396BB801CE0101960E9465
:100EA000E97ABE016F5F7F4F81EF95E10E94BF6AD3
:100EB000CE0101960E94A86B66E47AE081EF95E18D
:100EC0000E946F6A17C06BE37AE0CE0101960E9420
:100ED000286C4AE050E060E070E0CE010196FCDD55
:100EE000CE0101960E94A86B6BE17AE081EF95E15B
:100EF0000E94396B19821A821B821C821D821E82FB
:100F00001F82188629813A814B815C816D817E81A7
:100F10008F81988528960FB6F894DEBF0FBECDBF9F
:100F2000DF91CF911F910F91FF90EF90DF90CF90C5
:100F3000BF90AF909F908F907F906F905F904F90F9
:100F40003F902F9008951F93CF93DF93CDB7DEB7D7
:100F50002C970FB6F894DEBF0FBECDBFFE0173967F
:100F6000219131913093860220938502A4EDBAE05D
:100F700080E090E02817390734F0419151914D936A
:100F80005D930196F7CF8B8D9C8D9093DF118093AD
:100F9000DE118D8D9E8D9093E1118093E011AC96C2
:100FA0008FADAC97BE0165597F4F8F3239F4CE01BA
:100FB00007960E94386C63E774E006C0CE0107967E
:100FC0000E94386C68E774E0CE0101960E94386C8C
:100FD000BE01695F7F4FCE0101960E94286BBC0164
:100FE00086E698E10E94936BCE0101960E94A86B61
:100FF000CE0107960E94A86B66E678E1CE010196C5
:101000000E94306CCE010196D5DBCE0101960E9484
:10101000A86B69E874E0CE0101960E94386CBE01AD
:101020006F5F7F4F86E698E10E942363182FCE0101
:1010300001960E94A86B40916A1850916B18112379
:10104000A1F0BA016250710986E698E10E945E6AD9
:10105000682FCE0101960E94086CBE016F5F7F4F22
:1010600088E498E10E94C56A24C04150510966E6AF
:1010700078E1CE0101960E948C36BE016F5F7F4FF2
:1010800088E498E10E94C56ACE0101960E94A86B8F
:1010900066E678E1CE0101960E94306C69E874E062
:1010A000CE0101960E94116BBC0186E698E10E9478
:1010B000936BCE0101960E94A86B64E477E1CE01A8
:1010C00007960E94386C61E974E0CE0101960E9497
:1010D000386CBE01695F7F4FCE0101960E94286B7C
:1010E000BC0180E698E10E94936BCE0101960E94BC
:1010F000A86BCE0107960E94A86B23968FAD23970D
:101100001F928F9322968FAD22971F928F932196D5
:101110008FAD21971F928F938FAD1F928F9386E390
:101120009AE09F938F9382EC9BE09F938F930E9412
:1011300065B6CF52DF4F88819981C15DD0409093D1
:10114000880280938702BE016D527F4FCE010196C7
:101150000E94386CBE016F5F7F4F8AE598E10E9464
:10116000C56ACE0101960E94A86BBE0162527F4FF4
:10117000CE0101960E94386CBE016F5F7F4F84E5FF
:1011800098E10E94C56ACE0101960E94A86B409129
:101190005818509159184250510964E578E1CE0130
:1011A00001960E948C36CE0101960E94344C6C59F7
:1011B0006093A802CE0101960E94A86BCD5EDE4F1F
:1011C000688179818A819B81C351D1400E94FBB0A3
:1011D0000FB6F894DEBF0FBECDBF9B01AC010E94DD
:1011E00092B3882389F08CE390E0A0E0B0E0CD5E7C
:1011F000DE4F88839983AA83BB83C351D140CE5EDF
:10120000DE4F1882C251D140CE5EDE4F8881C2517E
:10121000D140882399F0CD5EDE4F88819981AA81E3
:10122000BB81C351D1408093990290939A02A093BD
:101230009B02B0939C0281E080933E0B88E2FE010A
:10124000E651FF4FA2EEBAE001900D928A95E1F7C8
:10125000CF5CDE4F88819981AA81BB81C153D14087
:101260008093BF029093C002A093C102B093C202C8
:10127000CB5CDE4F88819981AA81BB81C553D14067
:101280008093AD029093AE02A093AF02B093B002F0
:101290002C960FB6F894DEBF0FBECDBFDF91CF9175
:1012A0001F910895EF92FF920F931F93CF93DF93B7
:1012B000CDB7DEB7E8970FB6F894DEBF0FBECDBF4F
:1012C00062ED7AE0CE0187960E94386C62ED7AE09A
:1012D000CE018D960E94386C02E010E024961FAF7C
:1012E0000EAF249786E0E1E6F3E0DE01D3960190AD
:1012F0000D928A95E1F786E0FE01F396DE01AC5B84
:10130000BF4F01900D928A95E1F72C961FAE1EAE4D
:101310002C97EE24E394F12C2E96FFAEEEAE2E9792
:1013200088E0E7E6F3E0DE01599601900D928A9598
:10133000E1F788E0FE017996DE01A25BBF4F0190E4
:101340000D928A95E1F788E1EFE6F3E0DE01119670
:1013500001900D928A95E1F788E1FE013196DE0158
:10136000AA5ABF4F01900D928A95E1F780918703A9
:1013700090918803A0918903B0918A03E2968CAF83
:101380009DAFAEAFBFAFE29769EA7AE0CE01879634
:101390000E947E6B60E0CE0187960E949E6A4BA5FC
:1013A0005CA5BE016E587F4FCE0187960E942D3EF0
:1013B0006AEF7AE0CE018D960E94396B67E179E0A1
:1013C00088E498E10E947E6B60E0CE018D960E94D9
:1013D0009E6A49A95AA9BE0166567F4FCE018D96D5
:1013E0000E942D3E62ED7AE0CE0187960E947E6BD0
:1013F00062ED7AE0CE018D960E947E6BC250DF4F87
:1014000019821882CE5FD040809187029091880225
:10141000C050DF4F99838883C050D14080E090E076
:10142000A0E7B2E4CA5BDE4F88839983AA83BB83BB
:10143000C654D140C65BDE4F19830883CA54D140DD
:1014400080E090E0A0E2B2E4C45BDE4F8883998341
:10145000AA83BB83CC54D14080E090E0A4E3B2E403
:10146000C05BDE4F88839983AA83BB83C055D1407C
:1014700084EB90E0CC5ADE4F99838883C455D140E9
:1014800088E790E0CA5ADE4F99838883C655D140D9
:101490008CE291E0A0E0B0E0C85ADE4F88839983E7
:1014A000AA83BB83C855D140C45ADE4FF982E88273
:1014B000CC55D140C25ADE4F19830883CE55D14056
:1014C00060E08AE598E10E949E6A60E084E598E128
:1014D0000E949E6A40915E1850915F18BE016E5F37
:1014E0007E4F8AE598E10E942D3E40915818509118
:1014F0005918BE01635F7E4F84E598E10E942D3E3E
:1015000088E2E2EEFAE0DE01A75EBE4F01900D92A6
:101510008A95E1F78CE390E0A0E0B0E0CE5BDE4F8F
:1015200088839983AA83BB83C254D140CF5BDE4FAB
:101530001882C154D14084EE98E3AEE8B2E4C05AB8
:10154000DE4F88839983AA83BB83C056D14084EE43
:1015500098E3AEE8B1E4CC59DE4F88839983AA833F
:10156000BB83C456D14084EF91E09093AC0280934A
:10157000AB02BE016E5B7F4F8AD564EF71E080E005
:1015800090E00E94418263EE7AE0CE0181960E9453
:10159000286CCE0181960ED9CE0181960E94A86B4F
:1015A000CE018D960E94A86BCE0187960E94A86BF3
:1015B000E8960FB6F894DEBF0FBECDBFDF91CF9196
:1015C0001F910F91FF90EF900895EF92FF920F936C
:1015D0001F93CF93DF93CDB7DEB768970FB6F8941C
:1015E000DEBF0FBECDBF62ED7AE0CE0143960E9412
:1015F000386C6AED7BE0CE0101960E94286CCE012A
:1016000001960E943B7CCE0101960E94A86B6AA1C4
:101610007BA1CE0101960E94E97ACE010196CAD83B
:10162000CE0101960E94A86B6DEC7BE0CE01019685
:101630000E94286CCE0101960E943B7CCE0101964F
:101640000E94A86B7E0186E2E80EF11C01E010E02A
:101650008AA19BA1801791070CF1F701619171910B
:101660007F01CE0101960E94E97ACE0101960E9487
:101670003B7CCE0101960E94A86B6AE175E0CE0129
:1016800001960E94386CCE0101960E943B7CCE01EF
:1016900001960E94A86B0F5F1F4FDACF6AE175E0D9
:1016A000CE0101960E94386CCE01019683D8CE01FE
:1016B00001960E94A86B6EEB7BE0CE0101960E9422
:1016C000286CCE0101960E943B7CCE0101960E94BF
:1016D000A86B6091DE117091DF11CE0101960E941E
:1016E000E97ACE0101960E943B7CCE0101960E94D0
:1016F000A86B6AE175E0CE0101960E94386CCE01BC
:1017000001960E943B7CCE0101960E94A86B6091DD
:10171000E0117091E111CE0101960E94E97ACE01AB
:10172000019648D8CE0101960E94A86B67EA7BE03B
:10173000CE0101960E94286CCE0101960E943B7C4E
:10174000CE0101960E94A86BBE01625D7F4FCE0163
:1017500001960E94386CCE0101960E943B7CCE011E
:1017600001960E94A86B6AE175E0CE0101960E9485
:10177000386CCE0101960E943B7CCE0101960E94FE
:10178000A86BBE016E5C7F4FCE0101960E94386C43
:10179000CE0101960FD8CE0101960E94A86B67E991
:1017A0007BE0CE0101960E94286CCE01019602D802
:1017B000CE0101960E94A86B7E01FEE3EF0EF11CA4
:1017C00001E010E08AA19BA1801791070CF448C0AA
:1017D000B801CE0107960E94E97A66ED76E0CE0167
:1017E00001960E94386CBE01695F7F4FCE01019661
:1017F0000E94286BBC01CE010D960E94306CCE0178
:101800000D960E943B7CCE010D960E94A86BCE01E6
:1018100001960E94A86BCE0107960E94A86B66E015
:1018200076E0CE0101960E94386CCE0101960E94AE
:101830003B7CCE0101960E94A86BB701CE010196B8
:101840000E94386CCE0101960E94DA83CE01019687
:101850000E94A86B0F5F1F4F88E0E80EF11CB2CF0B
:1018600067E87BE0CE0101960E94286CCE010196CC
:101870000E943B7CCE0101960E94A86B62EC7BE04B
:10188000CE0101960E94386CCE0101960E94DA8347
:10189000CE0101960E94A86B68E77BE0CE0101961D
:1018A0000E94286CCE0101960E943B7CCE010196DD
:1018B0000E94A86BBE016E5A7F4FCE0101960E9416
:1018C000386CCE0101960E94DA83CE0101960E9407
:1018D000A86B61EB7AE0CE0101960E94386CCE01D4
:1018E00001960E943B7CCE0101960E94A86BBE012E
:1018F00066587F4FCE0101960E94386CCE0101964A
:101900000E94DA83CE0101960E94A86BC252DF4F7B
:1019100088819981CE5DD040892B71F460E77BE0AE
:10192000CE0101960E94286CCE0101960E94DA83B6
:10193000CE0101960E94A86BC252DF4F8881998127
:10194000CE5DD040019771F466E67BE0CE01019652
:101950000E94286CCE0101960E94DA83CE01019686
:101960000E94A86BC252DF4F88819981CE5DD04022
:10197000029771F46DE57BE0CE0101960E94286C20
:10198000CE0101960E94DA83CE0101960E94A86BD7
:1019900067E57BE0CE0101960E94286CCE0101969E
:1019A0000E943B7CCE0101960E94A86BC052DF4F83
:1019B00068817981C05ED040CE0101960E94E97AAB
:1019C000CE0101960E94DA83CE0101960E94A86B97
:1019D00040915F115091601160916111709162119D
:1019E00021E0CE0107960E94AD6B6FE976E0CE0153
:1019F00001960E94386CBE01695F7F4FCE0101964F
:101A00000E94286B60EB76E00E94116BBC01CE0156
:101A10000D960E94306CCE010D960E94DA83CE01A5
:101A20000D960E94A86BCE0101960E94A86BCE0174
:101A300007960E94A86B40915711509158116091E0
:101A4000591170915A1121E0CE0107960E94AD6B99
:101A500069EA76E0CE0101960E94386CBE01695FAA
:101A60007F4FCE0101960E94286B60EB76E00E94CA
:101A7000116BBC01CE010D960E94306CCE010D960B
:101A80000E94DA83CE010D960E94A86BCE010196CA
:101A90000E94A86BCE0107960E94A86B6AE37BE0C8
:101AA000CE0101960E94286CCE0101960E943B7CDB
:101AB000CE0101960E94A86B4091BF025091C002D6
:101AC0006091C1027091C20225E0CE0101960E9490
:101AD000AD6BCE0101960E94DA83CE0101960E9481
:101AE000A86B60E27BE0CE0101960E94286CCE01DB
:101AF00001960E943B7CCE0101960E94A86B40910A
:101B0000AD025091AE026091AF027091B00225E03B
:101B1000CE0101960E94AD6BCE0101960E94DA8340
:101B2000CE0101960E94A86B60E17BE0CE01019698
:101B30000E94286CCE0101960E943B7CCE0101964A
:101B40000E94A86B6091DD027091DE02CE010196C9
:101B50000E94E97ACE0101960E94DA83CE010196B5
:101B60000E94A86BCE0143960E94A86B68960FB6A0
:101B7000F894DEBF0FBECDBFDF91CF911F910F91C3
:101B8000FF90EF9008950F931F93CF93DF9300D0B2
:101B900000D0CDB7DEB72091FA182223A9F08C012E
:101BA00066ED76E0CE0101960E94386CB801CE0158
:101BB00001960E94286BBC0189EB93E10E94446D61
:101BC000CE0101960E94A86B26960FB6F894DEBF50
:101BD0000FBECDBFDF91CF911F910F9108956F92EE
:101BE0007F928F929F92AF92BF92CF92DF92EF92AD
:101BF000FF920F931F93CF93DF93CDB7DEB7C258F9
:101C0000D1090FB6F894DEBF0FBECDBF7C016B01CA
